Archive member included because of file (symbol)

C:/Program Files/Microchip/mplabc32/v1.12/bin/../lib/gcc/pic32mx/3.4.4/../../../../pic32mx/lib/size\libc.a(memset.o)
                              output_pic32_ssd1963\FSIO.o (memset)
C:/Program Files/Microchip/mplabc32/v1.12/bin/../lib/gcc/pic32mx/3.4.4/../../../../pic32mx/lib/size\libc.a(strcpy.o)
                              output_pic32_ssd1963\FSIO.o (strcpy)
C:/Program Files/Microchip/mplabc32/v1.12/bin/../lib/gcc/pic32mx/3.4.4/../../../../pic32mx/lib/size\libc.a(strlen.o)
                              output_pic32_ssd1963\FSIO.o (strlen)
C:/Program Files/Microchip/mplabc32/v1.12/bin/../lib/gcc/pic32mx/3.4.4/../../../../pic32mx/lib/size\libc.a(general-exception.o)
                              C:/Program Files/Microchip/mplabc32/v1.12/bin/../lib/gcc/pic32mx/3.4.4/../../../../pic32mx/lib/size/crt0.o (_general_exception_context)
C:/Program Files/Microchip/mplabc32/v1.12/bin/../lib/gcc/pic32mx/3.4.4/../../../../pic32mx/lib/size\libc.a(ctypef.o)
                              output_pic32_ssd1963\FSIO.o (tolower)
C:/Program Files/Microchip/mplabc32/v1.12/bin/../lib/gcc/pic32mx/3.4.4/../../../../pic32mx/lib/size\libc.a(malloc.o)
                              output_pic32_ssd1963\Window.o (malloc)
C:/Program Files/Microchip/mplabc32/v1.12/bin/../lib/gcc/pic32mx/3.4.4/../../../../pic32mx/lib/size\libc.a(memcpy.o)
                              C:/Program Files/Microchip/mplabc32/v1.12/bin/../lib/gcc/pic32mx/3.4.4/../../../../pic32mx/lib/size\libc.a(malloc.o) (memcpy)
C:/Program Files/Microchip/mplabc32/v1.12/bin/../lib/gcc/pic32mx/3.4.4/../../../../pic32mx/lib/size\libc.a(rand.o)
                              output_pic32_ssd1963\Games.o (srand)
C:/Program Files/Microchip/mplabc32/v1.12/bin/../lib/gcc/pic32mx/3.4.4/../../../../pic32mx/lib/size\libc.a(strchr.o)
                              output_pic32_ssd1963\FSIO.o (strchr)
C:/Program Files/Microchip/mplabc32/v1.12/bin/../lib/gcc/pic32mx/3.4.4/../../../../pic32mx/lib/size\libc.a(strncpy.o)
                              output_pic32_ssd1963\FSIO.o (strncpy)
C:/Program Files/Microchip/mplabc32/v1.12/bin/../lib/gcc/pic32mx/3.4.4/../../../../pic32mx/lib/size\libc.a(sbrk.o)
                              C:/Program Files/Microchip/mplabc32/v1.12/bin/../lib/gcc/pic32mx/3.4.4/../../../../pic32mx/lib/size\libc.a(malloc.o) (sbrk)
C:/Program Files/Microchip/mplabc32/v1.12/bin/../lib/gcc/pic32mx/3.4.4/../../../../pic32mx/lib/size\libc.a(default-general-exception-handler.o)
                              C:/Program Files/Microchip/mplabc32/v1.12/bin/../lib/gcc/pic32mx/3.4.4/../../../../pic32mx/lib/size\libc.a(general-exception.o) (_general_exception_handler)
C:/Program Files/Microchip/mplabc32/v1.12/bin/../lib/gcc/pic32mx/3.4.4/../../../../pic32mx/lib/size\libc.a(default-bootstrap-exception-handler.o)
                              C:/Program Files/Microchip/mplabc32/v1.12/bin/../lib/gcc/pic32mx/3.4.4/../../../../pic32mx/lib/size/crt0.o (_bootstrap_exception_handler)
C:/Program Files/Microchip/mplabc32/v1.12/bin/../lib/gcc/pic32mx/3.4.4/../../../../pic32mx/lib/size\libc.a(default-on-reset.o)
                              C:/Program Files/Microchip/mplabc32/v1.12/bin/../lib/gcc/pic32mx/3.4.4/../../../../pic32mx/lib/size/crt0.o (_on_reset)
C:/Program Files/Microchip/mplabc32/v1.12/bin/../lib/gcc/pic32mx/3.4.4/../../../../pic32mx/lib/size\libc.a(default-on-bootstrap.o)
                              C:/Program Files/Microchip/mplabc32/v1.12/bin/../lib/gcc/pic32mx/3.4.4/../../../../pic32mx/lib/size/crt0.o (_on_bootstrap)
C:/Program Files/Microchip/mplabc32/v1.12/bin/../lib/gcc/pic32mx/3.4.4/../../../../pic32mx/lib/size\libc.a(default-nmi-handler.o)
                              C:/Program Files/Microchip/mplabc32/v1.12/bin/../lib/gcc/pic32mx/3.4.4/../../../../pic32mx/lib/size/crt0.o (_nmi_handler)
C:/Program Files/Microchip/mplabc32/v1.12/bin/../lib/gcc/pic32mx/3.4.4/../../../../pic32mx/lib/size\libc.a(ctype.o)
                              C:/Program Files/Microchip/mplabc32/v1.12/bin/../lib/gcc/pic32mx/3.4.4/../../../../pic32mx/lib/size\libc.a(ctypef.o) (_ctype)
C:/Program Files/Microchip/mplabc32/v1.12/bin/../lib/gcc/pic32mx/3.4.4/../../../../pic32mx/lib/size\libc.a(errno.o)
                              C:/Program Files/Microchip/mplabc32/v1.12/bin/../lib/gcc/pic32mx/3.4.4/../../../../pic32mx/lib/size\libc.a(sbrk.o) (errno)
C:/Program Files/Microchip/mplabc32/v1.12/bin/../lib/gcc/pic32mx/3.4.4/../../../../pic32mx/lib/size\libm.a(fp32.o)
                              output_pic32_ssd1963\Meter.o (fpmul)
C:/Program Files/Microchip/mplabc32/v1.12/bin/../lib/gcc/pic32mx/3.4.4/../../../../pic32mx/lib/size\libm.a(fpcos32.o)
                              output_pic32_ssd1963\Meter.o (cosf)
C:/Program Files/Microchip/mplabc32/v1.12/bin/../lib/gcc/pic32mx/3.4.4/../../../../pic32mx/lib/size\libm.a(fpsin32.o)
                              output_pic32_ssd1963\Meter.o (sinf)
C:/Program Files/Microchip/mplabc32/v1.12/bin/../lib/gcc/pic32mx/3.4.4/../../../../pic32mx/lib/size\libm.a(fpreduct32.o)
                              C:/Program Files/Microchip/mplabc32/v1.12/bin/../lib/gcc/pic32mx/3.4.4/../../../../pic32mx/lib/size\libm.a(fpcos32.o) (fpreduct)
C:/Program Files/Microchip/mplabc32/v1.12/bin/../lib/gcc/pic32mx/3.4.4/../../../../pic32mx/lib/size\libm.a(sincof32.o)
                              C:/Program Files/Microchip/mplabc32/v1.12/bin/../lib/gcc/pic32mx/3.4.4/../../../../pic32mx/lib/size\libm.a(fpcos32.o) (_sincof)
C:/Program Files/Microchip/mplabc32/v1.12/bin/../lib/gcc/pic32mx/3.4.4/../../../../pic32mx/lib/size\libmchp_peripheral.a(open_core_timer_lib.o)
                              output_pic32_ssd1963\DisplayDriver.o (OpenCoreTimer)
C:/Program Files/Microchip/mplabc32/v1.12/bin/../lib/gcc/pic32mx/3.4.4/../../../../pic32mx/lib/size\libmchp_peripheral_32MX360F512L.a(pcache.o)
                              output_pic32_ssd1963\MainDemo.o (CheKseg0CacheOn)
C:/Program Files/Microchip/mplabc32/v1.12/bin/../lib/gcc/pic32mx/3.4.4/../../../../pic32mx/lib/size\libmchp_peripheral_32MX360F512L.a(int_disable_interrupts_lib.o)
                              output_pic32_ssd1963\MainDemo.o (INTDisableInterrupts)
C:/Program Files/Microchip/mplabc32/v1.12/bin/../lib/gcc/pic32mx/3.4.4/../../../../pic32mx/lib/size\libmchp_peripheral_32MX360F512L.a(int_restore_interrupts_lib.o)
                              output_pic32_ssd1963\MainDemo.o (INTRestoreInterrupts)
C:/Program Files/Microchip/mplabc32/v1.12/bin/../lib/gcc/pic32mx/3.4.4/../../../../pic32mx/lib/size\libmchp_peripheral_32MX360F512L.a(int_enable_mv_int_lib.o)
                              output_pic32_ssd1963\MainDemo.o (INTEnableSystemMultiVectoredInt)
C:/Program Files/Microchip/mplabc32/v1.12/bin/../lib/gcc/pic32mx/3.4.4/../../../../pic32mx/lib/size\libmchp_peripheral_32MX360F512L.a(rtcc_init_lib.o)
                              output_pic32_ssd1963\rtcc.o (RtccInit)
C:/Program Files/Microchip/mplabc32/v1.12/bin/../lib/gcc/pic32mx/3.4.4/../../../../pic32mx/lib/size\libmchp_peripheral_32MX360F512L.a(rtcc_set_date_lib.o)
                              output_pic32_ssd1963\rtcc.o (RtccSetDate)
C:/Program Files/Microchip/mplabc32/v1.12/bin/../lib/gcc/pic32mx/3.4.4/../../../../pic32mx/lib/size\libmchp_peripheral_32MX360F512L.a(rtcc_set_time_lib.o)
                              output_pic32_ssd1963\rtcc.o (RtccSetTime)
C:/Program Files/Microchip/mplabc32/v1.12/bin/../lib/gcc/pic32mx/3.4.4/../../../../pic32mx/lib/size\libmchp_peripheral_32MX360F512L.a(spi_getc_spi2_lib_legacy.o)
                              output_pic32_ssd1963\SD-SPI.o (getcSPI2)
C:/Program Files/Microchip/mplabc32/v1.12/bin/../lib/gcc/pic32mx/3.4.4/../../../../pic32mx/lib/size\libmchp_peripheral_32MX360F512L.a(spi_open_spi2_lib_legacy.o)
                              output_pic32_ssd1963\SD-SPI.o (OpenSPI2)
C:/Program Files/Microchip/mplabc32/v1.12/bin/../lib/gcc/pic32mx/3.4.4/../../../../pic32mx/lib/size\libmchp_peripheral_32MX360F512L.a(spi_brg_tbl_lib_legacy.o)
                              C:/Program Files/Microchip/mplabc32/v1.12/bin/../lib/gcc/pic32mx/3.4.4/../../../../pic32mx/lib/size\libmchp_peripheral_32MX360F512L.a(spi_open_spi2_lib_legacy.o) (_SpiBrgConvTbl)
C:/Program Files/Microchip/mplabc32/v1.12/bin/../lib/gcc/pic32mx/3.4.4/../../../../pic32mx/lib/size\libmchp_peripheral_32MX360F512L.a(int_enable_interrupts_lib.o)
                              C:/Program Files/Microchip/mplabc32/v1.12/bin/../lib/gcc/pic32mx/3.4.4/../../../../pic32mx/lib/size\libmchp_peripheral_32MX360F512L.a(int_enable_mv_int_lib.o) (INTEnableInterrupts)
C:/Program Files/Microchip/mplabc32/v1.12/bin/../lib/gcc/pic32mx/3.4.4/../../../../pic32mx/lib/size\libmchp_peripheral_32MX360F512L.a(int_tbl_lib.o)
                              C:/Program Files/Microchip/mplabc32/v1.12/bin/../lib/gcc/pic32mx/3.4.4/../../../../pic32mx/lib/size\libmchp_peripheral_32MX360F512L.a(rtcc_init_lib.o) (INTClearFlag)
C:/Program Files/Microchip/mplabc32/v1.12/bin/../lib/gcc/pic32mx/3.4.4/../../../../pic32mx/lib/size\libmchp_peripheral_32MX360F512L.a(_rtcc_set_time_and_date_lib.o)
                              C:/Program Files/Microchip/mplabc32/v1.12/bin/../lib/gcc/pic32mx/3.4.4/../../../../pic32mx/lib/size\libmchp_peripheral_32MX360F512L.a(rtcc_set_date_lib.o) (_RtccSetTimeAndDate)
C:/Program Files/Microchip/mplabc32/v1.12/bin/../lib/gcc/pic32mx/3.4.4/../../../../pic32mx/lib/size\libmchp_peripheral_32MX360F512L.a(_rtcc_wait_clock_off_lib.o)
                              C:/Program Files/Microchip/mplabc32/v1.12/bin/../lib/gcc/pic32mx/3.4.4/../../../../pic32mx/lib/size\libmchp_peripheral_32MX360F512L.a(rtcc_init_lib.o) (_RtccWaitClockOff)
C:/Program Files/Microchip/mplabc32/v1.12/bin/../lib/gcc/pic32mx/3.4.4/../../../../pic32mx/lib/size\libmchp_peripheral_32MX360F512L.a(read_core_timer_lib.o)
                              C:/Program Files/Microchip/mplabc32/v1.12/bin/../lib/gcc/pic32mx/3.4.4/../../../../pic32mx/lib/size\libmchp_peripheral_32MX360F512L.a(_rtcc_wait_clock_off_lib.o) (ReadCoreTimer)

Allocating common symbols
Common symbol       size              file

_cursorY            0x2               output_pic32_ssd1963\Primitive.o
deltaR              0x1               output_pic32_ssd1963\RGBDemo.o
ecgVerX2            0x2               output_pic32_ssd1963\ECG.o
snake               0x264             output_pic32_ssd1963\Games.o
_rpnlX2             0x2               output_pic32_ssd1963\GOL.o
gDataBuffer         0x200             output_pic32_ssd1963\FSIO.o
LabelColorScheme    0x4               output_pic32_ssd1963\RGBDemo.o
RedLim              0x1               output_pic32_ssd1963\RGBDemo.o
_activePage         0x1               output_pic32_ssd1963\DisplayDriver.o
gEnableDemoFlag     0x4               output_pic32_ssd1963\DemoSteps.o
IMG_wWidth          0x2               output_pic32_ssd1963\ImageDecoder.o
ecgVerY1            0x2               output_pic32_ssd1963\ECG.o
ecgHorY1            0x2               output_pic32_ssd1963\ECG.o
HWLang              0x90              output_pic32_ssd1963\MultiFontsDemo.o
IMG_bAlignCenter    0x1               output_pic32_ssd1963\ImageDecoder.o
gFileSlotOpen       0x3               output_pic32_ssd1963\FSIO.o
IMG_wStartX         0x2               output_pic32_ssd1963\ImageDecoder.o
gTimeCrtMS          0x1               output_pic32_ssd1963\FSIO.o
iconScheme          0x4               output_pic32_ssd1963\MainDemo.o
MDD_SDSPI_finalLBA  0x4               output_pic32_ssd1963\SD-SPI.o
_fontOrientation    0x1               output_pic32_ssd1963\Primitive.o
chartType           0x4               output_pic32_ssd1963\GraphShow.o
_fontFirstChar      0x2               output_pic32_ssd1963\Primitive.o
cwd                 0x3c              output_pic32_ssd1963\FSIO.o
PixArray            0x24              output_pic32_ssd1963\SlideShowDemo.o
IMG_wHeight         0x2               output_pic32_ssd1963\ImageDecoder.o
navScheme           0x4               output_pic32_ssd1963\MainDemo.o
defaultString       0xd               output_pic32_ssd1963\FSIO.o
_rpnlR              0x2               output_pic32_ssd1963\GOL.o
usbErrorCode        0x1               output_pic32_ssd1963\MainDemo.o
IMG_bDownScalingFactor
                    0x1               output_pic32_ssd1963\ImageDecoder.o
RedMin              0x1               output_pic32_ssd1963\RGBDemo.o
RedMax              0x1               output_pic32_ssd1963\RGBDemo.o
deltaB              0x1               output_pic32_ssd1963\RGBDemo.o
_rtcc_flag          0x1               output_pic32_ssd1963\rtcc.o
tempCWDobj          0x3c              output_pic32_ssd1963\FSIO.o
altScheme           0x4               output_pic32_ssd1963\MainDemo.o
IMG_wStartY         0x2               output_pic32_ssd1963\ImageDecoder.o
_clipRgn            0x2               output_pic32_ssd1963\DisplayDriver.o
_fontHeight         0x2               output_pic32_ssd1963\Primitive.o
gMediaSectorSize    0x2               output_pic32_ssd1963\SD-SPI.o
pNavList            0x4               output_pic32_ssd1963\MainDemo.o
vs1003TestWord      0x2               output_pic32_ssd1963\MainDemo.o
MoScheme            0x4               output_pic32_ssd1963\TimeDateDemo.o
IMG_wImageWidth     0x2               output_pic32_ssd1963\ImageDecoder.o
IMG_wImageHeight    0x2               output_pic32_ssd1963\ImageDecoder.o
tempBuffer          0x14              output_pic32_ssd1963\ECG.o
_cursorX            0x2               output_pic32_ssd1963\Primitive.o
pScore              0x4               output_pic32_ssd1963\Games.o
pHWData             0x4               output_pic32_ssd1963\MultiFontsDemo.o
_rpnlX1             0x2               output_pic32_ssd1963\GOL.o
graphScheme         0x4               output_pic32_ssd1963\MainDemo.o
_fontLastChar       0x2               output_pic32_ssd1963\Primitive.o
FadeDirGreen        0x1               output_pic32_ssd1963\RGBDemo.o
_font               0x4               output_pic32_ssd1963\Primitive.o
FadeModeEnable      0x1               output_pic32_ssd1963\RGBDemo.o
_visualPage         0x1               output_pic32_ssd1963\DisplayDriver.o
RGBBlueScheme       0x4               output_pic32_ssd1963\RGBDemo.o
_lineType           0x2               output_pic32_ssd1963\Primitive.o
GreenMax            0x1               output_pic32_ssd1963\RGBDemo.o
gFATBuffer          0x200             output_pic32_ssd1963\FSIO.o
ControlColorScheme  0x4               output_pic32_ssd1963\RGBDemo.o
score               0x2               output_pic32_ssd1963\Games.o
gTimeCrtTime        0x2               output_pic32_ssd1963\FSIO.o
gFileArray          0xb4              output_pic32_ssd1963\FSIO.o
FatRootDirClusterValue
                    0x4               output_pic32_ssd1963\FSIO.o
FontScheme2         0x4               output_pic32_ssd1963\MultiFontsDemo.o
sdCardStatus        0x1               output_pic32_ssd1963\DemoSelection.o
pPicture            0x4               output_pic32_ssd1963\Animation.o
ecgBuffer           0x200             output_pic32_ssd1963\ECG.o
pMonth              0x4               output_pic32_ssd1963\TimeDateDemo.o
gDiskData           0x26              output_pic32_ssd1963\FSIO.o
_clipRight          0x2               output_pic32_ssd1963\DisplayDriver.o
FadeDirRed          0x1               output_pic32_ssd1963\RGBDemo.o
PolyPoints          0x20              output_pic32_ssd1963\RGBDemo.o
gTimeWrtDate        0x2               output_pic32_ssd1963\FSIO.o
demoCount           0x2               output_pic32_ssd1963\DemoSteps.o
pPixData            0x4               output_pic32_ssd1963\SlideShowDemo.o
deltaG              0x1               output_pic32_ssd1963\RGBDemo.o
DemoTitle           0x3c              output_pic32_ssd1963\GraphShow.o
pWkDay              0x4               output_pic32_ssd1963\TimeDateDemo.o
dumScheme           0x4               output_pic32_ssd1963\TimeDateDemo.o
UpdateCurrent       0x1               output_pic32_ssd1963\RGBDemo.o
ecgHorX1            0x2               output_pic32_ssd1963\ECG.o
ecgHorX2            0x2               output_pic32_ssd1963\ECG.o
buffer              0xc               output_pic32_ssd1963\ECG.o
MinScheme           0x4               output_pic32_ssd1963\TimeDateDemo.o
IMG_blAbortImageDecoding
                    0x1               output_pic32_ssd1963\ImageDecoder.o
BlueMax             0x1               output_pic32_ssd1963\RGBDemo.o
_clipBottom         0x2               output_pic32_ssd1963\DisplayDriver.o
_time               0x10              output_pic32_ssd1963\rtcc.o
demoTick            0x4               output_pic32_ssd1963\DemoSelection.o
usbHIDStatus        0x1               output_pic32_ssd1963\MainDemo.o
UpdateColor         0x1               output_pic32_ssd1963\RGBDemo.o
_rpnlEmbossDkColor  0x2               output_pic32_ssd1963\GOL.o
Preset1ColorScheme  0x4               output_pic32_ssd1963\RGBDemo.o
RGBGreenScheme      0x4               output_pic32_ssd1963\RGBDemo.o
RGBRedScheme        0x4               output_pic32_ssd1963\RGBDemo.o
ecgVerX1            0x2               output_pic32_ssd1963\ECG.o
gTimeCrtDate        0x2               output_pic32_ssd1963\FSIO.o
scoreInfo           0x34              output_pic32_ssd1963\Games.o
_rpnlEmbossSize     0x2               output_pic32_ssd1963\GOL.o
GreenMin            0x1               output_pic32_ssd1963\RGBDemo.o
_clipTop            0x2               output_pic32_ssd1963\DisplayDriver.o
_time_chk           0x10              output_pic32_ssd1963\rtcc.o
_color              0x2               output_pic32_ssd1963\DisplayDriver.o
SlideShowScheme     0x4               output_pic32_ssd1963\SlideShowDemo.o
FadeDirBlue         0x1               output_pic32_ssd1963\RGBDemo.o
SecScheme           0x4               output_pic32_ssd1963\TimeDateDemo.o
pMeter              0x4               output_pic32_ssd1963\Animation.o
prevDemoTime        0x4               output_pic32_ssd1963\DemoSteps.o
GreenLim            0x1               output_pic32_ssd1963\RGBDemo.o
TempClusterCalc     0x4               output_pic32_ssd1963\FSIO.o
_clipLeft           0x2               output_pic32_ssd1963\DisplayDriver.o
gamesGrid           0x4               output_pic32_ssd1963\Games.o
dirCleared          0x1               output_pic32_ssd1963\FSIO.o
_rpnlY2             0x2               output_pic32_ssd1963\GOL.o
_rpnlEmbossLtColor  0x2               output_pic32_ssd1963\GOL.o
usbMSDStatus        0x1               output_pic32_ssd1963\MainDemo.o
BlueLim             0x1               output_pic32_ssd1963\RGBDemo.o
ecgVerY2            0x2               output_pic32_ssd1963\ECG.o
meterScheme         0x4               output_pic32_ssd1963\MainDemo.o
gFileTemp           0x3c              output_pic32_ssd1963\FSIO.o
dTypeCnt            0x2               output_pic32_ssd1963\GraphShow.o
pScoreText          0x4               output_pic32_ssd1963\Games.o
pulseCounter        0x2               output_pic32_ssd1963\Beep.o
_rpnlFaceColor      0x2               output_pic32_ssd1963\GOL.o
defaultDirection    0x2               output_pic32_ssd1963\Games.o
IMG_pLoopCallbackFn
                    0x4               output_pic32_ssd1963\ImageDecoder.o
balls               0x18              output_pic32_ssd1963\Games.o
defaultArray        0xa               output_pic32_ssd1963\FSIO.o
field               0x1100            output_pic32_ssd1963\Games.o
_rpnlY1             0x2               output_pic32_ssd1963\GOL.o
gridScheme          0x4               output_pic32_ssd1963\MainDemo.o
_lineThickness      0x1               output_pic32_ssd1963\Primitive.o
gSDMode             0x1               output_pic32_ssd1963\SD-SPI.o
updateIntensity     0x1               output_pic32_ssd1963\RGBDemo.o
BlueMin             0x1               output_pic32_ssd1963\RGBDemo.o
Preset2ColorScheme  0x4               output_pic32_ssd1963\RGBDemo.o
DayScheme           0x4               output_pic32_ssd1963\TimeDateDemo.o
pScoreInfo          0x4               output_pic32_ssd1963\Games.o
HourScheme          0x4               output_pic32_ssd1963\TimeDateDemo.o
gTimeAccDate        0x2               output_pic32_ssd1963\FSIO.o
WkDayScheme         0x4               output_pic32_ssd1963\TimeDateDemo.o
FSerrno             0x1               output_pic32_ssd1963\FSIO.o
ecgHorY2            0x2               output_pic32_ssd1963\ECG.o
gTimeWrtTime        0x2               output_pic32_ssd1963\FSIO.o

Microchip PIC32 Memory-Usage Report

kseg0 Program-Memory Usage
section                    address  length [bytes]      (dec)  Description
-------                 ----------  -------------------------  -----------
.text                   0x9d000000        0x1b754      112468  Application's executable code 
.rodata                 0x9d01b754        0x43620      276000  Read-only constant data 
.data                   0x9d05ed74          0x1a8         424  Data-initialization template 
.sdata                  0x9d05ef1c          0x15c         348  Small data-initialization template 
      Total kseg0_program_mem used  :     0x5f078      389240  74.2% of 0x80000

kseg0 Boot-Memory Usage
section                    address  length [bytes]      (dec)  Description
-------                 ----------  -------------------------  -----------
.startup                0x9fc00490          0x1e0         480  C startup code 
         Total kseg0_boot_mem used  :       0x1e0         480  19.9% of 0x970

Exception-Memory Usage 
section                    address  length [bytes]      (dec)  Description
-------                 ----------  -------------------------  -----------
.app_excpt              0x9fc01180           0x10          16  General-Exception handler 
.vector_8               0x9fc01300            0x8           8  Interrupt Vector 8 
.vector_12              0x9fc01380            0x8           8  Interrupt Vector 12 
.vector_16              0x9fc01400            0x8           8  Interrupt Vector 16 
          Total exception_mem used  :        0x28          40  1.0% of 0x1000

kseg1 Boot-Memory Usage
section                    address  length [bytes]      (dec)  Description
-------                 ----------  -------------------------  -----------
.reset                  0xbfc00000           0x10          16  Reset handler 
.bev_excpt              0xbfc00380           0x10          16  BEV-Exception handler 
         Total kseg1_boot_mem used  :        0x20          32  2.7% of 0x490
        --------------------------------------------------------------------------
         Total Program Memory used  :     0x5f2a0      389792  73.3% of 0x81e00
        --------------------------------------------------------------------------


kseg1 Data-Memory Usage
section                    address  length [bytes]      (dec)  Description
-------                 ----------  -------------------------  -----------
.data                   0xa0000000          0x1a8         424  Initialized data 
.sdata                  0xa00001a8          0x15c         348  Small initialized data 
.sbss                   0xa0000304          0x336         822  Small uninitialized data 
.bss                    0xa000063c         0x1734        5940  Uninitialized data 
.heap                   0xa0001d70         0x2400        9216  Dynamic Memory heap 
.stack                  0xa0004170          0x800        2048  Minimum space reserved for stack 
         Total kseg1_data_mem used  :      0x496e       18798  57.4% of 0x8000
        --------------------------------------------------------------------------
            Total Data Memory used  :      0x496e       18798  57.4% of 0x8000
        --------------------------------------------------------------------------

Discarded input sections

 .data          0x00000000        0x0 C:/Program Files/Microchip/mplabc32/v1.12/bin/../lib/gcc/pic32mx/3.4.4/../../../../pic32mx/lib/size/crt0.o
 .bss           0x00000000        0x0 C:/Program Files/Microchip/mplabc32/v1.12/bin/../lib/gcc/pic32mx/3.4.4/../../../../pic32mx/lib/size/crt0.o
 .reginfo       0x00000000       0x18 C:/Program Files/Microchip/mplabc32/v1.12/bin/../lib/gcc/pic32mx/3.4.4/../../../../pic32mx/lib/size/crt0.o
 .pdr           0x00000000       0xa0 C:/Program Files/Microchip/mplabc32/v1.12/bin/../lib/gcc/pic32mx/3.4.4/../../../../pic32mx/lib/size/crt0.o
 .data          0x00000000        0x0 output_pic32_ssd1963\MainDemo.o
 .bss           0x00000000        0x0 output_pic32_ssd1963\MainDemo.o
 .reginfo       0x00000000       0x18 output_pic32_ssd1963\MainDemo.o
 .pdr           0x00000000      0x120 output_pic32_ssd1963\MainDemo.o
 .bss           0x00000000        0x0 output_pic32_ssd1963\rtcc.o
 .reginfo       0x00000000       0x18 output_pic32_ssd1963\rtcc.o
 .pdr           0x00000000      0x160 output_pic32_ssd1963\rtcc.o
 .text          0x00000000        0x0 output_pic32_ssd1963\Fonts.o
 .data          0x00000000        0x0 output_pic32_ssd1963\Fonts.o
 .bss           0x00000000        0x0 output_pic32_ssd1963\Fonts.o
 .reginfo       0x00000000       0x18 output_pic32_ssd1963\Fonts.o
 .pdr           0x00000000        0x0 output_pic32_ssd1963\Fonts.o
 .data          0x00000000        0x0 output_pic32_ssd1963\DemoSelection.o
 .bss           0x00000000        0x0 output_pic32_ssd1963\DemoSelection.o
 .reginfo       0x00000000       0x18 output_pic32_ssd1963\DemoSelection.o
 .pdr           0x00000000       0xc0 output_pic32_ssd1963\DemoSelection.o
 .data          0x00000000        0x0 output_pic32_ssd1963\Animation.o
 .bss           0x00000000        0x0 output_pic32_ssd1963\Animation.o
 .reginfo       0x00000000       0x18 output_pic32_ssd1963\Animation.o
 .pdr           0x00000000       0x80 output_pic32_ssd1963\Animation.o
 .text          0x00000000        0x0 output_pic32_ssd1963\AnimationBitmaps.o
 .data          0x00000000        0x0 output_pic32_ssd1963\AnimationBitmaps.o
 .bss           0x00000000        0x0 output_pic32_ssd1963\AnimationBitmaps.o
 .reginfo       0x00000000       0x18 output_pic32_ssd1963\AnimationBitmaps.o
 .pdr           0x00000000        0x0 output_pic32_ssd1963\AnimationBitmaps.o
 .data          0x00000000        0x0 output_pic32_ssd1963\ECG.o
 .bss           0x00000000        0x0 output_pic32_ssd1963\ECG.o
 .reginfo       0x00000000       0x18 output_pic32_ssd1963\ECG.o
 .pdr           0x00000000      0x180 output_pic32_ssd1963\ECG.o
 .bss           0x00000000        0x0 output_pic32_ssd1963\Games.o
 .reginfo       0x00000000       0x18 output_pic32_ssd1963\Games.o
 .pdr           0x00000000       0xe0 output_pic32_ssd1963\Games.o
 .text          0x00000000        0x0 output_pic32_ssd1963\SnakeBitmaps.o
 .data          0x00000000        0x0 output_pic32_ssd1963\SnakeBitmaps.o
 .bss           0x00000000        0x0 output_pic32_ssd1963\SnakeBitmaps.o
 .reginfo       0x00000000       0x18 output_pic32_ssd1963\SnakeBitmaps.o
 .pdr           0x00000000        0x0 output_pic32_ssd1963\SnakeBitmaps.o
 .text          0x00000000        0x0 output_pic32_ssd1963\ECGBitmaps.o
 .data          0x00000000        0x0 output_pic32_ssd1963\ECGBitmaps.o
 .bss           0x00000000        0x0 output_pic32_ssd1963\ECGBitmaps.o
 .reginfo       0x00000000       0x18 output_pic32_ssd1963\ECGBitmaps.o
 .pdr           0x00000000        0x0 output_pic32_ssd1963\ECGBitmaps.o
 .bss           0x00000000        0x0 output_pic32_ssd1963\RGBDemo.o
 .reginfo       0x00000000       0x18 output_pic32_ssd1963\RGBDemo.o
 .pdr           0x00000000      0x180 output_pic32_ssd1963\RGBDemo.o
 .data          0x00000000       0x64 output_pic32_ssd1963\MultiFontsDemo.o
 .bss           0x00000000        0x0 output_pic32_ssd1963\MultiFontsDemo.o
 .reginfo       0x00000000       0x18 output_pic32_ssd1963\MultiFontsDemo.o
 .pdr           0x00000000       0xa0 output_pic32_ssd1963\MultiFontsDemo.o
 .text          0x00000000        0x0 output_pic32_ssd1963\HelloWorldFonts.o
 .data          0x00000000        0x0 output_pic32_ssd1963\HelloWorldFonts.o
 .bss           0x00000000        0x0 output_pic32_ssd1963\HelloWorldFonts.o
 .reginfo       0x00000000       0x18 output_pic32_ssd1963\HelloWorldFonts.o
 .pdr           0x00000000        0x0 output_pic32_ssd1963\HelloWorldFonts.o
 .rodata        0x00000000      0xd28 output_pic32_ssd1963\HelloWorldFonts.o
 .bss           0x00000000        0x0 output_pic32_ssd1963\TimeDateDemo.o
 .reginfo       0x00000000       0x18 output_pic32_ssd1963\TimeDateDemo.o
 .pdr           0x00000000       0x80 output_pic32_ssd1963\TimeDateDemo.o
 .data          0x00000000        0x0 output_pic32_ssd1963\DrawTool.o
 .bss           0x00000000        0x0 output_pic32_ssd1963\DrawTool.o
 .reginfo       0x00000000       0x18 output_pic32_ssd1963\DrawTool.o
 .pdr           0x00000000       0xa0 output_pic32_ssd1963\DrawTool.o
 .data          0x00000000        0x0 output_pic32_ssd1963\SlideShowDemo.o
 .bss           0x00000000        0x0 output_pic32_ssd1963\SlideShowDemo.o
 .reginfo       0x00000000       0x18 output_pic32_ssd1963\SlideShowDemo.o
 .pdr           0x00000000       0x60 output_pic32_ssd1963\SlideShowDemo.o
 .text          0x00000000        0x0 output_pic32_ssd1963\Icons.o
 .data          0x00000000        0x0 output_pic32_ssd1963\Icons.o
 .bss           0x00000000        0x0 output_pic32_ssd1963\Icons.o
 .reginfo       0x00000000       0x18 output_pic32_ssd1963\Icons.o
 .pdr           0x00000000        0x0 output_pic32_ssd1963\Icons.o
 .rodata        0x00000000      0x244 output_pic32_ssd1963\Icons.o
 .data          0x00000000        0x0 output_pic32_ssd1963\DemoSteps.o
 .bss           0x00000000        0x0 output_pic32_ssd1963\DemoSteps.o
 .reginfo       0x00000000       0x18 output_pic32_ssd1963\DemoSteps.o
 .pdr           0x00000000       0x40 output_pic32_ssd1963\DemoSteps.o
 .data          0x00000000        0x0 output_pic32_ssd1963\SideButtons.o
 .bss           0x00000000        0x0 output_pic32_ssd1963\SideButtons.o
 .reginfo       0x00000000       0x18 output_pic32_ssd1963\SideButtons.o
 .pdr           0x00000000       0x20 output_pic32_ssd1963\SideButtons.o
 .text          0x00000000        0x0 output_pic32_ssd1963\BitmapFile.o
 .data          0x00000000        0x0 output_pic32_ssd1963\BitmapFile.o
 .bss           0x00000000        0x0 output_pic32_ssd1963\BitmapFile.o
 .reginfo       0x00000000       0x18 output_pic32_ssd1963\BitmapFile.o
 .pdr           0x00000000        0x0 output_pic32_ssd1963\BitmapFile.o
 .bss           0x00000000        0x0 output_pic32_ssd1963\GraphShow.o
 .reginfo       0x00000000       0x18 output_pic32_ssd1963\GraphShow.o
 .pdr           0x00000000       0xe0 output_pic32_ssd1963\GraphShow.o
 .sdata         0x00000000        0x4 output_pic32_ssd1963\GraphShow.o
 .text          0x00000000     0x674c output_pic32_ssd1963\FSIO.o
 .data          0x00000000        0x0 output_pic32_ssd1963\FSIO.o
 .bss           0x00000000        0x0 output_pic32_ssd1963\FSIO.o
 .reginfo       0x00000000       0x18 output_pic32_ssd1963\FSIO.o
 .pdr           0x00000000      0x7a0 output_pic32_ssd1963\FSIO.o
 .sdata         0x00000000        0xc output_pic32_ssd1963\FSIO.o
 .sbss          0x00000000        0xc output_pic32_ssd1963\FSIO.o
 .rodata        0x00000000       0xec output_pic32_ssd1963\FSIO.o
 .rodata.str1.4
                0x00000000        0x4 output_pic32_ssd1963\FSIO.o
 COMMON         0x00000000      0x5aa output_pic32_ssd1963\FSIO.o
 .text          0x00000000      0xaa8 output_pic32_ssd1963\SD-SPI.o
 .data          0x00000000        0x0 output_pic32_ssd1963\SD-SPI.o
 .bss           0x00000000        0x0 output_pic32_ssd1963\SD-SPI.o
 .reginfo       0x00000000       0x18 output_pic32_ssd1963\SD-SPI.o
 .pdr           0x00000000      0x1e0 output_pic32_ssd1963\SD-SPI.o
 .rodata        0x00000000       0xd8 output_pic32_ssd1963\SD-SPI.o
 .sbss          0x00000000        0x8 output_pic32_ssd1963\SD-SPI.o
 .text          0x00000000     0x1ba0 output_pic32_ssd1963\JpegDecoder.o
 .data          0x00000000        0x0 output_pic32_ssd1963\JpegDecoder.o
 .bss           0x00000000        0x0 output_pic32_ssd1963\JpegDecoder.o
 .reginfo       0x00000000       0x18 output_pic32_ssd1963\JpegDecoder.o
 .pdr           0x00000000      0x1c0 output_pic32_ssd1963\JpegDecoder.o
 .rodata        0x00000000       0x50 output_pic32_ssd1963\JpegDecoder.o
 .text          0x00000000     0x15c4 output_pic32_ssd1963\BmpDecoder.o
 .data          0x00000000        0x0 output_pic32_ssd1963\BmpDecoder.o
 .bss           0x00000000        0x0 output_pic32_ssd1963\BmpDecoder.o
 .reginfo       0x00000000       0x18 output_pic32_ssd1963\BmpDecoder.o
 .pdr           0x00000000       0x60 output_pic32_ssd1963\BmpDecoder.o
 .text          0x00000000      0xfdc output_pic32_ssd1963\GifDecoder.o
 .data          0x00000000        0x0 output_pic32_ssd1963\GifDecoder.o
 .bss           0x00000000        0x0 output_pic32_ssd1963\GifDecoder.o
 .reginfo       0x00000000       0x18 output_pic32_ssd1963\GifDecoder.o
 .pdr           0x00000000      0x1e0 output_pic32_ssd1963\GifDecoder.o
 .rodata        0x00000000       0x1c output_pic32_ssd1963\GifDecoder.o
 .text          0x00000000      0x208 output_pic32_ssd1963\ImageDecoder.o
 .data          0x00000000        0x0 output_pic32_ssd1963\ImageDecoder.o
 .bss           0x00000000        0x0 output_pic32_ssd1963\ImageDecoder.o
 .reginfo       0x00000000       0x18 output_pic32_ssd1963\ImageDecoder.o
 .pdr           0x00000000       0x80 output_pic32_ssd1963\ImageDecoder.o
 .text          0x00000000      0x520 output_pic32_ssd1963\jidctint.o
 .data          0x00000000        0x0 output_pic32_ssd1963\jidctint.o
 .bss           0x00000000        0x0 output_pic32_ssd1963\jidctint.o
 .reginfo       0x00000000       0x18 output_pic32_ssd1963\jidctint.o
 .pdr           0x00000000       0x20 output_pic32_ssd1963\jidctint.o
 .data          0x00000000        0x0 output_pic32_ssd1963\TouchScreen.o
 .bss           0x00000000        0x0 output_pic32_ssd1963\TouchScreen.o
 .reginfo       0x00000000       0x18 output_pic32_ssd1963\TouchScreen.o
 .pdr           0x00000000      0x140 output_pic32_ssd1963\TouchScreen.o
 .data          0x00000000        0x0 output_pic32_ssd1963\Beep.o
 .bss           0x00000000        0x0 output_pic32_ssd1963\Beep.o
 .reginfo       0x00000000       0x18 output_pic32_ssd1963\Beep.o
 .pdr           0x00000000       0x60 output_pic32_ssd1963\Beep.o
 .data          0x00000000        0x0 output_pic32_ssd1963\EEPROM.o
 .bss           0x00000000        0x0 output_pic32_ssd1963\EEPROM.o
 .reginfo       0x00000000       0x18 output_pic32_ssd1963\EEPROM.o
 .pdr           0x00000000      0x140 output_pic32_ssd1963\EEPROM.o
 .data          0x00000000        0x0 output_pic32_ssd1963\Window.o
 .bss           0x00000000        0x0 output_pic32_ssd1963\Window.o
 .reginfo       0x00000000       0x18 output_pic32_ssd1963\Window.o
 .pdr           0x00000000       0x80 output_pic32_ssd1963\Window.o
 .data          0x00000000        0x0 output_pic32_ssd1963\Button.o
 .bss           0x00000000        0x0 output_pic32_ssd1963\Button.o
 .reginfo       0x00000000       0x18 output_pic32_ssd1963\Button.o
 .pdr           0x00000000       0xa0 output_pic32_ssd1963\Button.o
 .bss           0x00000000        0x0 output_pic32_ssd1963\Chart.o
 .reginfo       0x00000000       0x18 output_pic32_ssd1963\Chart.o
 .pdr           0x00000000      0x220 output_pic32_ssd1963\Chart.o
 .data          0x00000000        0x0 output_pic32_ssd1963\CheckBox.o
 .bss           0x00000000        0x0 output_pic32_ssd1963\CheckBox.o
 .reginfo       0x00000000       0x18 output_pic32_ssd1963\CheckBox.o
 .pdr           0x00000000       0xa0 output_pic32_ssd1963\CheckBox.o
 .data          0x00000000        0x0 output_pic32_ssd1963\DisplayDriver.o
 .bss           0x00000000        0x0 output_pic32_ssd1963\DisplayDriver.o
 .reginfo       0x00000000       0x18 output_pic32_ssd1963\DisplayDriver.o
 .pdr           0x00000000      0x300 output_pic32_ssd1963\DisplayDriver.o
 .data          0x00000000        0x0 output_pic32_ssd1963\EditBox.o
 .bss           0x00000000        0x0 output_pic32_ssd1963\EditBox.o
 .reginfo       0x00000000       0x18 output_pic32_ssd1963\EditBox.o
 .pdr           0x00000000       0xe0 output_pic32_ssd1963\EditBox.o
 .data          0x00000000        0x0 output_pic32_ssd1963\Grid.o
 .bss           0x00000000        0x0 output_pic32_ssd1963\Grid.o
 .reginfo       0x00000000       0x18 output_pic32_ssd1963\Grid.o
 .pdr           0x00000000      0x140 output_pic32_ssd1963\Grid.o
 .data          0x00000000        0x0 output_pic32_ssd1963\GroupBox.o
 .bss           0x00000000        0x0 output_pic32_ssd1963\GroupBox.o
 .reginfo       0x00000000       0x18 output_pic32_ssd1963\GroupBox.o
 .pdr           0x00000000       0x60 output_pic32_ssd1963\GroupBox.o
 .data          0x00000000        0x0 output_pic32_ssd1963\ListBox.o
 .bss           0x00000000        0x0 output_pic32_ssd1963\ListBox.o
 .reginfo       0x00000000       0x18 output_pic32_ssd1963\ListBox.o
 .pdr           0x00000000      0x160 output_pic32_ssd1963\ListBox.o
 .data          0x00000000        0x0 output_pic32_ssd1963\Meter.o
 .reginfo       0x00000000       0x18 output_pic32_ssd1963\Meter.o
 .pdr           0x00000000       0xc0 output_pic32_ssd1963\Meter.o
 .data          0x00000000        0x0 output_pic32_ssd1963\Picture.o
 .bss           0x00000000        0x0 output_pic32_ssd1963\Picture.o
 .reginfo       0x00000000       0x18 output_pic32_ssd1963\Picture.o
 .pdr           0x00000000       0x60 output_pic32_ssd1963\Picture.o
 .data          0x00000000        0x0 output_pic32_ssd1963\Primitive.o
 .bss           0x00000000        0x0 output_pic32_ssd1963\Primitive.o
 .reginfo       0x00000000       0x18 output_pic32_ssd1963\Primitive.o
 .pdr           0x00000000      0x1c0 output_pic32_ssd1963\Primitive.o
 .data          0x00000000        0x0 output_pic32_ssd1963\RadioButton.o
 .bss           0x00000000        0x0 output_pic32_ssd1963\RadioButton.o
 .reginfo       0x00000000       0x18 output_pic32_ssd1963\RadioButton.o
 .pdr           0x00000000       0xe0 output_pic32_ssd1963\RadioButton.o
 .data          0x00000000        0x0 output_pic32_ssd1963\Slider.o
 .bss           0x00000000        0x0 output_pic32_ssd1963\Slider.o
 .reginfo       0x00000000       0x18 output_pic32_ssd1963\Slider.o
 .pdr           0x00000000      0x160 output_pic32_ssd1963\Slider.o
 .data          0x00000000        0x0 output_pic32_ssd1963\StaticText.o
 .bss           0x00000000        0x0 output_pic32_ssd1963\StaticText.o
 .reginfo       0x00000000       0x18 output_pic32_ssd1963\StaticText.o
 .pdr           0x00000000       0x80 output_pic32_ssd1963\StaticText.o
 .text          0x00000000        0x0 output_pic32_ssd1963\GOLFontDefault.o
 .data          0x00000000        0x0 output_pic32_ssd1963\GOLFontDefault.o
 .bss           0x00000000        0x0 output_pic32_ssd1963\GOLFontDefault.o
 .reginfo       0x00000000       0x18 output_pic32_ssd1963\GOLFontDefault.o
 .pdr           0x00000000        0x0 output_pic32_ssd1963\GOLFontDefault.o
 .data          0x00000000        0x0 output_pic32_ssd1963\GOL.o
 .bss           0x00000000        0x0 output_pic32_ssd1963\GOL.o
 .reginfo       0x00000000       0x18 output_pic32_ssd1963\GOL.o
 .pdr           0x00000000      0x1e0 output_pic32_ssd1963\GOL.o
 .text          0x00000000      0x410 output_pic32_ssd1963\uart2.o
 .data          0x00000000        0x0 output_pic32_ssd1963\uart2.o
 .bss           0x00000000        0x0 output_pic32_ssd1963\uart2.o
 .reginfo       0x00000000       0x18 output_pic32_ssd1963\uart2.o
 .pdr           0x00000000      0x180 output_pic32_ssd1963\uart2.o
 .rodata        0x00000000       0x10 output_pic32_ssd1963\uart2.o
 .text          0x00000000        0x0 output_pic32_ssd1963\JPEGDemo.o
 .data          0x00000000        0x0 output_pic32_ssd1963\JPEGDemo.o
 .bss           0x00000000        0x0 output_pic32_ssd1963\JPEGDemo.o
 .reginfo       0x00000000       0x18 output_pic32_ssd1963\JPEGDemo.o
 .pdr           0x00000000        0x0 output_pic32_ssd1963\JPEGDemo.o
 .text          0x00000000        0x0 output_pic32_ssd1963\IconsC32.o
 .data          0x00000000        0x0 output_pic32_ssd1963\IconsC32.o
 .bss           0x00000000        0x0 output_pic32_ssd1963\IconsC32.o
 .reginfo       0x00000000       0x18 output_pic32_ssd1963\IconsC32.o
 .pdr           0x00000000        0x0 output_pic32_ssd1963\IconsC32.o
 .text          0x00000000        0x0 output_pic32_ssd1963\SlideShowC32.o
 .data          0x00000000        0x0 output_pic32_ssd1963\SlideShowC32.o
 .bss           0x00000000        0x0 output_pic32_ssd1963\SlideShowC32.o
 .reginfo       0x00000000       0x18 output_pic32_ssd1963\SlideShowC32.o
 .pdr           0x00000000        0x0 output_pic32_ssd1963\SlideShowC32.o
 .text          0x00000000      0x548 output_pic32_ssd1963\vs1003b.o
 .data          0x00000000        0x0 output_pic32_ssd1963\vs1003b.o
 .bss           0x00000000        0x0 output_pic32_ssd1963\vs1003b.o
 .reginfo       0x00000000       0x18 output_pic32_ssd1963\vs1003b.o
 .pdr           0x00000000      0x120 output_pic32_ssd1963\vs1003b.o
 .data          0x00000000        0x0 C:/Program Files/Microchip/mplabc32/v1.12/bin/../lib/gcc/pic32mx/3.4.4/../../../../pic32mx/lib/size\libc.a(memset.o)
 .bss           0x00000000        0x0 C:/Program Files/Microchip/mplabc32/v1.12/bin/../lib/gcc/pic32mx/3.4.4/../../../../pic32mx/lib/size\libc.a(memset.o)
 .reginfo       0x00000000       0x18 C:/Program Files/Microchip/mplabc32/v1.12/bin/../lib/gcc/pic32mx/3.4.4/../../../../pic32mx/lib/size\libc.a(memset.o)
 .pdr           0x00000000       0x20 C:/Program Files/Microchip/mplabc32/v1.12/bin/../lib/gcc/pic32mx/3.4.4/../../../../pic32mx/lib/size\libc.a(memset.o)
 .text          0x00000000      0x1a0 C:/Program Files/Microchip/mplabc32/v1.12/bin/../lib/gcc/pic32mx/3.4.4/../../../../pic32mx/lib/size\libc.a(strcpy.o)
 .data          0x00000000        0x0 C:/Program Files/Microchip/mplabc32/v1.12/bin/../lib/gcc/pic32mx/3.4.4/../../../../pic32mx/lib/size\libc.a(strcpy.o)
 .bss           0x00000000        0x0 C:/Program Files/Microchip/mplabc32/v1.12/bin/../lib/gcc/pic32mx/3.4.4/../../../../pic32mx/lib/size\libc.a(strcpy.o)
 .reginfo       0x00000000       0x18 C:/Program Files/Microchip/mplabc32/v1.12/bin/../lib/gcc/pic32mx/3.4.4/../../../../pic32mx/lib/size\libc.a(strcpy.o)
 .pdr           0x00000000       0x20 C:/Program Files/Microchip/mplabc32/v1.12/bin/../lib/gcc/pic32mx/3.4.4/../../../../pic32mx/lib/size\libc.a(strcpy.o)
 .text          0x00000000      0x168 C:/Program Files/Microchip/mplabc32/v1.12/bin/../lib/gcc/pic32mx/3.4.4/../../../../pic32mx/lib/size\libc.a(strlen.o)
 .data          0x00000000        0x0 C:/Program Files/Microchip/mplabc32/v1.12/bin/../lib/gcc/pic32mx/3.4.4/../../../../pic32mx/lib/size\libc.a(strlen.o)
 .bss           0x00000000        0x0 C:/Program Files/Microchip/mplabc32/v1.12/bin/../lib/gcc/pic32mx/3.4.4/../../../../pic32mx/lib/size\libc.a(strlen.o)
 .reginfo       0x00000000       0x18 C:/Program Files/Microchip/mplabc32/v1.12/bin/../lib/gcc/pic32mx/3.4.4/../../../../pic32mx/lib/size\libc.a(strlen.o)
 .pdr           0x00000000       0x20 C:/Program Files/Microchip/mplabc32/v1.12/bin/../lib/gcc/pic32mx/3.4.4/../../../../pic32mx/lib/size\libc.a(strlen.o)
 .text          0x00000000        0x0 C:/Program Files/Microchip/mplabc32/v1.12/bin/../lib/gcc/pic32mx/3.4.4/../../../../pic32mx/lib/size\libc.a(general-exception.o)
 .data          0x00000000        0x0 C:/Program Files/Microchip/mplabc32/v1.12/bin/../lib/gcc/pic32mx/3.4.4/../../../../pic32mx/lib/size\libc.a(general-exception.o)
 .bss           0x00000000        0x0 C:/Program Files/Microchip/mplabc32/v1.12/bin/../lib/gcc/pic32mx/3.4.4/../../../../pic32mx/lib/size\libc.a(general-exception.o)
 .reginfo       0x00000000       0x18 C:/Program Files/Microchip/mplabc32/v1.12/bin/../lib/gcc/pic32mx/3.4.4/../../../../pic32mx/lib/size\libc.a(general-exception.o)
 .pdr           0x00000000       0x20 C:/Program Files/Microchip/mplabc32/v1.12/bin/../lib/gcc/pic32mx/3.4.4/../../../../pic32mx/lib/size\libc.a(general-exception.o)
 .text          0x00000000        0x0 C:/Program Files/Microchip/mplabc32/v1.12/bin/../lib/gcc/pic32mx/3.4.4/../../../../pic32mx/lib/size\libc.a(ctypef.o)
 .data          0x00000000        0x0 C:/Program Files/Microchip/mplabc32/v1.12/bin/../lib/gcc/pic32mx/3.4.4/../../../../pic32mx/lib/size\libc.a(ctypef.o)
 .bss           0x00000000        0x0 C:/Program Files/Microchip/mplabc32/v1.12/bin/../lib/gcc/pic32mx/3.4.4/../../../../pic32mx/lib/size\libc.a(ctypef.o)
 .reginfo       0x00000000       0x18 C:/Program Files/Microchip/mplabc32/v1.12/bin/../lib/gcc/pic32mx/3.4.4/../../../../pic32mx/lib/size\libc.a(ctypef.o)
 .pdr           0x00000000      0x220 C:/Program Files/Microchip/mplabc32/v1.12/bin/../lib/gcc/pic32mx/3.4.4/../../../../pic32mx/lib/size\libc.a(ctypef.o)
 .text.tolower  0x00000000       0x20 C:/Program Files/Microchip/mplabc32/v1.12/bin/../lib/gcc/pic32mx/3.4.4/../../../../pic32mx/lib/size\libc.a(ctypef.o)
 .text.toupper  0x00000000       0x20 C:/Program Files/Microchip/mplabc32/v1.12/bin/../lib/gcc/pic32mx/3.4.4/../../../../pic32mx/lib/size\libc.a(ctypef.o)
 .text.isalnum  0x00000000       0x18 C:/Program Files/Microchip/mplabc32/v1.12/bin/../lib/gcc/pic32mx/3.4.4/../../../../pic32mx/lib/size\libc.a(ctypef.o)
 .text.isalpha  0x00000000       0x18 C:/Program Files/Microchip/mplabc32/v1.12/bin/../lib/gcc/pic32mx/3.4.4/../../../../pic32mx/lib/size\libc.a(ctypef.o)
 .text.isascii  0x00000000        0x8 C:/Program Files/Microchip/mplabc32/v1.12/bin/../lib/gcc/pic32mx/3.4.4/../../../../pic32mx/lib/size\libc.a(ctypef.o)
 .text.iscntrl  0x00000000       0x18 C:/Program Files/Microchip/mplabc32/v1.12/bin/../lib/gcc/pic32mx/3.4.4/../../../../pic32mx/lib/size\libc.a(ctypef.o)
 .text.isdigit  0x00000000       0x18 C:/Program Files/Microchip/mplabc32/v1.12/bin/../lib/gcc/pic32mx/3.4.4/../../../../pic32mx/lib/size\libc.a(ctypef.o)
 .text.isgraph  0x00000000       0x18 C:/Program Files/Microchip/mplabc32/v1.12/bin/../lib/gcc/pic32mx/3.4.4/../../../../pic32mx/lib/size\libc.a(ctypef.o)
 .text.islower  0x00000000       0x18 C:/Program Files/Microchip/mplabc32/v1.12/bin/../lib/gcc/pic32mx/3.4.4/../../../../pic32mx/lib/size\libc.a(ctypef.o)
 .text.isprint  0x00000000       0x18 C:/Program Files/Microchip/mplabc32/v1.12/bin/../lib/gcc/pic32mx/3.4.4/../../../../pic32mx/lib/size\libc.a(ctypef.o)
 .text.ispunct  0x00000000       0x18 C:/Program Files/Microchip/mplabc32/v1.12/bin/../lib/gcc/pic32mx/3.4.4/../../../../pic32mx/lib/size\libc.a(ctypef.o)
 .text.isspace  0x00000000       0x18 C:/Program Files/Microchip/mplabc32/v1.12/bin/../lib/gcc/pic32mx/3.4.4/../../../../pic32mx/lib/size\libc.a(ctypef.o)
 .text.isupper  0x00000000       0x18 C:/Program Files/Microchip/mplabc32/v1.12/bin/../lib/gcc/pic32mx/3.4.4/../../../../pic32mx/lib/size\libc.a(ctypef.o)
 .text.isxdigit
                0x00000000       0x18 C:/Program Files/Microchip/mplabc32/v1.12/bin/../lib/gcc/pic32mx/3.4.4/../../../../pic32mx/lib/size\libc.a(ctypef.o)
 .text.toascii  0x00000000        0x8 C:/Program Files/Microchip/mplabc32/v1.12/bin/../lib/gcc/pic32mx/3.4.4/../../../../pic32mx/lib/size\libc.a(ctypef.o)
 .text._tolower
                0x00000000        0x8 C:/Program Files/Microchip/mplabc32/v1.12/bin/../lib/gcc/pic32mx/3.4.4/../../../../pic32mx/lib/size\libc.a(ctypef.o)
 .text._toupper
                0x00000000        0x8 C:/Program Files/Microchip/mplabc32/v1.12/bin/../lib/gcc/pic32mx/3.4.4/../../../../pic32mx/lib/size\libc.a(ctypef.o)
 .text          0x00000000        0x0 C:/Program Files/Microchip/mplabc32/v1.12/bin/../lib/gcc/pic32mx/3.4.4/../../../../pic32mx/lib/size\libc.a(malloc.o)
 .data          0x00000000        0x0 C:/Program Files/Microchip/mplabc32/v1.12/bin/../lib/gcc/pic32mx/3.4.4/../../../../pic32mx/lib/size\libc.a(malloc.o)
 .bss           0x00000000        0x0 C:/Program Files/Microchip/mplabc32/v1.12/bin/../lib/gcc/pic32mx/3.4.4/../../../../pic32mx/lib/size\libc.a(malloc.o)
 .reginfo       0x00000000       0x18 C:/Program Files/Microchip/mplabc32/v1.12/bin/../lib/gcc/pic32mx/3.4.4/../../../../pic32mx/lib/size\libc.a(malloc.o)
 .pdr           0x00000000       0x60 C:/Program Files/Microchip/mplabc32/v1.12/bin/../lib/gcc/pic32mx/3.4.4/../../../../pic32mx/lib/size\libc.a(malloc.o)
 .text.realloc  0x00000000       0xcc C:/Program Files/Microchip/mplabc32/v1.12/bin/../lib/gcc/pic32mx/3.4.4/../../../../pic32mx/lib/size\libc.a(malloc.o)
 .text          0x00000000      0x168 C:/Program Files/Microchip/mplabc32/v1.12/bin/../lib/gcc/pic32mx/3.4.4/../../../../pic32mx/lib/size\libc.a(memcpy.o)
 .data          0x00000000        0x0 C:/Program Files/Microchip/mplabc32/v1.12/bin/../lib/gcc/pic32mx/3.4.4/../../../../pic32mx/lib/size\libc.a(memcpy.o)
 .bss           0x00000000        0x0 C:/Program Files/Microchip/mplabc32/v1.12/bin/../lib/gcc/pic32mx/3.4.4/../../../../pic32mx/lib/size\libc.a(memcpy.o)
 .reginfo       0x00000000       0x18 C:/Program Files/Microchip/mplabc32/v1.12/bin/../lib/gcc/pic32mx/3.4.4/../../../../pic32mx/lib/size\libc.a(memcpy.o)
 .pdr           0x00000000       0x20 C:/Program Files/Microchip/mplabc32/v1.12/bin/../lib/gcc/pic32mx/3.4.4/../../../../pic32mx/lib/size\libc.a(memcpy.o)
 .text          0x00000000        0x0 C:/Program Files/Microchip/mplabc32/v1.12/bin/../lib/gcc/pic32mx/3.4.4/../../../../pic32mx/lib/size\libc.a(rand.o)
 .data          0x00000000        0x0 C:/Program Files/Microchip/mplabc32/v1.12/bin/../lib/gcc/pic32mx/3.4.4/../../../../pic32mx/lib/size\libc.a(rand.o)
 .bss           0x00000000        0x0 C:/Program Files/Microchip/mplabc32/v1.12/bin/../lib/gcc/pic32mx/3.4.4/../../../../pic32mx/lib/size\libc.a(rand.o)
 .reginfo       0x00000000       0x18 C:/Program Files/Microchip/mplabc32/v1.12/bin/../lib/gcc/pic32mx/3.4.4/../../../../pic32mx/lib/size\libc.a(rand.o)
 .pdr           0x00000000       0x40 C:/Program Files/Microchip/mplabc32/v1.12/bin/../lib/gcc/pic32mx/3.4.4/../../../../pic32mx/lib/size\libc.a(rand.o)
 .text          0x00000000        0x0 C:/Program Files/Microchip/mplabc32/v1.12/bin/../lib/gcc/pic32mx/3.4.4/../../../../pic32mx/lib/size\libc.a(strchr.o)
 .data          0x00000000        0x0 C:/Program Files/Microchip/mplabc32/v1.12/bin/../lib/gcc/pic32mx/3.4.4/../../../../pic32mx/lib/size\libc.a(strchr.o)
 .bss           0x00000000        0x0 C:/Program Files/Microchip/mplabc32/v1.12/bin/../lib/gcc/pic32mx/3.4.4/../../../../pic32mx/lib/size\libc.a(strchr.o)
 .reginfo       0x00000000       0x18 C:/Program Files/Microchip/mplabc32/v1.12/bin/../lib/gcc/pic32mx/3.4.4/../../../../pic32mx/lib/size\libc.a(strchr.o)
 .pdr           0x00000000       0x20 C:/Program Files/Microchip/mplabc32/v1.12/bin/../lib/gcc/pic32mx/3.4.4/../../../../pic32mx/lib/size\libc.a(strchr.o)
 .text.strchr   0x00000000       0x28 C:/Program Files/Microchip/mplabc32/v1.12/bin/../lib/gcc/pic32mx/3.4.4/../../../../pic32mx/lib/size\libc.a(strchr.o)
 .text          0x00000000        0x0 C:/Program Files/Microchip/mplabc32/v1.12/bin/../lib/gcc/pic32mx/3.4.4/../../../../pic32mx/lib/size\libc.a(strncpy.o)
 .data          0x00000000        0x0 C:/Program Files/Microchip/mplabc32/v1.12/bin/../lib/gcc/pic32mx/3.4.4/../../../../pic32mx/lib/size\libc.a(strncpy.o)
 .bss           0x00000000        0x0 C:/Program Files/Microchip/mplabc32/v1.12/bin/../lib/gcc/pic32mx/3.4.4/../../../../pic32mx/lib/size\libc.a(strncpy.o)
 .reginfo       0x00000000       0x18 C:/Program Files/Microchip/mplabc32/v1.12/bin/../lib/gcc/pic32mx/3.4.4/../../../../pic32mx/lib/size\libc.a(strncpy.o)
 .pdr           0x00000000       0x20 C:/Program Files/Microchip/mplabc32/v1.12/bin/../lib/gcc/pic32mx/3.4.4/../../../../pic32mx/lib/size\libc.a(strncpy.o)
 .text.strncpy  0x00000000       0x48 C:/Program Files/Microchip/mplabc32/v1.12/bin/../lib/gcc/pic32mx/3.4.4/../../../../pic32mx/lib/size\libc.a(strncpy.o)
 .text          0x00000000        0x0 C:/Program Files/Microchip/mplabc32/v1.12/bin/../lib/gcc/pic32mx/3.4.4/../../../../pic32mx/lib/size\libc.a(sbrk.o)
 .data          0x00000000        0x0 C:/Program Files/Microchip/mplabc32/v1.12/bin/../lib/gcc/pic32mx/3.4.4/../../../../pic32mx/lib/size\libc.a(sbrk.o)
 .bss           0x00000000        0x0 C:/Program Files/Microchip/mplabc32/v1.12/bin/../lib/gcc/pic32mx/3.4.4/../../../../pic32mx/lib/size\libc.a(sbrk.o)
 .reginfo       0x00000000       0x18 C:/Program Files/Microchip/mplabc32/v1.12/bin/../lib/gcc/pic32mx/3.4.4/../../../../pic32mx/lib/size\libc.a(sbrk.o)
 .pdr           0x00000000       0xa0 C:/Program Files/Microchip/mplabc32/v1.12/bin/../lib/gcc/pic32mx/3.4.4/../../../../pic32mx/lib/size\libc.a(sbrk.o)
 .text.getpagesize
                0x00000000        0x8 C:/Program Files/Microchip/mplabc32/v1.12/bin/../lib/gcc/pic32mx/3.4.4/../../../../pic32mx/lib/size\libc.a(sbrk.o)
 .text          0x00000000        0x0 C:/Program Files/Microchip/mplabc32/v1.12/bin/../lib/gcc/pic32mx/3.4.4/../../../../pic32mx/lib/size\libc.a(default-general-exception-handler.o)
 .data          0x00000000        0x0 C:/Program Files/Microchip/mplabc32/v1.12/bin/../lib/gcc/pic32mx/3.4.4/../../../../pic32mx/lib/size\libc.a(default-general-exception-handler.o)
 .bss           0x00000000        0x0 C:/Program Files/Microchip/mplabc32/v1.12/bin/../lib/gcc/pic32mx/3.4.4/../../../../pic32mx/lib/size\libc.a(default-general-exception-handler.o)
 .reginfo       0x00000000       0x18 C:/Program Files/Microchip/mplabc32/v1.12/bin/../lib/gcc/pic32mx/3.4.4/../../../../pic32mx/lib/size\libc.a(default-general-exception-handler.o)
 .pdr           0x00000000       0x20 C:/Program Files/Microchip/mplabc32/v1.12/bin/../lib/gcc/pic32mx/3.4.4/../../../../pic32mx/lib/size\libc.a(default-general-exception-handler.o)
 .text          0x00000000        0x0 C:/Program Files/Microchip/mplabc32/v1.12/bin/../lib/gcc/pic32mx/3.4.4/../../../../pic32mx/lib/size\libc.a(default-bootstrap-exception-handler.o)
 .data          0x00000000        0x0 C:/Program Files/Microchip/mplabc32/v1.12/bin/../lib/gcc/pic32mx/3.4.4/../../../../pic32mx/lib/size\libc.a(default-bootstrap-exception-handler.o)
 .bss           0x00000000        0x0 C:/Program Files/Microchip/mplabc32/v1.12/bin/../lib/gcc/pic32mx/3.4.4/../../../../pic32mx/lib/size\libc.a(default-bootstrap-exception-handler.o)
 .reginfo       0x00000000       0x18 C:/Program Files/Microchip/mplabc32/v1.12/bin/../lib/gcc/pic32mx/3.4.4/../../../../pic32mx/lib/size\libc.a(default-bootstrap-exception-handler.o)
 .pdr           0x00000000       0x20 C:/Program Files/Microchip/mplabc32/v1.12/bin/../lib/gcc/pic32mx/3.4.4/../../../../pic32mx/lib/size\libc.a(default-bootstrap-exception-handler.o)
 .text          0x00000000        0x0 C:/Program Files/Microchip/mplabc32/v1.12/bin/../lib/gcc/pic32mx/3.4.4/../../../../pic32mx/lib/size\libc.a(default-on-reset.o)
 .data          0x00000000        0x0 C:/Program Files/Microchip/mplabc32/v1.12/bin/../lib/gcc/pic32mx/3.4.4/../../../../pic32mx/lib/size\libc.a(default-on-reset.o)
 .bss           0x00000000        0x0 C:/Program Files/Microchip/mplabc32/v1.12/bin/../lib/gcc/pic32mx/3.4.4/../../../../pic32mx/lib/size\libc.a(default-on-reset.o)
 .reginfo       0x00000000       0x18 C:/Program Files/Microchip/mplabc32/v1.12/bin/../lib/gcc/pic32mx/3.4.4/../../../../pic32mx/lib/size\libc.a(default-on-reset.o)
 .pdr           0x00000000       0x20 C:/Program Files/Microchip/mplabc32/v1.12/bin/../lib/gcc/pic32mx/3.4.4/../../../../pic32mx/lib/size\libc.a(default-on-reset.o)
 .text          0x00000000        0x0 C:/Program Files/Microchip/mplabc32/v1.12/bin/../lib/gcc/pic32mx/3.4.4/../../../../pic32mx/lib/size\libc.a(default-on-bootstrap.o)
 .data          0x00000000        0x0 C:/Program Files/Microchip/mplabc32/v1.12/bin/../lib/gcc/pic32mx/3.4.4/../../../../pic32mx/lib/size\libc.a(default-on-bootstrap.o)
 .bss           0x00000000        0x0 C:/Program Files/Microchip/mplabc32/v1.12/bin/../lib/gcc/pic32mx/3.4.4/../../../../pic32mx/lib/size\libc.a(default-on-bootstrap.o)
 .reginfo       0x00000000       0x18 C:/Program Files/Microchip/mplabc32/v1.12/bin/../lib/gcc/pic32mx/3.4.4/../../../../pic32mx/lib/size\libc.a(default-on-bootstrap.o)
 .pdr           0x00000000       0x20 C:/Program Files/Microchip/mplabc32/v1.12/bin/../lib/gcc/pic32mx/3.4.4/../../../../pic32mx/lib/size\libc.a(default-on-bootstrap.o)
 .data          0x00000000        0x0 C:/Program Files/Microchip/mplabc32/v1.12/bin/../lib/gcc/pic32mx/3.4.4/../../../../pic32mx/lib/size\libc.a(default-nmi-handler.o)
 .bss           0x00000000        0x0 C:/Program Files/Microchip/mplabc32/v1.12/bin/../lib/gcc/pic32mx/3.4.4/../../../../pic32mx/lib/size\libc.a(default-nmi-handler.o)
 .reginfo       0x00000000       0x18 C:/Program Files/Microchip/mplabc32/v1.12/bin/../lib/gcc/pic32mx/3.4.4/../../../../pic32mx/lib/size\libc.a(default-nmi-handler.o)
 .pdr           0x00000000       0x20 C:/Program Files/Microchip/mplabc32/v1.12/bin/../lib/gcc/pic32mx/3.4.4/../../../../pic32mx/lib/size\libc.a(default-nmi-handler.o)
 .text          0x00000000        0x0 C:/Program Files/Microchip/mplabc32/v1.12/bin/../lib/gcc/pic32mx/3.4.4/../../../../pic32mx/lib/size\libc.a(ctype.o)
 .data          0x00000000        0x0 C:/Program Files/Microchip/mplabc32/v1.12/bin/../lib/gcc/pic32mx/3.4.4/../../../../pic32mx/lib/size\libc.a(ctype.o)
 .bss           0x00000000        0x0 C:/Program Files/Microchip/mplabc32/v1.12/bin/../lib/gcc/pic32mx/3.4.4/../../../../pic32mx/lib/size\libc.a(ctype.o)
 .reginfo       0x00000000       0x18 C:/Program Files/Microchip/mplabc32/v1.12/bin/../lib/gcc/pic32mx/3.4.4/../../../../pic32mx/lib/size\libc.a(ctype.o)
 .pdr           0x00000000        0x0 C:/Program Files/Microchip/mplabc32/v1.12/bin/../lib/gcc/pic32mx/3.4.4/../../../../pic32mx/lib/size\libc.a(ctype.o)
 .rodata._ctype
                0x00000000      0x104 C:/Program Files/Microchip/mplabc32/v1.12/bin/../lib/gcc/pic32mx/3.4.4/../../../../pic32mx/lib/size\libc.a(ctype.o)
 .text          0x00000000        0x0 C:/Program Files/Microchip/mplabc32/v1.12/bin/../lib/gcc/pic32mx/3.4.4/../../../../pic32mx/lib/size\libc.a(errno.o)
 .data          0x00000000        0x0 C:/Program Files/Microchip/mplabc32/v1.12/bin/../lib/gcc/pic32mx/3.4.4/../../../../pic32mx/lib/size\libc.a(errno.o)
 .bss           0x00000000        0x0 C:/Program Files/Microchip/mplabc32/v1.12/bin/../lib/gcc/pic32mx/3.4.4/../../../../pic32mx/lib/size\libc.a(errno.o)
 .reginfo       0x00000000       0x18 C:/Program Files/Microchip/mplabc32/v1.12/bin/../lib/gcc/pic32mx/3.4.4/../../../../pic32mx/lib/size\libc.a(errno.o)
 .pdr           0x00000000        0x0 C:/Program Files/Microchip/mplabc32/v1.12/bin/../lib/gcc/pic32mx/3.4.4/../../../../pic32mx/lib/size\libc.a(errno.o)
 .data          0x00000000        0x0 C:/Program Files/Microchip/mplabc32/v1.12/bin/../lib/gcc/pic32mx/3.4.4/../../../../pic32mx/lib/size\libm.a(fp32.o)
 .bss           0x00000000        0x0 C:/Program Files/Microchip/mplabc32/v1.12/bin/../lib/gcc/pic32mx/3.4.4/../../../../pic32mx/lib/size\libm.a(fp32.o)
 .reginfo       0x00000000       0x18 C:/Program Files/Microchip/mplabc32/v1.12/bin/../lib/gcc/pic32mx/3.4.4/../../../../pic32mx/lib/size\libm.a(fp32.o)
 .pdr           0x00000000        0x0 C:/Program Files/Microchip/mplabc32/v1.12/bin/../lib/gcc/pic32mx/3.4.4/../../../../pic32mx/lib/size\libm.a(fp32.o)
 .data          0x00000000        0x0 C:/Program Files/Microchip/mplabc32/v1.12/bin/../lib/gcc/pic32mx/3.4.4/../../../../pic32mx/lib/size\libm.a(fpcos32.o)
 .bss           0x00000000        0x0 C:/Program Files/Microchip/mplabc32/v1.12/bin/../lib/gcc/pic32mx/3.4.4/../../../../pic32mx/lib/size\libm.a(fpcos32.o)
 .reginfo       0x00000000       0x18 C:/Program Files/Microchip/mplabc32/v1.12/bin/../lib/gcc/pic32mx/3.4.4/../../../../pic32mx/lib/size\libm.a(fpcos32.o)
 .pdr           0x00000000        0x0 C:/Program Files/Microchip/mplabc32/v1.12/bin/../lib/gcc/pic32mx/3.4.4/../../../../pic32mx/lib/size\libm.a(fpcos32.o)
 .data          0x00000000        0x0 C:/Program Files/Microchip/mplabc32/v1.12/bin/../lib/gcc/pic32mx/3.4.4/../../../../pic32mx/lib/size\libm.a(fpsin32.o)
 .bss           0x00000000        0x0 C:/Program Files/Microchip/mplabc32/v1.12/bin/../lib/gcc/pic32mx/3.4.4/../../../../pic32mx/lib/size\libm.a(fpsin32.o)
 .reginfo       0x00000000       0x18 C:/Program Files/Microchip/mplabc32/v1.12/bin/../lib/gcc/pic32mx/3.4.4/../../../../pic32mx/lib/size\libm.a(fpsin32.o)
 .pdr           0x00000000        0x0 C:/Program Files/Microchip/mplabc32/v1.12/bin/../lib/gcc/pic32mx/3.4.4/../../../../pic32mx/lib/size\libm.a(fpsin32.o)
 .data          0x00000000        0x0 C:/Program Files/Microchip/mplabc32/v1.12/bin/../lib/gcc/pic32mx/3.4.4/../../../../pic32mx/lib/size\libm.a(fpreduct32.o)
 .bss           0x00000000        0x0 C:/Program Files/Microchip/mplabc32/v1.12/bin/../lib/gcc/pic32mx/3.4.4/../../../../pic32mx/lib/size\libm.a(fpreduct32.o)
 .reginfo       0x00000000       0x18 C:/Program Files/Microchip/mplabc32/v1.12/bin/../lib/gcc/pic32mx/3.4.4/../../../../pic32mx/lib/size\libm.a(fpreduct32.o)
 .pdr           0x00000000        0x0 C:/Program Files/Microchip/mplabc32/v1.12/bin/../lib/gcc/pic32mx/3.4.4/../../../../pic32mx/lib/size\libm.a(fpreduct32.o)
 .text          0x00000000        0x0 C:/Program Files/Microchip/mplabc32/v1.12/bin/../lib/gcc/pic32mx/3.4.4/../../../../pic32mx/lib/size\libm.a(sincof32.o)
 .bss           0x00000000        0x0 C:/Program Files/Microchip/mplabc32/v1.12/bin/../lib/gcc/pic32mx/3.4.4/../../../../pic32mx/lib/size\libm.a(sincof32.o)
 .reginfo       0x00000000       0x18 C:/Program Files/Microchip/mplabc32/v1.12/bin/../lib/gcc/pic32mx/3.4.4/../../../../pic32mx/lib/size\libm.a(sincof32.o)
 .pdr           0x00000000        0x0 C:/Program Files/Microchip/mplabc32/v1.12/bin/../lib/gcc/pic32mx/3.4.4/../../../../pic32mx/lib/size\libm.a(sincof32.o)
 .text          0x00000000        0x0 C:/Program Files/Microchip/mplabc32/v1.12/bin/../lib/gcc/pic32mx/3.4.4/../../../../pic32mx/lib/size\libmchp_peripheral.a(open_core_timer_lib.o)
 .data          0x00000000        0x0 C:/Program Files/Microchip/mplabc32/v1.12/bin/../lib/gcc/pic32mx/3.4.4/../../../../pic32mx/lib/size\libmchp_peripheral.a(open_core_timer_lib.o)
 .bss           0x00000000        0x0 C:/Program Files/Microchip/mplabc32/v1.12/bin/../lib/gcc/pic32mx/3.4.4/../../../../pic32mx/lib/size\libmchp_peripheral.a(open_core_timer_lib.o)
 .reginfo       0x00000000       0x18 C:/Program Files/Microchip/mplabc32/v1.12/bin/../lib/gcc/pic32mx/3.4.4/../../../../pic32mx/lib/size\libmchp_peripheral.a(open_core_timer_lib.o)
 .pdr           0x00000000       0x20 C:/Program Files/Microchip/mplabc32/v1.12/bin/../lib/gcc/pic32mx/3.4.4/../../../../pic32mx/lib/size\libmchp_peripheral.a(open_core_timer_lib.o)
 .text          0x00000000        0x0 C:/Program Files/Microchip/mplabc32/v1.12/bin/../lib/gcc/pic32mx/3.4.4/../../../../pic32mx/lib/size\libmchp_peripheral_32MX360F512L.a(pcache.o)
 .data          0x00000000        0x0 C:/Program Files/Microchip/mplabc32/v1.12/bin/../lib/gcc/pic32mx/3.4.4/../../../../pic32mx/lib/size\libmchp_peripheral_32MX360F512L.a(pcache.o)
 .bss           0x00000000        0x0 C:/Program Files/Microchip/mplabc32/v1.12/bin/../lib/gcc/pic32mx/3.4.4/../../../../pic32mx/lib/size\libmchp_peripheral_32MX360F512L.a(pcache.o)
 .reginfo       0x00000000       0x18 C:/Program Files/Microchip/mplabc32/v1.12/bin/../lib/gcc/pic32mx/3.4.4/../../../../pic32mx/lib/size\libmchp_peripheral_32MX360F512L.a(pcache.o)
 .pdr           0x00000000       0x40 C:/Program Files/Microchip/mplabc32/v1.12/bin/../lib/gcc/pic32mx/3.4.4/../../../../pic32mx/lib/size\libmchp_peripheral_32MX360F512L.a(pcache.o)
 .text.CheKseg0CacheOff
                0x00000000       0x18 C:/Program Files/Microchip/mplabc32/v1.12/bin/../lib/gcc/pic32mx/3.4.4/../../../../pic32mx/lib/size\libmchp_peripheral_32MX360F512L.a(pcache.o)
 .text          0x00000000        0x0 C:/Program Files/Microchip/mplabc32/v1.12/bin/../lib/gcc/pic32mx/3.4.4/../../../../pic32mx/lib/size\libmchp_peripheral_32MX360F512L.a(int_disable_interrupts_lib.o)
 .data          0x00000000        0x0 C:/Program Files/Microchip/mplabc32/v1.12/bin/../lib/gcc/pic32mx/3.4.4/../../../../pic32mx/lib/size\libmchp_peripheral_32MX360F512L.a(int_disable_interrupts_lib.o)
 .bss           0x00000000        0x0 C:/Program Files/Microchip/mplabc32/v1.12/bin/../lib/gcc/pic32mx/3.4.4/../../../../pic32mx/lib/size\libmchp_peripheral_32MX360F512L.a(int_disable_interrupts_lib.o)
 .reginfo       0x00000000       0x18 C:/Program Files/Microchip/mplabc32/v1.12/bin/../lib/gcc/pic32mx/3.4.4/../../../../pic32mx/lib/size\libmchp_peripheral_32MX360F512L.a(int_disable_interrupts_lib.o)
 .pdr           0x00000000       0x20 C:/Program Files/Microchip/mplabc32/v1.12/bin/../lib/gcc/pic32mx/3.4.4/../../../../pic32mx/lib/size\libmchp_peripheral_32MX360F512L.a(int_disable_interrupts_lib.o)
 .text          0x00000000        0x0 C:/Program Files/Microchip/mplabc32/v1.12/bin/../lib/gcc/pic32mx/3.4.4/../../../../pic32mx/lib/size\libmchp_peripheral_32MX360F512L.a(int_restore_interrupts_lib.o)
 .data          0x00000000        0x0 C:/Program Files/Microchip/mplabc32/v1.12/bin/../lib/gcc/pic32mx/3.4.4/../../../../pic32mx/lib/size\libmchp_peripheral_32MX360F512L.a(int_restore_interrupts_lib.o)
 .bss           0x00000000        0x0 C:/Program Files/Microchip/mplabc32/v1.12/bin/../lib/gcc/pic32mx/3.4.4/../../../../pic32mx/lib/size\libmchp_peripheral_32MX360F512L.a(int_restore_interrupts_lib.o)
 .reginfo       0x00000000       0x18 C:/Program Files/Microchip/mplabc32/v1.12/bin/../lib/gcc/pic32mx/3.4.4/../../../../pic32mx/lib/size\libmchp_peripheral_32MX360F512L.a(int_restore_interrupts_lib.o)
 .pdr           0x00000000       0x20 C:/Program Files/Microchip/mplabc32/v1.12/bin/../lib/gcc/pic32mx/3.4.4/../../../../pic32mx/lib/size\libmchp_peripheral_32MX360F512L.a(int_restore_interrupts_lib.o)
 .text          0x00000000        0x0 C:/Program Files/Microchip/mplabc32/v1.12/bin/../lib/gcc/pic32mx/3.4.4/../../../../pic32mx/lib/size\libmchp_peripheral_32MX360F512L.a(int_enable_mv_int_lib.o)
 .data          0x00000000        0x0 C:/Program Files/Microchip/mplabc32/v1.12/bin/../lib/gcc/pic32mx/3.4.4/../../../../pic32mx/lib/size\libmchp_peripheral_32MX360F512L.a(int_enable_mv_int_lib.o)
 .bss           0x00000000        0x0 C:/Program Files/Microchip/mplabc32/v1.12/bin/../lib/gcc/pic32mx/3.4.4/../../../../pic32mx/lib/size\libmchp_peripheral_32MX360F512L.a(int_enable_mv_int_lib.o)
 .reginfo       0x00000000       0x18 C:/Program Files/Microchip/mplabc32/v1.12/bin/../lib/gcc/pic32mx/3.4.4/../../../../pic32mx/lib/size\libmchp_peripheral_32MX360F512L.a(int_enable_mv_int_lib.o)
 .pdr           0x00000000       0x20 C:/Program Files/Microchip/mplabc32/v1.12/bin/../lib/gcc/pic32mx/3.4.4/../../../../pic32mx/lib/size\libmchp_peripheral_32MX360F512L.a(int_enable_mv_int_lib.o)
 .text          0x00000000        0x0 C:/Program Files/Microchip/mplabc32/v1.12/bin/../lib/gcc/pic32mx/3.4.4/../../../../pic32mx/lib/size\libmchp_peripheral_32MX360F512L.a(rtcc_init_lib.o)
 .data          0x00000000        0x0 C:/Program Files/Microchip/mplabc32/v1.12/bin/../lib/gcc/pic32mx/3.4.4/../../../../pic32mx/lib/size\libmchp_peripheral_32MX360F512L.a(rtcc_init_lib.o)
 .bss           0x00000000        0x0 C:/Program Files/Microchip/mplabc32/v1.12/bin/../lib/gcc/pic32mx/3.4.4/../../../../pic32mx/lib/size\libmchp_peripheral_32MX360F512L.a(rtcc_init_lib.o)
 .reginfo       0x00000000       0x18 C:/Program Files/Microchip/mplabc32/v1.12/bin/../lib/gcc/pic32mx/3.4.4/../../../../pic32mx/lib/size\libmchp_peripheral_32MX360F512L.a(rtcc_init_lib.o)
 .pdr           0x00000000       0x20 C:/Program Files/Microchip/mplabc32/v1.12/bin/../lib/gcc/pic32mx/3.4.4/../../../../pic32mx/lib/size\libmchp_peripheral_32MX360F512L.a(rtcc_init_lib.o)
 .text          0x00000000        0x0 C:/Program Files/Microchip/mplabc32/v1.12/bin/../lib/gcc/pic32mx/3.4.4/../../../../pic32mx/lib/size\libmchp_peripheral_32MX360F512L.a(rtcc_set_date_lib.o)
 .data          0x00000000        0x0 C:/Program Files/Microchip/mplabc32/v1.12/bin/../lib/gcc/pic32mx/3.4.4/../../../../pic32mx/lib/size\libmchp_peripheral_32MX360F512L.a(rtcc_set_date_lib.o)
 .bss           0x00000000        0x0 C:/Program Files/Microchip/mplabc32/v1.12/bin/../lib/gcc/pic32mx/3.4.4/../../../../pic32mx/lib/size\libmchp_peripheral_32MX360F512L.a(rtcc_set_date_lib.o)
 .reginfo       0x00000000       0x18 C:/Program Files/Microchip/mplabc32/v1.12/bin/../lib/gcc/pic32mx/3.4.4/../../../../pic32mx/lib/size\libmchp_peripheral_32MX360F512L.a(rtcc_set_date_lib.o)
 .pdr           0x00000000       0x20 C:/Program Files/Microchip/mplabc32/v1.12/bin/../lib/gcc/pic32mx/3.4.4/../../../../pic32mx/lib/size\libmchp_peripheral_32MX360F512L.a(rtcc_set_date_lib.o)
 .text          0x00000000        0x0 C:/Program Files/Microchip/mplabc32/v1.12/bin/../lib/gcc/pic32mx/3.4.4/../../../../pic32mx/lib/size\libmchp_peripheral_32MX360F512L.a(rtcc_set_time_lib.o)
 .data          0x00000000        0x0 C:/Program Files/Microchip/mplabc32/v1.12/bin/../lib/gcc/pic32mx/3.4.4/../../../../pic32mx/lib/size\libmchp_peripheral_32MX360F512L.a(rtcc_set_time_lib.o)
 .bss           0x00000000        0x0 C:/Program Files/Microchip/mplabc32/v1.12/bin/../lib/gcc/pic32mx/3.4.4/../../../../pic32mx/lib/size\libmchp_peripheral_32MX360F512L.a(rtcc_set_time_lib.o)
 .reginfo       0x00000000       0x18 C:/Program Files/Microchip/mplabc32/v1.12/bin/../lib/gcc/pic32mx/3.4.4/../../../../pic32mx/lib/size\libmchp_peripheral_32MX360F512L.a(rtcc_set_time_lib.o)
 .pdr           0x00000000       0x20 C:/Program Files/Microchip/mplabc32/v1.12/bin/../lib/gcc/pic32mx/3.4.4/../../../../pic32mx/lib/size\libmchp_peripheral_32MX360F512L.a(rtcc_set_time_lib.o)
 .text          0x00000000        0x0 C:/Program Files/Microchip/mplabc32/v1.12/bin/../lib/gcc/pic32mx/3.4.4/../../../../pic32mx/lib/size\libmchp_peripheral_32MX360F512L.a(spi_getc_spi2_lib_legacy.o)
 .data          0x00000000        0x0 C:/Program Files/Microchip/mplabc32/v1.12/bin/../lib/gcc/pic32mx/3.4.4/../../../../pic32mx/lib/size\libmchp_peripheral_32MX360F512L.a(spi_getc_spi2_lib_legacy.o)
 .bss           0x00000000        0x0 C:/Program Files/Microchip/mplabc32/v1.12/bin/../lib/gcc/pic32mx/3.4.4/../../../../pic32mx/lib/size\libmchp_peripheral_32MX360F512L.a(spi_getc_spi2_lib_legacy.o)
 .reginfo       0x00000000       0x18 C:/Program Files/Microchip/mplabc32/v1.12/bin/../lib/gcc/pic32mx/3.4.4/../../../../pic32mx/lib/size\libmchp_peripheral_32MX360F512L.a(spi_getc_spi2_lib_legacy.o)
 .pdr           0x00000000       0x20 C:/Program Files/Microchip/mplabc32/v1.12/bin/../lib/gcc/pic32mx/3.4.4/../../../../pic32mx/lib/size\libmchp_peripheral_32MX360F512L.a(spi_getc_spi2_lib_legacy.o)
 .text.getcSPI2
                0x00000000       0x24 C:/Program Files/Microchip/mplabc32/v1.12/bin/../lib/gcc/pic32mx/3.4.4/../../../../pic32mx/lib/size\libmchp_peripheral_32MX360F512L.a(spi_getc_spi2_lib_legacy.o)
 .text          0x00000000        0x0 C:/Program Files/Microchip/mplabc32/v1.12/bin/../lib/gcc/pic32mx/3.4.4/../../../../pic32mx/lib/size\libmchp_peripheral_32MX360F512L.a(spi_open_spi2_lib_legacy.o)
 .data          0x00000000        0x0 C:/Program Files/Microchip/mplabc32/v1.12/bin/../lib/gcc/pic32mx/3.4.4/../../../../pic32mx/lib/size\libmchp_peripheral_32MX360F512L.a(spi_open_spi2_lib_legacy.o)
 .bss           0x00000000        0x0 C:/Program Files/Microchip/mplabc32/v1.12/bin/../lib/gcc/pic32mx/3.4.4/../../../../pic32mx/lib/size\libmchp_peripheral_32MX360F512L.a(spi_open_spi2_lib_legacy.o)
 .reginfo       0x00000000       0x18 C:/Program Files/Microchip/mplabc32/v1.12/bin/../lib/gcc/pic32mx/3.4.4/../../../../pic32mx/lib/size\libmchp_peripheral_32MX360F512L.a(spi_open_spi2_lib_legacy.o)
 .pdr           0x00000000       0x20 C:/Program Files/Microchip/mplabc32/v1.12/bin/../lib/gcc/pic32mx/3.4.4/../../../../pic32mx/lib/size\libmchp_peripheral_32MX360F512L.a(spi_open_spi2_lib_legacy.o)
 .text.OpenSPI2
                0x00000000       0x64 C:/Program Files/Microchip/mplabc32/v1.12/bin/../lib/gcc/pic32mx/3.4.4/../../../../pic32mx/lib/size\libmchp_peripheral_32MX360F512L.a(spi_open_spi2_lib_legacy.o)
 .text          0x00000000        0x0 C:/Program Files/Microchip/mplabc32/v1.12/bin/../lib/gcc/pic32mx/3.4.4/../../../../pic32mx/lib/size\libmchp_peripheral_32MX360F512L.a(spi_brg_tbl_lib_legacy.o)
 .data          0x00000000        0x0 C:/Program Files/Microchip/mplabc32/v1.12/bin/../lib/gcc/pic32mx/3.4.4/../../../../pic32mx/lib/size\libmchp_peripheral_32MX360F512L.a(spi_brg_tbl_lib_legacy.o)
 .bss           0x00000000        0x0 C:/Program Files/Microchip/mplabc32/v1.12/bin/../lib/gcc/pic32mx/3.4.4/../../../../pic32mx/lib/size\libmchp_peripheral_32MX360F512L.a(spi_brg_tbl_lib_legacy.o)
 .reginfo       0x00000000       0x18 C:/Program Files/Microchip/mplabc32/v1.12/bin/../lib/gcc/pic32mx/3.4.4/../../../../pic32mx/lib/size\libmchp_peripheral_32MX360F512L.a(spi_brg_tbl_lib_legacy.o)
 .pdr           0x00000000        0x0 C:/Program Files/Microchip/mplabc32/v1.12/bin/../lib/gcc/pic32mx/3.4.4/../../../../pic32mx/lib/size\libmchp_peripheral_32MX360F512L.a(spi_brg_tbl_lib_legacy.o)
 .rodata._SpiBrgConvTbl
                0x00000000       0x80 C:/Program Files/Microchip/mplabc32/v1.12/bin/../lib/gcc/pic32mx/3.4.4/../../../../pic32mx/lib/size\libmchp_peripheral_32MX360F512L.a(spi_brg_tbl_lib_legacy.o)
 .text          0x00000000        0x0 C:/Program Files/Microchip/mplabc32/v1.12/bin/../lib/gcc/pic32mx/3.4.4/../../../../pic32mx/lib/size\libmchp_peripheral_32MX360F512L.a(int_enable_interrupts_lib.o)
 .data          0x00000000        0x0 C:/Program Files/Microchip/mplabc32/v1.12/bin/../lib/gcc/pic32mx/3.4.4/../../../../pic32mx/lib/size\libmchp_peripheral_32MX360F512L.a(int_enable_interrupts_lib.o)
 .bss           0x00000000        0x0 C:/Program Files/Microchip/mplabc32/v1.12/bin/../lib/gcc/pic32mx/3.4.4/../../../../pic32mx/lib/size\libmchp_peripheral_32MX360F512L.a(int_enable_interrupts_lib.o)
 .reginfo       0x00000000       0x18 C:/Program Files/Microchip/mplabc32/v1.12/bin/../lib/gcc/pic32mx/3.4.4/../../../../pic32mx/lib/size\libmchp_peripheral_32MX360F512L.a(int_enable_interrupts_lib.o)
 .pdr           0x00000000       0x20 C:/Program Files/Microchip/mplabc32/v1.12/bin/../lib/gcc/pic32mx/3.4.4/../../../../pic32mx/lib/size\libmchp_peripheral_32MX360F512L.a(int_enable_interrupts_lib.o)
 .text          0x00000000        0x0 C:/Program Files/Microchip/mplabc32/v1.12/bin/../lib/gcc/pic32mx/3.4.4/../../../../pic32mx/lib/size\libmchp_peripheral_32MX360F512L.a(int_tbl_lib.o)
 .data          0x00000000        0x0 C:/Program Files/Microchip/mplabc32/v1.12/bin/../lib/gcc/pic32mx/3.4.4/../../../../pic32mx/lib/size\libmchp_peripheral_32MX360F512L.a(int_tbl_lib.o)
 .bss           0x00000000        0x0 C:/Program Files/Microchip/mplabc32/v1.12/bin/../lib/gcc/pic32mx/3.4.4/../../../../pic32mx/lib/size\libmchp_peripheral_32MX360F512L.a(int_tbl_lib.o)
 .reginfo       0x00000000       0x18 C:/Program Files/Microchip/mplabc32/v1.12/bin/../lib/gcc/pic32mx/3.4.4/../../../../pic32mx/lib/size\libmchp_peripheral_32MX360F512L.a(int_tbl_lib.o)
 .pdr           0x00000000      0x120 C:/Program Files/Microchip/mplabc32/v1.12/bin/../lib/gcc/pic32mx/3.4.4/../../../../pic32mx/lib/size\libmchp_peripheral_32MX360F512L.a(int_tbl_lib.o)
 .rodata.__IntVectorTbl
                0x00000000      0x228 C:/Program Files/Microchip/mplabc32/v1.12/bin/../lib/gcc/pic32mx/3.4.4/../../../../pic32mx/lib/size\libmchp_peripheral_32MX360F512L.a(int_tbl_lib.o)
 .text.INTSetFlag
                0x00000000       0x28 C:/Program Files/Microchip/mplabc32/v1.12/bin/../lib/gcc/pic32mx/3.4.4/../../../../pic32mx/lib/size\libmchp_peripheral_32MX360F512L.a(int_tbl_lib.o)
 .text.INTGetFlag
                0x00000000       0x28 C:/Program Files/Microchip/mplabc32/v1.12/bin/../lib/gcc/pic32mx/3.4.4/../../../../pic32mx/lib/size\libmchp_peripheral_32MX360F512L.a(int_tbl_lib.o)
 .text.INTGetEnable
                0x00000000       0x28 C:/Program Files/Microchip/mplabc32/v1.12/bin/../lib/gcc/pic32mx/3.4.4/../../../../pic32mx/lib/size\libmchp_peripheral_32MX360F512L.a(int_tbl_lib.o)
 .text.INTSetVectorPriority
                0x00000000       0x3c C:/Program Files/Microchip/mplabc32/v1.12/bin/../lib/gcc/pic32mx/3.4.4/../../../../pic32mx/lib/size\libmchp_peripheral_32MX360F512L.a(int_tbl_lib.o)
 .text.INTGetVectorPriority
                0x00000000       0x2c C:/Program Files/Microchip/mplabc32/v1.12/bin/../lib/gcc/pic32mx/3.4.4/../../../../pic32mx/lib/size\libmchp_peripheral_32MX360F512L.a(int_tbl_lib.o)
 .text.INTSetVectorSubPriority
                0x00000000       0x3c C:/Program Files/Microchip/mplabc32/v1.12/bin/../lib/gcc/pic32mx/3.4.4/../../../../pic32mx/lib/size\libmchp_peripheral_32MX360F512L.a(int_tbl_lib.o)
 .text.INTGetVectorSubPriority
                0x00000000       0x2c C:/Program Files/Microchip/mplabc32/v1.12/bin/../lib/gcc/pic32mx/3.4.4/../../../../pic32mx/lib/size\libmchp_peripheral_32MX360F512L.a(int_tbl_lib.o)
 .text          0x00000000        0x0 C:/Program Files/Microchip/mplabc32/v1.12/bin/../lib/gcc/pic32mx/3.4.4/../../../../pic32mx/lib/size\libmchp_peripheral_32MX360F512L.a(_rtcc_set_time_and_date_lib.o)
 .data          0x00000000        0x0 C:/Program Files/Microchip/mplabc32/v1.12/bin/../lib/gcc/pic32mx/3.4.4/../../../../pic32mx/lib/size\libmchp_peripheral_32MX360F512L.a(_rtcc_set_time_and_date_lib.o)
 .bss           0x00000000        0x0 C:/Program Files/Microchip/mplabc32/v1.12/bin/../lib/gcc/pic32mx/3.4.4/../../../../pic32mx/lib/size\libmchp_peripheral_32MX360F512L.a(_rtcc_set_time_and_date_lib.o)
 .reginfo       0x00000000       0x18 C:/Program Files/Microchip/mplabc32/v1.12/bin/../lib/gcc/pic32mx/3.4.4/../../../../pic32mx/lib/size\libmchp_peripheral_32MX360F512L.a(_rtcc_set_time_and_date_lib.o)
 .pdr           0x00000000       0x20 C:/Program Files/Microchip/mplabc32/v1.12/bin/../lib/gcc/pic32mx/3.4.4/../../../../pic32mx/lib/size\libmchp_peripheral_32MX360F512L.a(_rtcc_set_time_and_date_lib.o)
 .text          0x00000000        0x0 C:/Program Files/Microchip/mplabc32/v1.12/bin/../lib/gcc/pic32mx/3.4.4/../../../../pic32mx/lib/size\libmchp_peripheral_32MX360F512L.a(_rtcc_wait_clock_off_lib.o)
 .data          0x00000000        0x0 C:/Program Files/Microchip/mplabc32/v1.12/bin/../lib/gcc/pic32mx/3.4.4/../../../../pic32mx/lib/size\libmchp_peripheral_32MX360F512L.a(_rtcc_wait_clock_off_lib.o)
 .bss           0x00000000        0x0 C:/Program Files/Microchip/mplabc32/v1.12/bin/../lib/gcc/pic32mx/3.4.4/../../../../pic32mx/lib/size\libmchp_peripheral_32MX360F512L.a(_rtcc_wait_clock_off_lib.o)
 .reginfo       0x00000000       0x18 C:/Program Files/Microchip/mplabc32/v1.12/bin/../lib/gcc/pic32mx/3.4.4/../../../../pic32mx/lib/size\libmchp_peripheral_32MX360F512L.a(_rtcc_wait_clock_off_lib.o)
 .pdr           0x00000000       0x40 C:/Program Files/Microchip/mplabc32/v1.12/bin/../lib/gcc/pic32mx/3.4.4/../../../../pic32mx/lib/size\libmchp_peripheral_32MX360F512L.a(_rtcc_wait_clock_off_lib.o)
 .text._RtccSetClockWait
                0x00000000       0x14 C:/Program Files/Microchip/mplabc32/v1.12/bin/../lib/gcc/pic32mx/3.4.4/../../../../pic32mx/lib/size\libmchp_peripheral_32MX360F512L.a(_rtcc_wait_clock_off_lib.o)
 .text          0x00000000        0x0 C:/Program Files/Microchip/mplabc32/v1.12/bin/../lib/gcc/pic32mx/3.4.4/../../../../pic32mx/lib/size\libmchp_peripheral_32MX360F512L.a(read_core_timer_lib.o)
 .data          0x00000000        0x0 C:/Program Files/Microchip/mplabc32/v1.12/bin/../lib/gcc/pic32mx/3.4.4/../../../../pic32mx/lib/size\libmchp_peripheral_32MX360F512L.a(read_core_timer_lib.o)
 .bss           0x00000000        0x0 C:/Program Files/Microchip/mplabc32/v1.12/bin/../lib/gcc/pic32mx/3.4.4/../../../../pic32mx/lib/size\libmchp_peripheral_32MX360F512L.a(read_core_timer_lib.o)
 .reginfo       0x00000000       0x18 C:/Program Files/Microchip/mplabc32/v1.12/bin/../lib/gcc/pic32mx/3.4.4/../../../../pic32mx/lib/size\libmchp_peripheral_32MX360F512L.a(read_core_timer_lib.o)
 .pdr           0x00000000       0x20 C:/Program Files/Microchip/mplabc32/v1.12/bin/../lib/gcc/pic32mx/3.4.4/../../../../pic32mx/lib/size\libmchp_peripheral_32MX360F512L.a(read_core_timer_lib.o)
 .text          0x00000000        0x0 C:/Program Files/Microchip/mplabc32/v1.12/bin/../lib/gcc/pic32mx/3.4.4/../../../../pic32mx/lib/./proc/32MX360F512L\processor.o
 .data          0x00000000        0x0 C:/Program Files/Microchip/mplabc32/v1.12/bin/../lib/gcc/pic32mx/3.4.4/../../../../pic32mx/lib/./proc/32MX360F512L\processor.o
 .bss           0x00000000        0x0 C:/Program Files/Microchip/mplabc32/v1.12/bin/../lib/gcc/pic32mx/3.4.4/../../../../pic32mx/lib/./proc/32MX360F512L\processor.o
 .reginfo       0x00000000       0x18 C:/Program Files/Microchip/mplabc32/v1.12/bin/../lib/gcc/pic32mx/3.4.4/../../../../pic32mx/lib/./proc/32MX360F512L\processor.o
 .pdr           0x00000000        0x0 C:/Program Files/Microchip/mplabc32/v1.12/bin/../lib/gcc/pic32mx/3.4.4/../../../../pic32mx/lib/./proc/32MX360F512L\processor.o

Memory Configuration

Name             Origin             Length             Attributes
kseg0_program_mem 0x9d000000         0x00080000         xr
kseg0_boot_mem   0x9fc00490         0x00000970
exception_mem    0x9fc01000         0x00001000
kseg1_boot_mem   0xbfc00000         0x00000490
debug_exec_mem   0xbfc02000         0x00000ff0
config3          0xbfc02ff0         0x00000004
config2          0xbfc02ff4         0x00000004
config1          0xbfc02ff8         0x00000004
config0          0xbfc02ffc         0x00000004
kseg1_data_mem   0xa0000000         0x00008000         w !x
sfrs             0xbf800000         0x00100000
configsfrs       0xbfc02ff0         0x00000010
*default*        0x00000000         0xffffffff

Linker script and memory map

LOAD C:/Program Files/Microchip/mplabc32/v1.12/bin/../lib/gcc/pic32mx/3.4.4/../../../../pic32mx/lib/size/crt0.o
LOAD output_pic32_ssd1963\MainDemo.o
LOAD output_pic32_ssd1963\rtcc.o
LOAD output_pic32_ssd1963\Fonts.o
LOAD output_pic32_ssd1963\DemoSelection.o
LOAD output_pic32_ssd1963\Animation.o
LOAD output_pic32_ssd1963\AnimationBitmaps.o
LOAD output_pic32_ssd1963\ECG.o
LOAD output_pic32_ssd1963\Games.o
LOAD output_pic32_ssd1963\SnakeBitmaps.o
LOAD output_pic32_ssd1963\ECGBitmaps.o
LOAD output_pic32_ssd1963\RGBDemo.o
LOAD output_pic32_ssd1963\MultiFontsDemo.o
LOAD output_pic32_ssd1963\HelloWorldFonts.o
LOAD output_pic32_ssd1963\TimeDateDemo.o
LOAD output_pic32_ssd1963\DrawTool.o
LOAD output_pic32_ssd1963\SlideShowDemo.o
LOAD output_pic32_ssd1963\Icons.o
LOAD output_pic32_ssd1963\DemoSteps.o
LOAD output_pic32_ssd1963\SideButtons.o
LOAD output_pic32_ssd1963\BitmapFile.o
LOAD output_pic32_ssd1963\GraphShow.o
LOAD output_pic32_ssd1963\FSIO.o
LOAD output_pic32_ssd1963\SD-SPI.o
LOAD output_pic32_ssd1963\JpegDecoder.o
LOAD output_pic32_ssd1963\BmpDecoder.o
LOAD output_pic32_ssd1963\GifDecoder.o
LOAD output_pic32_ssd1963\ImageDecoder.o
LOAD output_pic32_ssd1963\jidctint.o
LOAD output_pic32_ssd1963\TouchScreen.o
LOAD output_pic32_ssd1963\Beep.o
LOAD output_pic32_ssd1963\EEPROM.o
LOAD output_pic32_ssd1963\Window.o
LOAD output_pic32_ssd1963\Button.o
LOAD output_pic32_ssd1963\Chart.o
LOAD output_pic32_ssd1963\CheckBox.o
LOAD output_pic32_ssd1963\DisplayDriver.o
LOAD output_pic32_ssd1963\EditBox.o
LOAD output_pic32_ssd1963\Grid.o
LOAD output_pic32_ssd1963\GroupBox.o
LOAD output_pic32_ssd1963\ListBox.o
LOAD output_pic32_ssd1963\Meter.o
LOAD output_pic32_ssd1963\Picture.o
LOAD output_pic32_ssd1963\Primitive.o
LOAD output_pic32_ssd1963\RadioButton.o
LOAD output_pic32_ssd1963\Slider.o
LOAD output_pic32_ssd1963\StaticText.o
LOAD output_pic32_ssd1963\GOLFontDefault.o
LOAD output_pic32_ssd1963\GOL.o
LOAD output_pic32_ssd1963\uart2.o
LOAD output_pic32_ssd1963\JPEGDemo.o
LOAD output_pic32_ssd1963\IconsC32.o
LOAD output_pic32_ssd1963\SlideShowC32.o
LOAD output_pic32_ssd1963\vs1003b.o
                0x00000001                __MPLAB_BUILD = 0x1
                0x00002400                _min_heap_size = 0x2400
                0x00000800                _min_stack_size = 0x800
LOAD C:/Program Files/Microchip/mplabc32/v1.12/bin/../lib/gcc/pic32mx/3.4.4/size\libgcc.a
START GROUP
LOAD C:/Program Files/Microchip/mplabc32/v1.12/bin/../lib/gcc/pic32mx/3.4.4/../../../../pic32mx/lib/size\libdebug.a
LOAD C:/Program Files/Microchip/mplabc32/v1.12/bin/../lib/gcc/pic32mx/3.4.4/../../../../pic32mx/lib/size\libc.a
LOAD C:/Program Files/Microchip/mplabc32/v1.12/bin/../lib/gcc/pic32mx/3.4.4/../../../../pic32mx/lib/size\libm.a
LOAD C:/Program Files/Microchip/mplabc32/v1.12/bin/../lib/gcc/pic32mx/3.4.4/../../../../pic32mx/lib/size\libe.a
LOAD C:/Program Files/Microchip/mplabc32/v1.12/bin/../lib/gcc/pic32mx/3.4.4/../../../../pic32mx/lib/size\libdsp.a
LOAD C:/Program Files/Microchip/mplabc32/v1.12/bin/../lib/gcc/pic32mx/3.4.4/../../../../pic32mx/lib/size\libmchp_peripheral.a
LOAD C:/Program Files/Microchip/mplabc32/v1.12/bin/../lib/gcc/pic32mx/3.4.4/../../../../pic32mx/lib/size\libmchp_peripheral_32MX360F512L.a
END GROUP
LOAD C:/Program Files/Microchip/mplabc32/v1.12/bin/../lib/gcc/pic32mx/3.4.4/size\libgcc.a
                0x00000400                PROVIDE (_min_stack_size, 0x400)
                0x00000000                PROVIDE (_min_heap_size, 0x0)
LOAD C:/Program Files/Microchip/mplabc32/v1.12/bin/../lib/gcc/pic32mx/3.4.4/../../../../pic32mx/lib/./proc/32MX360F512L\processor.o
                0x00000001                PROVIDE (_vector_spacing, 0x1)
                0x9fc01000                _ebase_address = 0x9fc01000
                0xbfc00000                _RESET_ADDR = 0xbfc00000
                0xbfc00380                _BEV_EXCPT_ADDR = 0xbfc00380
                0xbfc00480                _DBG_EXCPT_ADDR = 0xbfc00480
                0xbfc02000                _DBG_CODE_ADDR = 0xbfc02000
                0x9fc01180                _GEN_EXCPT_ADDR = (_ebase_address + 0x180)

.config_BFC02FF0
 *(.config_BFC02FF0)

.config_BFC02FF4
                0xbfc02ff4        0x4
 *(.config_BFC02FF4)
 .config_BFC02FF4
                0xbfc02ff4        0x4 output_pic32_ssd1963\MainDemo.o

.config_BFC02FF8
                0xbfc02ff8        0x4
 *(.config_BFC02FF8)
 .config_BFC02FF8
                0xbfc02ff8        0x4 output_pic32_ssd1963\MainDemo.o

.config_BFC02FFC
                0xbfc02ffc        0x4
 *(.config_BFC02FFC)
 .config_BFC02FFC
                0xbfc02ffc        0x4 output_pic32_ssd1963\MainDemo.o

.reset          0xbfc00000       0x10
 *(.reset)
 .reset         0xbfc00000       0x10 C:/Program Files/Microchip/mplabc32/v1.12/bin/../lib/gcc/pic32mx/3.4.4/../../../../pic32mx/lib/size/crt0.o
                0xbfc00000                _reset

.bev_excpt      0xbfc00380       0x10
 *(.bev_handler)
 .bev_handler   0xbfc00380       0x10 C:/Program Files/Microchip/mplabc32/v1.12/bin/../lib/gcc/pic32mx/3.4.4/../../../../pic32mx/lib/size/crt0.o

.dbg_excpt      0xbfc00480        0x0
                0xbfc00480                . = (. + DEFINED (_DEBUGGER)?0x8:0x0)

.dbg_code       0xbfc02000        0x0
                0xbfc02000                . = (. + DEFINED (_DEBUGGER)?0xff0:0x0)

.app_excpt      0x9fc01180       0x10
 *(.gen_handler)
 .gen_handler   0x9fc01180       0x10 C:/Program Files/Microchip/mplabc32/v1.12/bin/../lib/gcc/pic32mx/3.4.4/../../../../pic32mx/lib/size/crt0.o

.vector_0       0x9fc01200        0x0
 *(.vector_0)
                0x00000001                ASSERT (((_vector_spacing == 0x0) || (SIZEOF (.vector_0) <= (_vector_spacing << 0x5))), function at exception vector 0 too large)

.vector_1       0x9fc01220        0x0
 *(.vector_1)
                0x00000001                ASSERT (((_vector_spacing == 0x0) || (SIZEOF (.vector_1) <= (_vector_spacing << 0x5))), function at exception vector 1 too large)

.vector_2       0x9fc01240        0x0
 *(.vector_2)
                0x00000001                ASSERT (((_vector_spacing == 0x0) || (SIZEOF (.vector_2) <= (_vector_spacing << 0x5))), function at exception vector 2 too large)

.vector_3       0x9fc01260        0x0
 *(.vector_3)
                0x00000001                ASSERT (((_vector_spacing == 0x0) || (SIZEOF (.vector_3) <= (_vector_spacing << 0x5))), function at exception vector 3 too large)

.vector_4       0x9fc01280        0x0
 *(.vector_4)
                0x00000001                ASSERT (((_vector_spacing == 0x0) || (SIZEOF (.vector_4) <= (_vector_spacing << 0x5))), function at exception vector 4 too large)

.vector_5       0x9fc012a0        0x0
 *(.vector_5)
                0x00000001                ASSERT (((_vector_spacing == 0x0) || (SIZEOF (.vector_5) <= (_vector_spacing << 0x5))), function at exception vector 5 too large)

.vector_6       0x9fc012c0        0x0
 *(.vector_6)
                0x00000001                ASSERT (((_vector_spacing == 0x0) || (SIZEOF (.vector_6) <= (_vector_spacing << 0x5))), function at exception vector 6 too large)

.vector_7       0x9fc012e0        0x0
 *(.vector_7)
                0x00000001                ASSERT (((_vector_spacing == 0x0) || (SIZEOF (.vector_7) <= (_vector_spacing << 0x5))), function at exception vector 7 too large)

.vector_8       0x9fc01300        0x8
 *(.vector_8)
 .vector_8      0x9fc01300        0x8 output_pic32_ssd1963\Beep.o
                0x00000001                ASSERT (((_vector_spacing == 0x0) || (SIZEOF (.vector_8) <= (_vector_spacing << 0x5))), function at exception vector 8 too large)

.vector_9       0x9fc01320        0x0
 *(.vector_9)
                0x00000001                ASSERT (((_vector_spacing == 0x0) || (SIZEOF (.vector_9) <= (_vector_spacing << 0x5))), function at exception vector 9 too large)

.vector_10      0x9fc01340        0x0
 *(.vector_10)
                0x00000001                ASSERT (((_vector_spacing == 0x0) || (SIZEOF (.vector_10) <= (_vector_spacing << 0x5))), function at exception vector 10 too large)

.vector_11      0x9fc01360        0x0
 *(.vector_11)
                0x00000001                ASSERT (((_vector_spacing == 0x0) || (SIZEOF (.vector_11) <= (_vector_spacing << 0x5))), function at exception vector 11 too large)

.vector_12      0x9fc01380        0x8
 *(.vector_12)
 .vector_12     0x9fc01380        0x8 output_pic32_ssd1963\TouchScreen.o
                0x00000001                ASSERT (((_vector_spacing == 0x0) || (SIZEOF (.vector_12) <= (_vector_spacing << 0x5))), function at exception vector 12 too large)

.vector_13      0x9fc013a0        0x0
 *(.vector_13)
                0x00000001                ASSERT (((_vector_spacing == 0x0) || (SIZEOF (.vector_13) <= (_vector_spacing << 0x5))), function at exception vector 13 too large)

.vector_14      0x9fc013c0        0x0
 *(.vector_14)
                0x00000001                ASSERT (((_vector_spacing == 0x0) || (SIZEOF (.vector_14) <= (_vector_spacing << 0x5))), function at exception vector 14 too large)

.vector_15      0x9fc013e0        0x0
 *(.vector_15)
                0x00000001                ASSERT (((_vector_spacing == 0x0) || (SIZEOF (.vector_15) <= (_vector_spacing << 0x5))), function at exception vector 15 too large)

.vector_16      0x9fc01400        0x8
 *(.vector_16)
 .vector_16     0x9fc01400        0x8 output_pic32_ssd1963\MainDemo.o
                0x00000001                ASSERT (((_vector_spacing == 0x0) || (SIZEOF (.vector_16) <= (_vector_spacing << 0x5))), function at exception vector 16 too large)

.vector_17      0x9fc01420        0x0
 *(.vector_17)
                0x00000001                ASSERT (((_vector_spacing == 0x0) || (SIZEOF (.vector_17) <= (_vector_spacing << 0x5))), function at exception vector 17 too large)

.vector_18      0x9fc01440        0x0
 *(.vector_18)
                0x00000001                ASSERT (((_vector_spacing == 0x0) || (SIZEOF (.vector_18) <= (_vector_spacing << 0x5))), function at exception vector 18 too large)

.vector_19      0x9fc01460        0x0
 *(.vector_19)
                0x00000001                ASSERT (((_vector_spacing == 0x0) || (SIZEOF (.vector_19) <= (_vector_spacing << 0x5))), function at exception vector 19 too large)

.vector_20      0x9fc01480        0x0
 *(.vector_20)
                0x00000001                ASSERT (((_vector_spacing == 0x0) || (SIZEOF (.vector_20) <= (_vector_spacing << 0x5))), function at exception vector 20 too large)

.vector_21      0x9fc014a0        0x0
 *(.vector_21)
                0x00000001                ASSERT (((_vector_spacing == 0x0) || (SIZEOF (.vector_21) <= (_vector_spacing << 0x5))), function at exception vector 21 too large)

.vector_22      0x9fc014c0        0x0
 *(.vector_22)
                0x00000001                ASSERT (((_vector_spacing == 0x0) || (SIZEOF (.vector_22) <= (_vector_spacing << 0x5))), function at exception vector 22 too large)

.vector_23      0x9fc014e0        0x0
 *(.vector_23)
                0x00000001                ASSERT (((_vector_spacing == 0x0) || (SIZEOF (.vector_23) <= (_vector_spacing << 0x5))), function at exception vector 23 too large)

.vector_24      0x9fc01500        0x0
 *(.vector_24)
                0x00000001                ASSERT (((_vector_spacing == 0x0) || (SIZEOF (.vector_24) <= (_vector_spacing << 0x5))), function at exception vector 24 too large)

.vector_25      0x9fc01520        0x0
 *(.vector_25)
                0x00000001                ASSERT (((_vector_spacing == 0x0) || (SIZEOF (.vector_25) <= (_vector_spacing << 0x5))), function at exception vector 25 too large)

.vector_26      0x9fc01540        0x0
 *(.vector_26)
                0x00000001                ASSERT (((_vector_spacing == 0x0) || (SIZEOF (.vector_26) <= (_vector_spacing << 0x5))), function at exception vector 26 too large)

.vector_27      0x9fc01560        0x0
 *(.vector_27)
                0x00000001                ASSERT (((_vector_spacing == 0x0) || (SIZEOF (.vector_27) <= (_vector_spacing << 0x5))), function at exception vector 27 too large)

.vector_28      0x9fc01580        0x0
 *(.vector_28)
                0x00000001                ASSERT (((_vector_spacing == 0x0) || (SIZEOF (.vector_28) <= (_vector_spacing << 0x5))), function at exception vector 28 too large)

.vector_29      0x9fc015a0        0x0
 *(.vector_29)
                0x00000001                ASSERT (((_vector_spacing == 0x0) || (SIZEOF (.vector_29) <= (_vector_spacing << 0x5))), function at exception vector 29 too large)

.vector_30      0x9fc015c0        0x0
 *(.vector_30)
                0x00000001                ASSERT (((_vector_spacing == 0x0) || (SIZEOF (.vector_30) <= (_vector_spacing << 0x5))), function at exception vector 30 too large)

.vector_31      0x9fc015e0        0x0
 *(.vector_31)
                0x00000001                ASSERT (((_vector_spacing == 0x0) || (SIZEOF (.vector_31) <= (_vector_spacing << 0x5))), function at exception vector 31 too large)

.vector_32      0x9fc01600        0x0
 *(.vector_32)
                0x00000001                ASSERT (((_vector_spacing == 0x0) || (SIZEOF (.vector_32) <= (_vector_spacing << 0x5))), function at exception vector 32 too large)

.vector_33      0x9fc01620        0x0
 *(.vector_33)
                0x00000001                ASSERT (((_vector_spacing == 0x0) || (SIZEOF (.vector_33) <= (_vector_spacing << 0x5))), function at exception vector 33 too large)

.vector_34      0x9fc01640        0x0
 *(.vector_34)
                0x00000001                ASSERT (((_vector_spacing == 0x0) || (SIZEOF (.vector_34) <= (_vector_spacing << 0x5))), function at exception vector 34 too large)

.vector_35      0x9fc01660        0x0
 *(.vector_35)
                0x00000001                ASSERT (((_vector_spacing == 0x0) || (SIZEOF (.vector_35) <= (_vector_spacing << 0x5))), function at exception vector 35 too large)

.vector_36      0x9fc01680        0x0
 *(.vector_36)
                0x00000001                ASSERT (((_vector_spacing == 0x0) || (SIZEOF (.vector_36) <= (_vector_spacing << 0x5))), function at exception vector 36 too large)

.vector_37      0x9fc016a0        0x0
 *(.vector_37)
                0x00000001                ASSERT (((_vector_spacing == 0x0) || (SIZEOF (.vector_37) <= (_vector_spacing << 0x5))), function at exception vector 37 too large)

.vector_38      0x9fc016c0        0x0
 *(.vector_38)
                0x00000001                ASSERT (((_vector_spacing == 0x0) || (SIZEOF (.vector_38) <= (_vector_spacing << 0x5))), function at exception vector 38 too large)

.vector_39      0x9fc016e0        0x0
 *(.vector_39)
                0x00000001                ASSERT (((_vector_spacing == 0x0) || (SIZEOF (.vector_39) <= (_vector_spacing << 0x5))), function at exception vector 39 too large)

.vector_40      0x9fc01700        0x0
 *(.vector_40)
                0x00000001                ASSERT (((_vector_spacing == 0x0) || (SIZEOF (.vector_40) <= (_vector_spacing << 0x5))), function at exception vector 40 too large)

.vector_41      0x9fc01720        0x0
 *(.vector_41)
                0x00000001                ASSERT (((_vector_spacing == 0x0) || (SIZEOF (.vector_41) <= (_vector_spacing << 0x5))), function at exception vector 41 too large)

.vector_42      0x9fc01740        0x0
 *(.vector_42)
                0x00000001                ASSERT (((_vector_spacing == 0x0) || (SIZEOF (.vector_42) <= (_vector_spacing << 0x5))), function at exception vector 42 too large)

.vector_43      0x9fc01760        0x0
 *(.vector_43)
                0x00000001                ASSERT (((_vector_spacing == 0x0) || (SIZEOF (.vector_43) <= (_vector_spacing << 0x5))), function at exception vector 43 too large)

.vector_44      0x9fc01780        0x0
 *(.vector_44)
                0x00000001                ASSERT (((_vector_spacing == 0x0) || (SIZEOF (.vector_44) <= (_vector_spacing << 0x5))), function at exception vector 44 too large)

.vector_45      0x9fc017a0        0x0
 *(.vector_45)
                0x00000001                ASSERT (((_vector_spacing == 0x0) || (SIZEOF (.vector_45) <= (_vector_spacing << 0x5))), function at exception vector 45 too large)

.vector_46      0x9fc017c0        0x0
 *(.vector_46)
                0x00000001                ASSERT (((_vector_spacing == 0x0) || (SIZEOF (.vector_46) <= (_vector_spacing << 0x5))), function at exception vector 46 too large)

.vector_47      0x9fc017e0        0x0
 *(.vector_47)
                0x00000001                ASSERT (((_vector_spacing == 0x0) || (SIZEOF (.vector_47) <= (_vector_spacing << 0x5))), function at exception vector 47 too large)

.vector_48      0x9fc01800        0x0
 *(.vector_48)
                0x00000001                ASSERT (((_vector_spacing == 0x0) || (SIZEOF (.vector_48) <= (_vector_spacing << 0x5))), function at exception vector 48 too large)

.vector_49      0x9fc01820        0x0
 *(.vector_49)
                0x00000001                ASSERT (((_vector_spacing == 0x0) || (SIZEOF (.vector_49) <= (_vector_spacing << 0x5))), function at exception vector 49 too large)

.vector_50      0x9fc01840        0x0
 *(.vector_50)
                0x00000001                ASSERT (((_vector_spacing == 0x0) || (SIZEOF (.vector_50) <= (_vector_spacing << 0x5))), function at exception vector 50 too large)

.vector_51      0x9fc01860        0x0
 *(.vector_51)
                0x00000001                ASSERT (((_vector_spacing == 0x0) || (SIZEOF (.vector_51) <= (_vector_spacing << 0x5))), function at exception vector 51 too large)

.vector_52      0x9fc01880        0x0
 *(.vector_52)
                0x00000001                ASSERT (((_vector_spacing == 0x0) || (SIZEOF (.vector_52) <= (_vector_spacing << 0x5))), function at exception vector 52 too large)

.vector_53      0x9fc018a0        0x0
 *(.vector_53)
                0x00000001                ASSERT (((_vector_spacing == 0x0) || (SIZEOF (.vector_53) <= (_vector_spacing << 0x5))), function at exception vector 53 too large)

.vector_54      0x9fc018c0        0x0
 *(.vector_54)
                0x00000001                ASSERT (((_vector_spacing == 0x0) || (SIZEOF (.vector_54) <= (_vector_spacing << 0x5))), function at exception vector 54 too large)

.vector_55      0x9fc018e0        0x0
 *(.vector_55)
                0x00000001                ASSERT (((_vector_spacing == 0x0) || (SIZEOF (.vector_55) <= (_vector_spacing << 0x5))), function at exception vector 55 too large)

.vector_56      0x9fc01900        0x0
 *(.vector_56)
                0x00000001                ASSERT (((_vector_spacing == 0x0) || (SIZEOF (.vector_56) <= (_vector_spacing << 0x5))), function at exception vector 56 too large)

.vector_57      0x9fc01920        0x0
 *(.vector_57)
                0x00000001                ASSERT (((_vector_spacing == 0x0) || (SIZEOF (.vector_57) <= (_vector_spacing << 0x5))), function at exception vector 57 too large)

.vector_58      0x9fc01940        0x0
 *(.vector_58)
                0x00000001                ASSERT (((_vector_spacing == 0x0) || (SIZEOF (.vector_58) <= (_vector_spacing << 0x5))), function at exception vector 58 too large)

.vector_59      0x9fc01960        0x0
 *(.vector_59)
                0x00000001                ASSERT (((_vector_spacing == 0x0) || (SIZEOF (.vector_59) <= (_vector_spacing << 0x5))), function at exception vector 59 too large)

.vector_60      0x9fc01980        0x0
 *(.vector_60)
                0x00000001                ASSERT (((_vector_spacing == 0x0) || (SIZEOF (.vector_60) <= (_vector_spacing << 0x5))), function at exception vector 60 too large)

.vector_61      0x9fc019a0        0x0
 *(.vector_61)
                0x00000001                ASSERT (((_vector_spacing == 0x0) || (SIZEOF (.vector_61) <= (_vector_spacing << 0x5))), function at exception vector 61 too large)

.vector_62      0x9fc019c0        0x0
 *(.vector_62)
                0x00000001                ASSERT (((_vector_spacing == 0x0) || (SIZEOF (.vector_62) <= (_vector_spacing << 0x5))), function at exception vector 62 too large)

.vector_63      0x9fc019e0        0x0
 *(.vector_63)
                0x00000001                ASSERT (((_vector_spacing == 0x0) || (SIZEOF (.vector_63) <= (_vector_spacing << 0x5))), function at exception vector 63 too large)

.startup        0x9fc00490      0x1e0
 *(.startup)
 .startup       0x9fc00490      0x1e0 C:/Program Files/Microchip/mplabc32/v1.12/bin/../lib/gcc/pic32mx/3.4.4/../../../../pic32mx/lib/size/crt0.o

.text           0x9d000000    0x1b754
                0x9d000000                _text_begin = .
 *(.text .stub .text.* .gnu.linkonce.t.*)
 .text          0x9d000000       0x10 C:/Program Files/Microchip/mplabc32/v1.12/bin/../lib/gcc/pic32mx/3.4.4/../../../../pic32mx/lib/size/crt0.o
                0x9d000008                __crt0_exit
 .text          0x9d000010      0xae8 output_pic32_ssd1963\MainDemo.o
                0x9d000010                main
                0x9d000350                GOLMsgCallback
                0x9d000444                GOLDrawCallback
                0x9d000674                StartScreen
                0x9d000890                CreateCtrlButtons
                0x9d0009c8                _T4Interrupt
                0x9d000a40                TickInit
                0x9d000ab4                ExternalMemoryCallback
 .text          0x9d000af8      0xa38 output_pic32_ssd1963\rtcc.o
                0x9d000af8                RTCCProcessEvents
                0x9d001038                RTCCInit
                0x9d001098                RTCCSet
                0x9d00110c                RTCCUnlock
                0x9d00113c                RTCCSetBinSec
                0x9d001198                RTCCSetBinMin
                0x9d0011f4                RTCCSetBinHour
                0x9d001250                RTCCCalculateWeekDay
                0x9d00134c                RTCCSetBinDay
                0x9d00143c                RTCCSetBinMonth
                0x9d001498                RTCCSetBinYear
 .text          0x9d001530      0x8f4 output_pic32_ssd1963\DemoSelection.o
                0x9d001530                CreateDemoSelection
                0x9d00159c                CreateDemoSelectionPage0
                0x9d0017ac                CreateDemoSelectionPage1
                0x9d0018f8                CheckDemoStatus
                0x9d00193c                MsgDemoSelection
                0x9d001df8                InitDemoSelectStyleScheme
 .text          0x9d001e24      0x700 output_pic32_ssd1963\Animation.o
                0x9d001e24                NextAnimation
                0x9d002038                CreateAnimation
                0x9d002350                MsgAnimation
                0x9d0024ec                InitAnimationStyleScheme
 .text          0x9d002524     0x11cc output_pic32_ssd1963\ECG.o
                0x9d002524                UpdateECG
                0x9d002888                CreateECG
                0x9d002980                GetECGSamples
                0x9d002a34                PanelECG
                0x9d002bb0                GraphECG
                0x9d002f18                MsgECG
                0x9d00304c                ECGDrawArrow
                0x9d0032fc                ECGCalculation
                0x9d00348c                GetPotSamples
                0x9d003540                ECGShortToString
                0x9d0036a4                GetNoise
                0x9d0036b4                InitECGStyleScheme
 .text          0x9d0036f0      0xd00 output_pic32_ssd1963\Games.o
                0x9d0036f0                InitializeRandomNumberGenerator
                0x9d003720                Random
                0x9d003778                DrawSnake
                0x9d003e14                ProcessMessageSnake
                0x9d003f54                ShowScreenSnake
                0x9d0041ac                ShowScreenScore
                0x9d0043e0                InitGamesStyleScheme
 .text          0x9d0043f0     0x1e88 output_pic32_ssd1963\RGBDemo.o
                0x9d0043f0                CreateRGBDemo
                0x9d004a30                RGBDemoMsgCallback
                0x9d005364                RGBDemoDrawCallback
                0x9d00595c                LoadLightData
                0x9d005964                Int2Str
                0x9d0059c4                FadeColorControl
                0x9d005bb4                ShowCurrentColor
                0x9d005c40                DrawColorPalette
                0x9d005d58                DrawIntensityLevel
                0x9d005f78                CalculatePaletteColor
                0x9d00614c                DrawColorPointer
                0x9d006238                UpdateColorPointer
 .text          0x9d006278      0x67c output_pic32_ssd1963\MultiFontsDemo.o
                0x9d006278                CreateMultiFontsDemo
                0x9d0063a0                AnimateText
                0x9d006564                MultiFontDemoMsgCallback
                0x9d006664                MultiFontDemoDrawCallback
                0x9d0066a8                InitHWData
 .text          0x9d0068f4     0x1090 output_pic32_ssd1963\TimeDateDemo.o
                0x9d0068f4                CreateTimeDateDemo
                0x9d006e84                TimeDateDemoMsgCallback
                0x9d007680                TimeDateDemoDrawCallback
                0x9d00790c                UpdateTimeVars
 .text          0x9d007984      0x618 output_pic32_ssd1963\DrawTool.o
                0x9d007984                CreateDrawTool
                0x9d007a08                CreateColorButtons
                0x9d007c84                DrawToolFrame
                0x9d007d34                DrawToolPad
                0x9d007d6c                MsgDrawTool
 .text          0x9d007f9c      0x2dc output_pic32_ssd1963\SlideShowDemo.o
                0x9d007f9c                CreateSlideShowDemo
                0x9d008048                SlideShowDemoMsgCallback
                0x9d00816c                InitPixData
 .text          0x9d008278       0xf8 output_pic32_ssd1963\DemoSteps.o
                0x9d008278                InitDemoMode
                0x9d008288                UpdateDemoMode
 .text          0x9d008370      0x168 output_pic32_ssd1963\SideButtons.o
                0x9d008370                SideButtonsMsg
 .text          0x9d0084d8      0xb10 output_pic32_ssd1963\GraphShow.o
                0x9d0084d8                CreateGraphDemo
                0x9d0086a0                InitGraphDemoStyleScheme
                0x9d0086d0                GraphMsgCallback
                0x9d0089c4                SetUpNextDemo
                0x9d008d08                UpdateGraphDemo
                0x9d008da4                xcharStrCopyAppend
                0x9d008df4                AssembleTitleString
 .text          0x9d008fe8     0x11c8 output_pic32_ssd1963\TouchScreen.o
                0x9d008fe8                _T3Interrupt
                0x9d00947c                TouchInit
                0x9d009528                TouchGetX
                0x9d009578                TouchGetY
                0x9d0095cc                TouchGetMsg
                0x9d0096e4                TouchStoreCalibration
                0x9d009744                TouchLoadCalibration
                0x9d009788                TouchCalibration
                0x9d009ea8                TouchGetCalPoints
 .text          0x9d00a1b0      0x184 output_pic32_ssd1963\Beep.o
                0x9d00a1b0                _T2Interrupt
                0x9d00a2a0                BeepInit
 .text          0x9d00a334      0x5fc output_pic32_ssd1963\EEPROM.o
                0x9d00a334                EEPROMInit
                0x9d00a3e8                SPIPut
                0x9d00a420                EEPROMWriteByte
                0x9d00a4d0                EEPROMReadByte
                0x9d00a560                EEPROMWriteWord
                0x9d00a5a8                EEPROMReadWord
                0x9d00a5f4                EEPROMWriteEnable
                0x9d00a640                EEPROMReadStatus
                0x9d00a6b4                EEPROMWriteArray
                0x9d00a864                EEPROMReadArray
 .text          0x9d00a930      0x4f8 output_pic32_ssd1963\Window.o
                0x9d00a930                WndCreate
                0x9d00aa28                WndSetText
                0x9d00aa5c                WndTranslateMsg
                0x9d00ab28                WndDraw
 .text          0x9d00ae28      0x794 output_pic32_ssd1963\Button.o
                0x9d00ae28                BtnCreate
                0x9d00af40                BtnSetText
                0x9d00af88                BtnMsgDefault
                0x9d00b020                BtnTranslateMsg
                0x9d00b220                BtnDraw
 .text          0x9d00b5bc     0x47f0 output_pic32_ssd1963\Chart.o
                0x9d00b5bc                ChCreate
                0x9d00b768                ChTranslateMsg
                0x9d00b7dc                ChGetNextShowData
                0x9d00b814                ChParseShowData
                0x9d00b844                GetLongestNameLength
                0x9d00b8ec                word2xchar
                0x9d00b964                GetColorShade
                0x9d00ba20                ChDraw
                0x9d00f530                ChAddDataSeries
                0x9d00f5e0                ChRemoveDataSeries
                0x9d00f694                ChSetDataSeries
                0x9d00f6ec                ChSetSampleRange
                0x9d00f710                ChSetValueRange
                0x9d00f734                ChSetPercentRange
                0x9d00f758                FillSector
                0x9d00f9a8                GetCirclePoint
                0x9d00fa9c                DrawSector
 .text          0x9d00fdac      0x620 output_pic32_ssd1963\CheckBox.o
                0x9d00fdac                CbCreate
                0x9d00fe9c                CbSetText
                0x9d00fed0                CbMsgDefault
                0x9d00ff5c                CbTranslateMsg
                0x9d010050                CbDraw
 .text          0x9d0103cc     0x2488 output_pic32_ssd1963\DisplayDriver.o
                0x9d0103cc                DelayMs
                0x9d01065c                SetArea
                0x9d0108ac                SetScrollArea
                0x9d010a30                SetScrollStart
                0x9d010b04                EnterSleepMode
                0x9d010b68                ExitSleepMode
                0x9d010bcc                DisplayOff
                0x9d010c30                DisplayOn
                0x9d010c94                EnterDeepSleep
                0x9d010cf8                SetBacklight
                0x9d010e70                SetTearingCfg
                0x9d010f88                ResetDevice
                0x9d011b74                PutPixel
                0x9d011c80                GetPixel
                0x9d011c88                Bar
                0x9d011e20                ClearDevice
                0x9d011f24                PutImage
                0x9d011fe0                PutImage1BPP
                0x9d012200                PutImage4BPP
                0x9d01244c                PutImage8BPP
                0x9d012670                PutImage16BPP
 .text          0x9d012854      0x6c8 output_pic32_ssd1963\EditBox.o
                0x9d012854                EbCreate
                0x9d012960                EbSetText
                0x9d0129a8                EbAddChar
                0x9d0129f4                EbDeleteChar
                0x9d012a20                EbTranslateMsg
                0x9d012ad4                EbMsgDefault
                0x9d012b7c                EbDraw
 .text          0x9d012f1c      0xae4 output_pic32_ssd1963\Grid.o
                0x9d012f1c                GridCreate
                0x9d013058                GridDraw
                0x9d013560                GridFreeItems
                0x9d01359c                GridSetCell
                0x9d01360c                GridClearCellState
                0x9d01365c                GridSetFocus
                0x9d013690                GridSetCellState
                0x9d0136dc                GridGetCell
                0x9d013748                GridMsgDefault
                0x9d013908                GridTranslateMsg
 .text          0x9d013a00      0x578 output_pic32_ssd1963\GroupBox.o
                0x9d013a00                GbCreate
                0x9d013b08                GbTranslateMsg
                0x9d013b9c                GbDraw
 .text          0x9d013f78      0xc74 output_pic32_ssd1963\ListBox.o
                0x9d013f78                LbCreate
                0x9d0140ec                LbAddItem
                0x9d0141d0                LbDelItem
                0x9d014244                LbDelItemsList
                0x9d01428c                LbGetSel
                0x9d0142c4                LbChangeSel
                0x9d014324                LbSetFocusedItem
                0x9d014388                LbGetFocusedItem
                0x9d0143d4                LbTranslateMsg
                0x9d0144b8                LbMsgDefault
                0x9d01467c                LbDraw
 .text          0x9d014bec     0x1250 output_pic32_ssd1963\Meter.o
                0x9d014bec                MtrCreate
                0x9d014d48                MtrCalcDimensions
                0x9d014e8c                MtrSetVal
                0x9d014ed4                MtrMsgDefault
                0x9d014f18                MtrTranslateMsg
                0x9d014f64                MtrDraw
 .text          0x9d015e3c      0x3ec output_pic32_ssd1963\Picture.o
                0x9d015e3c                PictCreate
                0x9d015f1c                PictTranslateMsg
                0x9d015f90                PictDraw
 .text          0x9d016228     0x1528 output_pic32_ssd1963\Primitive.o
                0x9d016228                InitGraph
                0x9d016298                Arc
                0x9d0168f8                Line
                0x9d016c78                Bevel
                0x9d0170a8                FillBevel
                0x9d0172dc                DrawPoly
                0x9d017394                SetFont
                0x9d0173c8                OutText
                0x9d017428                OutTextXY
                0x9d017450                OutChar
                0x9d017660                GetTextWidth
                0x9d0176f0                GetTextHeight
                0x9d017710                GetImageWidth
                0x9d017730                GetImageHeight
 .text          0x9d017750      0x688 output_pic32_ssd1963\RadioButton.o
                0x9d017750                RbCreate
                0x9d017884                RbSetCheck
                0x9d0178cc                RbGetCheck
                0x9d017900                RbSetText
                0x9d017934                RbMsgDefault
                0x9d0179d8                RbTranslateMsg
                0x9d017ac8                RbDraw
 .text          0x9d017dd8      0xecc output_pic32_ssd1963\Slider.o
                0x9d017dd8                SldCreate
                0x9d017edc                SldSetThumbSize
                0x9d017f24                SldGetWidth
                0x9d017fbc                SldGetHeight
                0x9d01804c                SldGetMinMaxPos
                0x9d0180d4                SldSetRange
                0x9d01818c                SldSetPage
                0x9d0181e8                SldSetPos
                0x9d0182e0                SldMsgDefault
                0x9d0184b0                SldTranslateMsg
                0x9d0185e8                SldDraw
 .text          0x9d018ca4      0x4f4 output_pic32_ssd1963\StaticText.o
                0x9d018ca4                StCreate
                0x9d018d94                StSetText
                0x9d018dc8                StTranslateMsg
                0x9d018e3c                StDraw
 .text          0x9d019198      0xd2c output_pic32_ssd1963\GOL.o
                0x9d019198                GOLGetFocusPrev
                0x9d01922c                GOLGetFocusNext
                0x9d019280                GOLSetFocus
                0x9d0192e4                GOLCanBeFocused
                0x9d019338                GOLCreateScheme
                0x9d0193b4                GOLInit
                0x9d0193dc                GOLFree
                0x9d019480                GOLDeleteObject
                0x9d019540                GOLDeleteObjectByID
                0x9d019574                GOLFindObject
                0x9d0195a4                GOLAddObject
                0x9d0195e0                GOLDraw
                0x9d01975c                GOLRedrawRec
                0x9d019834                GOLMsg
                0x9d019ba4                GOLPanelDrawTsk
 .text          0x9d019ec4       0xa8 C:/Program Files/Microchip/mplabc32/v1.12/bin/../lib/gcc/pic32mx/3.4.4/../../../../pic32mx/lib/size\libc.a(memset.o)
                0x9d019ec4                memset
 .text.general_exception
                0x9d019f6c       0xd0 C:/Program Files/Microchip/mplabc32/v1.12/bin/../lib/gcc/pic32mx/3.4.4/../../../../pic32mx/lib/size\libc.a(general-exception.o)
                0x9d019f6c                _general_exception_context
 .text.malloc   0x9d01a03c      0x234 C:/Program Files/Microchip/mplabc32/v1.12/bin/../lib/gcc/pic32mx/3.4.4/../../../../pic32mx/lib/size\libc.a(malloc.o)
                0x9d01a03c                malloc
 .text.free     0x9d01a270       0x18 C:/Program Files/Microchip/mplabc32/v1.12/bin/../lib/gcc/pic32mx/3.4.4/../../../../pic32mx/lib/size\libc.a(malloc.o)
                0x9d01a270                free
 .text.srand    0x9d01a288       0x10 C:/Program Files/Microchip/mplabc32/v1.12/bin/../lib/gcc/pic32mx/3.4.4/../../../../pic32mx/lib/size\libc.a(rand.o)
                0x9d01a288                srand
 .text.rand     0x9d01a298       0x44 C:/Program Files/Microchip/mplabc32/v1.12/bin/../lib/gcc/pic32mx/3.4.4/../../../../pic32mx/lib/size\libc.a(rand.o)
                0x9d01a298                rand
 .text._stub_sbd_memlayout
                0x9d01a2dc       0x2c C:/Program Files/Microchip/mplabc32/v1.12/bin/../lib/gcc/pic32mx/3.4.4/../../../../pic32mx/lib/size\libc.a(sbrk.o)
                0x9d01a2dc                _sbd_memlayout
                0x9d01a2dc                _stub_sbd_memlayout
 .text._sbrk_init
                0x9d01a308      0x148 C:/Program Files/Microchip/mplabc32/v1.12/bin/../lib/gcc/pic32mx/3.4.4/../../../../pic32mx/lib/size\libc.a(sbrk.o)
                0x9d01a308                _sbrk_init
 .text._sbrk    0x9d01a450       0xa4 C:/Program Files/Microchip/mplabc32/v1.12/bin/../lib/gcc/pic32mx/3.4.4/../../../../pic32mx/lib/size\libc.a(sbrk.o)
                0x9d01a450                _sbrk
 .text.sbrk     0x9d01a4f4       0x5c C:/Program Files/Microchip/mplabc32/v1.12/bin/../lib/gcc/pic32mx/3.4.4/../../../../pic32mx/lib/size\libc.a(sbrk.o)
                0x9d01a4f4                sbrk
 .text._general_exception_handler
                0x9d01a550        0x8 C:/Program Files/Microchip/mplabc32/v1.12/bin/../lib/gcc/pic32mx/3.4.4/../../../../pic32mx/lib/size\libc.a(default-general-exception-handler.o)
                0x9d01a550                _general_exception_handler
 .text._bootstrap_exception_handler
                0x9d01a558        0x8 C:/Program Files/Microchip/mplabc32/v1.12/bin/../lib/gcc/pic32mx/3.4.4/../../../../pic32mx/lib/size\libc.a(default-bootstrap-exception-handler.o)
                0x9d01a558                _bootstrap_exception_handler
 .text._on_reset
                0x9d01a560        0x8 C:/Program Files/Microchip/mplabc32/v1.12/bin/../lib/gcc/pic32mx/3.4.4/../../../../pic32mx/lib/size\libc.a(default-on-reset.o)
                0x9d01a560                _on_reset
 .text._on_bootstrap
                0x9d01a568        0x8 C:/Program Files/Microchip/mplabc32/v1.12/bin/../lib/gcc/pic32mx/3.4.4/../../../../pic32mx/lib/size\libc.a(default-on-bootstrap.o)
                0x9d01a568                _on_bootstrap
 .text          0x9d01a570       0x18 C:/Program Files/Microchip/mplabc32/v1.12/bin/../lib/gcc/pic32mx/3.4.4/../../../../pic32mx/lib/size\libc.a(default-nmi-handler.o)
                0x9d01a570                _nmi_handler
 .text          0x9d01a588      0x8ec C:/Program Files/Microchip/mplabc32/v1.12/bin/../lib/gcc/pic32mx/3.4.4/../../../../pic32mx/lib/size\libm.a(fp32.o)
                0x9d01a588                fpsub
                0x9d01a588                __subsf3
                0x9d01a590                __addsf3
                0x9d01a590                fpadd
                0x9d01a7fc                __mulsf3
                0x9d01a7fc                fpmul
                0x9d01a9b4                fpdiv
                0x9d01a9b4                __divsf3
                0x9d01abe0                sitofp
                0x9d01abe0                litofp
                0x9d01abe0                __floatsisf
                0x9d01ac3c                ultofp
                0x9d01ac3c                uitofp
                0x9d01ac88                fptosi
                0x9d01ac88                fptoli
                0x9d01ac88                __fixsfsi
                0x9d01ad00                fptoui
                0x9d01ad00                __fixunssfsi
                0x9d01ad00                fptoul
                0x9d01ad74                __nesf2
                0x9d01ad74                fpcmp
                0x9d01ad74                __eqsf2
                0x9d01ad74                __gesf2
                0x9d01ad74                __ltsf2
                0x9d01ad74                __gtsf2
                0x9d01ad74                __lesf2
                0x9d01ae08                fpfabs
                0x9d01ae08                fabsf
                0x9d01ae18                __negsf2
                0x9d01ae28                fpnan
                0x9d01ae28                nanf
 .text          0x9d01ae74      0x114 C:/Program Files/Microchip/mplabc32/v1.12/bin/../lib/gcc/pic32mx/3.4.4/../../../../pic32mx/lib/size\libm.a(fpcos32.o)
                0x9d01ae74                cosf
                0x9d01ae74                fpcos
 .text          0x9d01af88      0x118 C:/Program Files/Microchip/mplabc32/v1.12/bin/../lib/gcc/pic32mx/3.4.4/../../../../pic32mx/lib/size\libm.a(fpsin32.o)
                0x9d01af88                sinf
                0x9d01af88                fpsin
 .text          0x9d01b0a0      0x108 C:/Program Files/Microchip/mplabc32/v1.12/bin/../lib/gcc/pic32mx/3.4.4/../../../../pic32mx/lib/size\libm.a(fpreduct32.o)
                0x9d01b0a0                fpreduct
 .text.OpenCoreTimer
                0x9d01b1a8        0xc C:/Program Files/Microchip/mplabc32/v1.12/bin/../lib/gcc/pic32mx/3.4.4/../../../../pic32mx/lib/size\libmchp_peripheral.a(open_core_timer_lib.o)
                0x9d01b1a8                OpenCoreTimer
 .text.CheKseg0CacheOn
                0x9d01b1b4       0x18 C:/Program Files/Microchip/mplabc32/v1.12/bin/../lib/gcc/pic32mx/3.4.4/../../../../pic32mx/lib/size\libmchp_peripheral_32MX360F512L.a(pcache.o)
                0x9d01b1b4                CheKseg0CacheOn
 .text.INTDisableInterrupts
                0x9d01b1cc        0x8 C:/Program Files/Microchip/mplabc32/v1.12/bin/../lib/gcc/pic32mx/3.4.4/../../../../pic32mx/lib/size\libmchp_peripheral_32MX360F512L.a(int_disable_interrupts_lib.o)
                0x9d01b1cc                INTDisableInterrupts
 .text.INTRestoreInterrupts
                0x9d01b1d4       0x1c C:/Program Files/Microchip/mplabc32/v1.12/bin/../lib/gcc/pic32mx/3.4.4/../../../../pic32mx/lib/size\libmchp_peripheral_32MX360F512L.a(int_restore_interrupts_lib.o)
                0x9d01b1d4                INTRestoreInterrupts
 .text.INTEnableSystemMultiVectoredInt
                0x9d01b1f0       0x34 C:/Program Files/Microchip/mplabc32/v1.12/bin/../lib/gcc/pic32mx/3.4.4/../../../../pic32mx/lib/size\libmchp_peripheral_32MX360F512L.a(int_enable_mv_int_lib.o)
                0x9d01b1f0                INTEnableSystemMultiVectoredInt
 .text.RtccInit
                0x9d01b224      0x180 C:/Program Files/Microchip/mplabc32/v1.12/bin/../lib/gcc/pic32mx/3.4.4/../../../../pic32mx/lib/size\libmchp_peripheral_32MX360F512L.a(rtcc_init_lib.o)
                0x9d01b224                RtccInit
 .text.RtccSetDate
                0x9d01b3a4       0x24 C:/Program Files/Microchip/mplabc32/v1.12/bin/../lib/gcc/pic32mx/3.4.4/../../../../pic32mx/lib/size\libmchp_peripheral_32MX360F512L.a(rtcc_set_date_lib.o)
                0x9d01b3a4                RtccSetDate
 .text.RtccSetTime
                0x9d01b3c8       0x24 C:/Program Files/Microchip/mplabc32/v1.12/bin/../lib/gcc/pic32mx/3.4.4/../../../../pic32mx/lib/size\libmchp_peripheral_32MX360F512L.a(rtcc_set_time_lib.o)
                0x9d01b3c8                RtccSetTime
 .text.INTEnableInterrupts
                0x9d01b3ec        0x8 C:/Program Files/Microchip/mplabc32/v1.12/bin/../lib/gcc/pic32mx/3.4.4/../../../../pic32mx/lib/size\libmchp_peripheral_32MX360F512L.a(int_enable_interrupts_lib.o)
                0x9d01b3ec                INTEnableInterrupts
 .text.INTClearFlag
                0x9d01b3f4       0x28 C:/Program Files/Microchip/mplabc32/v1.12/bin/../lib/gcc/pic32mx/3.4.4/../../../../pic32mx/lib/size\libmchp_peripheral_32MX360F512L.a(int_tbl_lib.o)
                0x9d01b3f4                INTClearFlag
 .text.INTEnable
                0x9d01b41c       0x38 C:/Program Files/Microchip/mplabc32/v1.12/bin/../lib/gcc/pic32mx/3.4.4/../../../../pic32mx/lib/size\libmchp_peripheral_32MX360F512L.a(int_tbl_lib.o)
                0x9d01b41c                INTEnable
 .text._RtccSetTimeAndDate
                0x9d01b454      0x210 C:/Program Files/Microchip/mplabc32/v1.12/bin/../lib/gcc/pic32mx/3.4.4/../../../../pic32mx/lib/size\libmchp_peripheral_32MX360F512L.a(_rtcc_set_time_and_date_lib.o)
                0x9d01b454                _RtccSetTimeAndDate
 .text._RtccWaitClockOff
                0x9d01b664       0xe8 C:/Program Files/Microchip/mplabc32/v1.12/bin/../lib/gcc/pic32mx/3.4.4/../../../../pic32mx/lib/size\libmchp_peripheral_32MX360F512L.a(_rtcc_wait_clock_off_lib.o)
                0x9d01b664                _RtccWaitClockOff
 .text.ReadCoreTimer
                0x9d01b74c        0x8 C:/Program Files/Microchip/mplabc32/v1.12/bin/../lib/gcc/pic32mx/3.4.4/../../../../pic32mx/lib/size\libmchp_peripheral_32MX360F512L.a(read_core_timer_lib.o)
                0x9d01b74c                ReadCoreTimer
 *(.text.*personality*)
 *(.gnu.warning)
 *(.mips16.fn.*)
 *(.mips16.call.*)
                0x9d01b754                _text_end = .

.rodata         0x9d01b754    0x43620
 *(.rodata .rodata.* .gnu.linkonce.r.*)
 .rodata        0x9d01b754      0x2e0 output_pic32_ssd1963\MainDemo.o
                0x9d01b754                NewGameStr
                0x9d01b75c                ExitStr
                0x9d01b768                ScaleStr
                0x9d01b774                SetStr
                0x9d01b77c                LeftArrowStr
                0x9d01b780                RightArrowStr
                0x9d01b784                UpArrowStr
                0x9d01b788                DownArrowStr
                0x9d01b78c                MeterStr
                0x9d01b794                ExtStr
                0x9d01b79c                EcgStr
                0x9d01b7a4                LabelStr
                0x9d01b7b0                NoiseStr
                0x9d01b7bc                CleanStr
                0x9d01b7c8                RateStr
                0x9d01b7e0                AmplitudeStr
                0x9d01b7f4                mVStr
                0x9d01b7fc                BeatsStr
                0x9d01b808                ClearStr
                0x9d01b814                DemoStr
                0x9d01b820                ErrMsgStandard
                0x9d01b834                ErrNotSupported
                0x9d01b854                ErrMsgFailedStr
                0x9d01b864                ErrMsgHUBAttachedStr
                0x9d01b86c                ErrMsgUDAttachedStr
                0x9d01b87c                ErrMsgEnumerationStr
                0x9d01b894                ErrMsgClientInitStr
                0x9d01b8c0                ErrMsgOutofMemoryStr
                0x9d01b8dc                ErrMsgUnpecifiedErrStr
                0x9d01b8f4                MsgTouchToProceedStr
                0x9d01b918                MsgTouchToCalibrateStr
 .rodata        0x9d01ba34       0x80 output_pic32_ssd1963\rtcc.o
 .rodata        0x9d01bab4     0x2538 output_pic32_ssd1963\Fonts.o
                0x9d01bab4                GOLSmallFont
                0x9d01babc                L22900
                0x9d01c370                GOLMediumFont
                0x9d01c378                L24301
                0x9d01cdfc                BigFonts
                0x9d01ce04                L29288
 .rodata        0x9d01dfec       0xbc output_pic32_ssd1963\DemoSelection.o
                0x9d01dfec                iconLightingStr
                0x9d01e000                iconLanguageStr
                0x9d01e014                iconGameStr
                0x9d01e020                iconAnimationStr
                0x9d01e034                iconDrawingStr
                0x9d01e044                iconECGStr
                0x9d01e04c                iconDateTimeStr
                0x9d01e058                iconPixFolderStr
                0x9d01e078                iconPix2FolderStr
                0x9d01e090                iconPix3FolderStr
 .rodata        0x9d01e0a8     0x2090 output_pic32_ssd1963\AnimationBitmaps.o
                0x9d01e0a8                Engine4
                0x9d01e0b0                L30198
                0x9d01e8cc                Engine3
                0x9d01e8d4                L22053
                0x9d01f0f0                Engine2
                0x9d01f0f8                L23187
                0x9d01f914                Engine1
                0x9d01f91c                L28742
 .rodata        0x9d020138       0xc0 output_pic32_ssd1963\ECG.o
                0x9d020138                ecgPoints
 .rodata        0x9d0201f8       0x88 output_pic32_ssd1963\Games.o
                0x9d0201f8                CrashedStr
                0x9d020214                ShuFullStr
                0x9d020240                InAKnotStr
 .rodata        0x9d020280      0xd70 output_pic32_ssd1963\SnakeBitmaps.o
                0x9d020280                body
                0x9d020288                L13935
                0x9d020710                head
                0x9d020718                L16164
                0x9d020ba0                food
                0x9d020ba8                L27882
 .rodata        0x9d020ff0      0x4c0 output_pic32_ssd1963\ECGBitmaps.o
                0x9d020ff0                eheart
                0x9d020ff8                L16936
                0x9d021250                eheart2
                0x9d021258                L30781
 .rodata        0x9d0214b0       0x74 output_pic32_ssd1963\RGBDemo.o
                0x9d0214b0                HIDHardwareMsgStr
                0x9d0214dc                NoHIDHardwareMsgStr
 .rodata        0x9d021524       0xac output_pic32_ssd1963\MultiFontsDemo.o
                0x9d021524                EnglishStr
                0x9d021540                FrenchStr
                0x9d021560                GermanStr
                0x9d021578                ItalianStr
                0x9d021590                DutchStr
 .rodata        0x9d0215d0      0x144 output_pic32_ssd1963\TimeDateDemo.o
                0x9d0215d0                Monday
                0x9d0215e0                Tuesday
                0x9d0215f0                Wednesday
                0x9d021604                Thursday
                0x9d021618                Friday
                0x9d02162c                Saturday
                0x9d021640                Sunday
                0x9d021650                January
                0x9d021664                February
                0x9d021678                March
                0x9d021684                April
                0x9d021690                May
                0x9d021698                June
                0x9d0216a4                July
                0x9d0216b0                August
                0x9d0216c0                September
                0x9d0216d4                October
                0x9d0216e4                November
                0x9d0216f8                December
 .rodata        0x9d021714       0x18 output_pic32_ssd1963\DrawTool.o
 .rodata        0x9d02172c      0x750 output_pic32_ssd1963\DemoSteps.o
                0x9d02172c                DemoPoints
 .rodata        0x9d021e7c      0x110 output_pic32_ssd1963\GraphShow.o
                0x9d021e7c                demoTypeList
                0x9d021ebc                BarStr
                0x9d021ec4                PieStr
                0x9d021ecc                ThreeDStr
                0x9d021ed4                LegendStr
                0x9d021ee4                ValueStr
                0x9d021ef0                DonutStr
                0x9d021efc                PercentStr
                0x9d021f00                ParenOpenStr
                0x9d021f04                ParenCloseStr
                0x9d021f08                CommaStr
                0x9d021f0c                SpaceStr
                0x9d021f10                SingleStr
                0x9d021f20                MultiStr
                0x9d021f2c                Var1Name
                0x9d021f38                Var2Name
                0x9d021f44                Var3Name
                0x9d021f50                Var4Name
                0x9d021f5c                Var5Name
                0x9d021f68                XName
                0x9d021f7c                YName
 .rodata        0x9d021f8c      0x228 output_pic32_ssd1963\TouchScreen.o
 .rodata        0x9d0221b4       0x1c output_pic32_ssd1963\Window.o
 .rodata        0x9d0221d0       0x18 output_pic32_ssd1963\Button.o
 .rodata        0x9d0221e8      0x1b4 output_pic32_ssd1963\Chart.o
                0x9d0221e8                ChartVarClr
                0x9d0222c4                sinTable
                0x9d022320                cosTable
 .rodata        0x9d02239c       0x1c output_pic32_ssd1963\CheckBox.o
 .rodata        0x9d0223b8       0x14 output_pic32_ssd1963\Grid.o
 .rodata        0x9d0223cc       0x38 output_pic32_ssd1963\GroupBox.o
 .rodata        0x9d022404       0x18 output_pic32_ssd1963\ListBox.o
 .rodata        0x9d02241c       0x9c output_pic32_ssd1963\Meter.o
                0x9d02241c                _sineTable
 .rodata.cst4   0x9d0224b8        0xc output_pic32_ssd1963\Meter.o
 .rodata        0x9d0224c4       0x1c output_pic32_ssd1963\Picture.o
 .rodata        0x9d0224e0       0x20 output_pic32_ssd1963\RadioButton.o
 .rodata        0x9d022500       0x28 output_pic32_ssd1963\Slider.o
 .rodata        0x9d022528       0x14 output_pic32_ssd1963\StaticText.o
 .rodata        0x9d02253c     0x1588 output_pic32_ssd1963\GOLFontDefault.o
                0x9d02253c                GOLFontDefault
                0x9d022544                L11903
 .rodata        0x9d023ac4       0x80 output_pic32_ssd1963\GOL.o
 .rodata        0x9d023b44     0xf500 output_pic32_ssd1963\IconsC32.o
                0x9d023b44                L4655
                0x9d02458c                L13843
                0x9d024fd4                L24657
                0x9d025a1c                L25738
                0x9d026464                L16628
                0x9d02706c                L23206
                0x9d0270f8                L555
                0x9d027b40                L27004
                0x9d028588                L9950
                0x9d02c974                L11754
                0x9d02d3bc                L20382
                0x9d02de04                L10406
                0x9d02e84c                L31503
                0x9d02f294                L25476
                0x9d02fcdc                L25223
                0x9d030724                L30216
                0x9d03116c                L7388
                0x9d031bb4                L2953
                0x9d0325fc                L16506
 .rodata        0x9d033044    0x2ba30 output_pic32_ssd1963\SlideShowC32.o
                0x9d033044                L8342
                0x9d03db0c                L8219
                0x9d052c94                L29143
 .rodata.__IntSrcTbl
                0x9d05ea74      0x300 C:/Program Files/Microchip/mplabc32/v1.12/bin/../lib/gcc/pic32mx/3.4.4/../../../../pic32mx/lib/size\libmchp_peripheral_32MX360F512L.a(int_tbl_lib.o)
                0x9d05ea74                __IntSrcTbl
 *(.rodata1)
                0x9d05ed74                . = ALIGN (0x4)

.sdata2         0x9d05ed74        0x0
 *(.sdata2 .sdata2.* .gnu.linkonce.s2.*)
                0x9d05ed74                . = ALIGN (0x4)

.sbss2          0x9d05ed74        0x0
 *(.sbss2 .sbss2.* .gnu.linkonce.sb2.*)
                0x9d05ed74                . = ALIGN (0x4)

.eh_frame_hdr
 *(.eh_frame_hdr)

.eh_frame
 *(.eh_frame)

.dbg_data       0xa0000000        0x0
                0xa0000000                . = (. + DEFINED (_DEBUGGER)?0x200:0x0)

.persist        0xa0000000        0x0
                0xa0000000                _persist_begin = .
 *(.persist .persist.*)
                0xa0000000                _persist_end = .

.data           0xa0000000      0x1a8 load address 0x9d05ed74
                0xa0000000                _data_begin = .
 *(.data .data.* .gnu.linkonce.d.*)
 .data          0xa0000000       0x20 output_pic32_ssd1963\rtcc.o
                0xa0000000                _time_str
                0xa0000010                _date_str
 .data          0xa0000020       0x28 output_pic32_ssd1963\Games.o
                0xa0000020                scoreText
 .data          0xa0000048        0xc output_pic32_ssd1963\RGBDemo.o
                0xa0000048                FadeStr
 .data          0xa0000054       0x50 output_pic32_ssd1963\TimeDateDemo.o
                0xa0000054                MoItems
                0xa0000088                WkDayItems
 .data          0xa00000a4       0xc0 output_pic32_ssd1963\GraphShow.o
                0xa00000a4                samples1
                0xa00000c4                samples2
                0xa00000e4                samples3
                0xa0000104                samples4
                0xa0000124                samples5
                0xa0000144                MyColorTable
 .data          0xa0000164       0x18 output_pic32_ssd1963\Chart.o
 .data          0xa000017c       0x24 C:/Program Files/Microchip/mplabc32/v1.12/bin/../lib/gcc/pic32mx/3.4.4/../../../../pic32mx/lib/size\libm.a(sincof32.o)
                0xa000017c                _sincof
                0xa000018c                _coscof
 .data._RtccWaitClkSteps
                0xa00001a0        0x4 C:/Program Files/Microchip/mplabc32/v1.12/bin/../lib/gcc/pic32mx/3.4.4/../../../../pic32mx/lib/size\libmchp_peripheral_32MX360F512L.a(_rtcc_wait_clock_off_lib.o)
                0xa00001a0                _RtccWaitClkSteps
 .data._RtccWaitClkStepSz
                0xa00001a4        0x4 C:/Program Files/Microchip/mplabc32/v1.12/bin/../lib/gcc/pic32mx/3.4.4/../../../../pic32mx/lib/size\libmchp_peripheral_32MX360F512L.a(_rtcc_wait_clock_off_lib.o)
                0xa00001a4                _RtccWaitClkStepSz
 *(.gnu.linkonce.d.*personality*)
 *(.data1)
                0x9d05ed74                _data_image_begin = LOADADDR (.data)

.eh_frame
 *(.eh_frame)
                0xa00001a8                . = .
                0xa00081a0                _gp = (ALIGN (0x10) + 0x7ff0)

.got
 *(.got.plt)
 *(.got)

.sdata          0xa00001a8      0x15c load address 0x9d05ef1c
                0xa00001a8                _sdata_begin = .
 *(.sdata .sdata.* .gnu.linkonce.s.*)
 .sdata         0xa00001a8        0xc output_pic32_ssd1963\Animation.o
                0xa00001a8                animate
 .sdata         0xa00001b4        0xc output_pic32_ssd1963\ECG.o
                0xa00001b4                heartStates
                0xa00001b6                noise
                0xa00001b7                label
 .sdata         0xa00001c0       0x30 output_pic32_ssd1963\RGBDemo.o
                0xa00001c0                OneStr
                0xa00001c4                TwoStr
                0xa00001c8                cptrState
                0xa00001cc                Pres1Red
                0xa00001cd                Pres1Green
                0xa00001ce                Pres1Blue
                0xa00001cf                Pres2Red
                0xa00001d0                Pres2Green
                0xa00001d1                Pres2Blue
                0xa00001d2                RedRange
                0xa00001d4                RedPage
                0xa00001d6                RedPos
                0xa00001d8                GreenRange
                0xa00001da                GreenPage
                0xa00001dc                GreenPos
                0xa00001de                BlueRange
                0xa00001e0                BluePage
                0xa00001e2                BluePos
                0xa00001e4                Intensity
                0xa00001e8                TickDiff
                0xa00001ec                PtrTickDiff
 .sdata         0xa00001f0        0xc output_pic32_ssd1963\MultiFontsDemo.o
                0xa00001f0                helloDelay
 .sdata         0xa00001fc       0x24 output_pic32_ssd1963\TimeDateDemo.o
 .sdata         0xa0000220        0x6 output_pic32_ssd1963\DrawTool.o
                0xa0000220                drawColor
 .sdata         0xa0000226        0x4 output_pic32_ssd1963\SideButtons.o
 .sdata         0xa000022a       0x10 output_pic32_ssd1963\TouchScreen.o
                0xa000022a                _calXMin
                0xa000022c                _calXMax
                0xa000022e                _calYMin
                0xa0000230                _calYMax
                0xa0000232                adcX
                0xa0000234                adcY
 *fill*         0xa000023a        0x2 00
 .sdata         0xa000023c        0x8 output_pic32_ssd1963\Chart.o
 .sdata         0xa0000244        0x4 output_pic32_ssd1963\Meter.o
 .sdata         0xa0000248       0x98 output_pic32_ssd1963\IconsC32.o
                0xa0000248                RGBLighting_4bpp_72x72
                0xa0000250                RGBLighting_mono_72x72
                0xa0000258                PCGaming2_mono_72x72
                0xa0000260                PCGaming2_4bpp_72x72
                0xa0000268                mchpLogo
                0xa0000270                mchpIcon0
                0xa0000278                Language_mono_72x72
                0xa0000280                Language_4bpp_72x72
                0xa0000288                intro
                0xa0000290                FolderPhoto_mono_72x72
                0xa0000298                FolderPhoto_4bpp_72x72
                0xa00002a0                ECG_mono_72x72
                0xa00002a8                ECG_4bpp_72x72
                0xa00002b0                DrawingScreen_mono_72x72
                0xa00002b8                DrawingScreen_4bpp_72x72
                0xa00002c0                DateAndTime_mono_72x72
                0xa00002c8                DateAndTime_4bpp_72x72
                0xa00002d0                Animation_mono_72x72
                0xa00002d8                Animation_4bpp_72x72
 .sdata         0xa00002e0       0x18 output_pic32_ssd1963\SlideShowC32.o
                0xa00002e0                rose
                0xa00002e8                sunset2
                0xa00002f0                vegas
 .sdata._maxbrk
                0xa00002f8        0x4 C:/Program Files/Microchip/mplabc32/v1.12/bin/../lib/gcc/pic32mx/3.4.4/../../../../pic32mx/lib/size\libc.a(sbrk.o)
                0xa00002f8                _maxbrk
 .sdata._minbrk
                0xa00002fc        0x4 C:/Program Files/Microchip/mplabc32/v1.12/bin/../lib/gcc/pic32mx/3.4.4/../../../../pic32mx/lib/size\libc.a(sbrk.o)
                0xa00002fc                _minbrk
 .sdata.curbrk  0xa0000300        0x4 C:/Program Files/Microchip/mplabc32/v1.12/bin/../lib/gcc/pic32mx/3.4.4/../../../../pic32mx/lib/size\libc.a(sbrk.o)
                0xa0000304                _sdata_end = .

.lit8
 *(.lit8)

.lit4
 *(.lit4)
                0xa0000304                . = ALIGN (0x4)
                0xa0000304                _data_end = .
                0xa0000304                _bss_begin = .

.sbss           0xa0000304      0x336 load address 0x9d05f078
                0xa0000304                _sbss_begin = .
 *(.dynsbss)
 *(.sbss .sbss.* .gnu.linkonce.sb.*)
 .sbss          0xa0000304       0x10 output_pic32_ssd1963\MainDemo.o
                0xa0000304                StaticTextLstStr
                0xa0000308                screenState
                0xa000030c                tick
 .sbss          0xa0000314        0x2 output_pic32_ssd1963\DemoSelection.o
                0xa0000314                page
 *fill*         0xa0000316        0x2 00
 .sbss          0xa0000318        0x8 output_pic32_ssd1963\Animation.o
 .sbss          0xa0000320       0x1c output_pic32_ssd1963\ECG.o
                0xa0000320                ecgStates
                0xa0000324                potInput
 .sbss          0xa000033c        0x8 output_pic32_ssd1963\Games.o
 .sbss          0xa0000344       0x2c output_pic32_ssd1963\RGBDemo.o
                0xa0000344                rgbState
 .sbss          0xa0000370        0xc output_pic32_ssd1963\MultiFontsDemo.o
                0xa0000370                update
 .sbss          0xa000037c        0xc output_pic32_ssd1963\TimeDateDemo.o
 .sbss          0xa0000388        0x4 output_pic32_ssd1963\GraphShow.o
 .sbss          0xa000038c        0xc output_pic32_ssd1963\TouchScreen.o
                0xa000038c                adcPot
                0xa0000390                state
 .sbss          0xa0000398        0x4 output_pic32_ssd1963\Window.o
 .sbss          0xa000039c        0xc output_pic32_ssd1963\Button.o
 .sbss          0xa00003a8       0x74 output_pic32_ssd1963\Chart.o
 .sbss          0xa000041c        0x4 output_pic32_ssd1963\CheckBox.o
 .sbss          0xa0000420        0x1 output_pic32_ssd1963\DisplayDriver.o
                0xa0000420                _gpioStatus
 *fill*         0xa0000421        0x3 00
 .sbss          0xa0000424        0x8 output_pic32_ssd1963\EditBox.o
 .sbss          0xa000042c        0xc output_pic32_ssd1963\GroupBox.o
 .sbss          0xa0000438        0xc output_pic32_ssd1963\ListBox.o
 .sbss          0xa0000444       0x20 output_pic32_ssd1963\Meter.o
 .sbss          0xa0000464        0xc output_pic32_ssd1963\Picture.o
 .sbss          0xa0000470       0x14 output_pic32_ssd1963\RadioButton.o
                0xa0000470                _pListButtons
 .sbss          0xa0000484       0x1c output_pic32_ssd1963\Slider.o
 .sbss          0xa00004a0        0xc output_pic32_ssd1963\StaticText.o
 .sbss          0xa00004ac       0x14 output_pic32_ssd1963\GOL.o
                0xa00004ac                _pGolObjects
                0xa00004b0                _pDefaultGolScheme
                0xa00004b4                _pObjectFocused
                0xa00004bc                _pRpnlBitmap
 .sbss.allocp   0xa00004c0        0x4 C:/Program Files/Microchip/mplabc32/v1.12/bin/../lib/gcc/pic32mx/3.4.4/../../../../pic32mx/lib/size\libc.a(malloc.o)
 .sbss.alloct   0xa00004c4        0x4 C:/Program Files/Microchip/mplabc32/v1.12/bin/../lib/gcc/pic32mx/3.4.4/../../../../pic32mx/lib/size\libc.a(malloc.o)
 .sbss.allocx   0xa00004c8        0x8 C:/Program Files/Microchip/mplabc32/v1.12/bin/../lib/gcc/pic32mx/3.4.4/../../../../pic32mx/lib/size\libc.a(malloc.o)
 .sbss.randx    0xa00004d0        0x4 C:/Program Files/Microchip/mplabc32/v1.12/bin/../lib/gcc/pic32mx/3.4.4/../../../../pic32mx/lib/size\libc.a(rand.o)
 .sbss.randf    0xa00004d4        0x1 C:/Program Files/Microchip/mplabc32/v1.12/bin/../lib/gcc/pic32mx/3.4.4/../../../../pic32mx/lib/size\libc.a(rand.o)
 *fill*         0xa00004d5        0x3 00
 .sbss.errno    0xa00004d8        0x4 C:/Program Files/Microchip/mplabc32/v1.12/bin/../lib/gcc/pic32mx/3.4.4/../../../../pic32mx/lib/size\libc.a(errno.o)
                0xa00004d8                errno
 *(.scommon)
 .scommon       0xa00004dc       0x28 output_pic32_ssd1963\MainDemo.o
                0xa00004dc                iconScheme
                0xa00004e0                navScheme
                0xa00004e4                usbErrorCode
                0xa00004e8                altScheme
                0xa00004ec                pNavList
                0xa00004f0                vs1003TestWord
                0xa00004f4                graphScheme
                0xa00004f8                usbHIDStatus
                0xa00004f9                usbMSDStatus
                0xa00004fc                meterScheme
                0xa0000500                gridScheme
 .scommon       0xa0000504        0x1 output_pic32_ssd1963\rtcc.o
                0xa0000504                _rtcc_flag
 *fill*         0xa0000505        0x3 00
 .scommon       0xa0000508        0x8 output_pic32_ssd1963\DemoSelection.o
                0xa0000508                sdCardStatus
                0xa000050c                demoTick
 .scommon       0xa0000510        0x8 output_pic32_ssd1963\Animation.o
                0xa0000510                pPicture
                0xa0000514                pMeter
 .scommon       0xa0000518       0x10 output_pic32_ssd1963\ECG.o
                0xa0000518                ecgVerX2
                0xa000051a                ecgVerY1
                0xa000051c                ecgHorY1
                0xa000051e                ecgHorX1
                0xa0000520                ecgHorX2
                0xa0000522                ecgVerX1
                0xa0000524                ecgVerY2
                0xa0000526                ecgHorY2
 .scommon       0xa0000528       0x18 output_pic32_ssd1963\Games.o
                0xa0000528                pScore
                0xa000052c                score
                0xa0000530                gamesGrid
                0xa0000534                pScoreText
                0xa0000538                defaultDirection
                0xa000053c                pScoreInfo
 .scommon       0xa0000540       0x3c output_pic32_ssd1963\RGBDemo.o
                0xa0000540                deltaR
                0xa0000544                LabelColorScheme
                0xa0000548                RedLim
                0xa0000549                RedMin
                0xa000054a                RedMax
                0xa000054b                deltaB
                0xa000054c                FadeDirGreen
                0xa000054d                FadeModeEnable
                0xa0000550                RGBBlueScheme
                0xa0000554                GreenMax
                0xa0000558                ControlColorScheme
                0xa000055c                FadeDirRed
                0xa000055d                deltaG
                0xa000055e                UpdateCurrent
                0xa000055f                BlueMax
                0xa0000560                UpdateColor
                0xa0000564                Preset1ColorScheme
                0xa0000568                RGBGreenScheme
                0xa000056c                RGBRedScheme
                0xa0000570                GreenMin
                0xa0000571                FadeDirBlue
                0xa0000572                GreenLim
                0xa0000573                BlueLim
                0xa0000574                updateIntensity
                0xa0000575                BlueMin
                0xa0000578                Preset2ColorScheme
 .scommon       0xa000057c        0x8 output_pic32_ssd1963\MultiFontsDemo.o
                0xa000057c                pHWData
                0xa0000580                FontScheme2
 .scommon       0xa0000584       0x24 output_pic32_ssd1963\TimeDateDemo.o
                0xa0000584                MoScheme
                0xa0000588                pMonth
                0xa000058c                pWkDay
                0xa0000590                dumScheme
                0xa0000594                MinScheme
                0xa0000598                SecScheme
                0xa000059c                DayScheme
                0xa00005a0                HourScheme
                0xa00005a4                WkDayScheme
 .scommon       0xa00005a8        0x8 output_pic32_ssd1963\SlideShowDemo.o
                0xa00005a8                pPixData
                0xa00005ac                SlideShowScheme
 .scommon       0xa00005b0        0xc output_pic32_ssd1963\DemoSteps.o
                0xa00005b0                gEnableDemoFlag
                0xa00005b4                demoCount
                0xa00005b8                prevDemoTime
 .scommon       0xa00005bc        0x6 output_pic32_ssd1963\GraphShow.o
                0xa00005bc                chartType
                0xa00005c0                dTypeCnt
 *fill*         0xa00005c2        0x2 00
 .scommon       0xa00005c4       0x1c output_pic32_ssd1963\FSIO.o
                0xa00005c4                gFileSlotOpen
                0xa00005c7                gTimeCrtMS
                0xa00005c8                gTimeCrtTime
                0xa00005cc                FatRootDirClusterValue
                0xa00005d0                gTimeWrtDate
                0xa00005d2                gTimeCrtDate
                0xa00005d4                TempClusterCalc
                0xa00005d8                dirCleared
                0xa00005da                gTimeAccDate
                0xa00005dc                FSerrno
                0xa00005de                gTimeWrtTime
 .scommon       0xa00005e0        0x7 output_pic32_ssd1963\SD-SPI.o
                0xa00005e0                MDD_SDSPI_finalLBA
                0xa00005e4                gMediaSectorSize
                0xa00005e6                gSDMode
 *fill*         0xa00005e7        0x1 00
 .scommon       0xa00005e8       0x18 output_pic32_ssd1963\ImageDecoder.o
                0xa00005e8                IMG_wWidth
                0xa00005ea                IMG_bAlignCenter
                0xa00005ec                IMG_wStartX
                0xa00005ee                IMG_wHeight
                0xa00005f0                IMG_bDownScalingFactor
                0xa00005f2                IMG_wStartY
                0xa00005f4                IMG_wImageWidth
                0xa00005f6                IMG_wImageHeight
                0xa00005f8                IMG_blAbortImageDecoding
                0xa00005fc                IMG_pLoopCallbackFn
 .scommon       0xa0000600        0x2 output_pic32_ssd1963\Beep.o
                0xa0000600                pulseCounter
 .scommon       0xa0000602       0x10 output_pic32_ssd1963\DisplayDriver.o
                0xa0000602                _activePage
                0xa0000604                _clipRgn
                0xa0000606                _visualPage
                0xa0000608                _clipRight
                0xa000060a                _clipBottom
                0xa000060c                _clipTop
                0xa000060e                _color
                0xa0000610                _clipLeft
 *fill*         0xa0000612        0x2 00
 .scommon       0xa0000614       0x13 output_pic32_ssd1963\Primitive.o
                0xa0000614                _cursorY
                0xa0000616                _fontOrientation
                0xa0000618                _fontFirstChar
                0xa000061a                _fontHeight
                0xa000061c                _cursorX
                0xa000061e                _fontLastChar
                0xa0000620                _font
                0xa0000624                _lineType
                0xa0000626                _lineThickness
 *fill*         0xa0000627        0x1 00
 .scommon       0xa0000628       0x12 output_pic32_ssd1963\GOL.o
                0xa0000628                _rpnlX2
                0xa000062a                _rpnlR
                0xa000062c                _rpnlX1
                0xa000062e                _rpnlEmbossDkColor
                0xa0000630                _rpnlEmbossSize
                0xa0000632                _rpnlY2
                0xa0000634                _rpnlEmbossLtColor
                0xa0000636                _rpnlFaceColor
                0xa0000638                _rpnlY1
                0xa000063a                _sbss_end = .

.bss            0xa000063c     0x1734 load address 0x9d05f078
 *(.dynbss)
 *(.bss .bss.* .gnu.linkonce.b.*)
 .bss           0xa000063c        0xc output_pic32_ssd1963\Meter.o
 .bss.allocs    0xa0000648       0x10 C:/Program Files/Microchip/mplabc32/v1.12/bin/../lib/gcc/pic32mx/3.4.4/../../../../pic32mx/lib/size\libc.a(malloc.o)
 .bss.mem.0     0xa0000658       0x18 C:/Program Files/Microchip/mplabc32/v1.12/bin/../lib/gcc/pic32mx/3.4.4/../../../../pic32mx/lib/size\libc.a(sbrk.o)
 *(COMMON)
 COMMON         0xa0000670       0x20 output_pic32_ssd1963\rtcc.o
                0xa0000670                _time
                0xa0000680                _time_chk
 COMMON         0xa0000690      0x220 output_pic32_ssd1963\ECG.o
                0xa0000690                tempBuffer
                0xa00006a4                ecgBuffer
                0xa00008a4                buffer
 COMMON         0xa00008b0     0x13b0 output_pic32_ssd1963\Games.o
                0xa00008b0                snake
                0xa0000b14                scoreInfo
                0xa0000b48                balls
                0xa0000b60                field
 COMMON         0xa0001c60       0x20 output_pic32_ssd1963\RGBDemo.o
                0xa0001c60                PolyPoints
 COMMON         0xa0001c80       0x90 output_pic32_ssd1963\MultiFontsDemo.o
                0xa0001c80                HWLang
 COMMON         0xa0001d10       0x24 output_pic32_ssd1963\SlideShowDemo.o
                0xa0001d10                PixArray
 COMMON         0xa0001d34       0x3c output_pic32_ssd1963\GraphShow.o
                0xa0001d34                DemoTitle
                0xa0001d70                . = ALIGN (0x4)
                0xa0001d70                . = ALIGN (0x4)
                0xa0001d70                _end = .
                0xa0001d70                _bss_end = .

.heap           0xa0001d70     0x2400 load address 0x9d05f078
                0xa0001d70                _heap = .
                0xa0004170                . = (. + _min_heap_size)
 *fill*         0xa0001d70     0x2400 00
                0xa0004170                . = ALIGN (0x8)

.stack          0xa0004170      0x800 load address 0x9d05f078
                0xa0004170                _splim = .
                0xa0004170                _SPLIM = .
                0xa0004970                . = (. + _min_stack_size)
 *fill*         0xa0004170      0x800 00
                0xa0004970                . = ALIGN (0x8)

.ramfunc        0xa0005000        0x0 load address 0x9d05f078
                0xa0005000                _ramfunc_begin = .
 *(.ramfunc .ramfunc.*)
                0xa0005000                . = ALIGN (0x4)
                0xa0005000                _ramfunc_end = .
                0x9d05f078                _ramfunc_image_begin = LOADADDR (.ramfunc)
                0x00000000                _ramfunc_length = SIZEOF (.ramfunc)
                0x00005000                _bmxdkpba_address = (_ramfunc_begin - 0xa0000000)
                0x00008000                _bmxdudba_address = 0x8000
                0x00008000                _bmxdupba_address = 0x8000
                0xa0008000                _stack = (_ramfunc_length > 0x0)?(_ramfunc_begin - 0x8):0xa0008000
                0x00000001                ASSERT (((_min_stack_size + _min_heap_size) <= (_stack - _heap)), Not enough space to allocate both stack and heap.  Reduce heap and/or stack size.)

/DISCARD/
 *(.pdr)
 *(.reginfo)
 *(.rel.dyn)
 *(.note.GNU-stack)

.stab
 *(.stab)

.stabstr
 *(.stabstr)

.stab.excl
 *(.stab.excl)

.stab.exclstr
 *(.stab.exclstr)

.stab.index
 *(.stab.index)

.stab.indexstr
 *(.stab.indexstr)

.mdebug.abi32   0x00000000        0x0
 .mdebug.abi32  0x00000000        0x0 output_pic32_ssd1963\MainDemo.o
 .mdebug.abi32  0x00000000        0x0 output_pic32_ssd1963\rtcc.o
 .mdebug.abi32  0x00000000        0x0 output_pic32_ssd1963\Fonts.o
 .mdebug.abi32  0x00000000        0x0 output_pic32_ssd1963\DemoSelection.o
 .mdebug.abi32  0x00000000        0x0 output_pic32_ssd1963\Animation.o
 .mdebug.abi32  0x00000000        0x0 output_pic32_ssd1963\AnimationBitmaps.o
 .mdebug.abi32  0x00000000        0x0 output_pic32_ssd1963\ECG.o
 .mdebug.abi32  0x00000000        0x0 output_pic32_ssd1963\Games.o
 .mdebug.abi32  0x00000000        0x0 output_pic32_ssd1963\SnakeBitmaps.o
 .mdebug.abi32  0x00000000        0x0 output_pic32_ssd1963\ECGBitmaps.o
 .mdebug.abi32  0x00000000        0x0 output_pic32_ssd1963\RGBDemo.o
 .mdebug.abi32  0x00000000        0x0 output_pic32_ssd1963\MultiFontsDemo.o
 .mdebug.abi32  0x00000000        0x0 output_pic32_ssd1963\HelloWorldFonts.o
 .mdebug.abi32  0x00000000        0x0 output_pic32_ssd1963\TimeDateDemo.o
 .mdebug.abi32  0x00000000        0x0 output_pic32_ssd1963\DrawTool.o
 .mdebug.abi32  0x00000000        0x0 output_pic32_ssd1963\SlideShowDemo.o
 .mdebug.abi32  0x00000000        0x0 output_pic32_ssd1963\Icons.o
 .mdebug.abi32  0x00000000        0x0 output_pic32_ssd1963\DemoSteps.o
 .mdebug.abi32  0x00000000        0x0 output_pic32_ssd1963\SideButtons.o
 .mdebug.abi32  0x00000000        0x0 output_pic32_ssd1963\BitmapFile.o
 .mdebug.abi32  0x00000000        0x0 output_pic32_ssd1963\GraphShow.o
 .mdebug.abi32  0x00000000        0x0 output_pic32_ssd1963\FSIO.o
 .mdebug.abi32  0x00000000        0x0 output_pic32_ssd1963\SD-SPI.o
 .mdebug.abi32  0x00000000        0x0 output_pic32_ssd1963\JpegDecoder.o
 .mdebug.abi32  0x00000000        0x0 output_pic32_ssd1963\BmpDecoder.o
 .mdebug.abi32  0x00000000        0x0 output_pic32_ssd1963\GifDecoder.o
 .mdebug.abi32  0x00000000        0x0 output_pic32_ssd1963\ImageDecoder.o
 .mdebug.abi32  0x00000000        0x0 output_pic32_ssd1963\jidctint.o
 .mdebug.abi32  0x00000000        0x0 output_pic32_ssd1963\TouchScreen.o
 .mdebug.abi32  0x00000000        0x0 output_pic32_ssd1963\Beep.o
 .mdebug.abi32  0x00000000        0x0 output_pic32_ssd1963\EEPROM.o
 .mdebug.abi32  0x00000000        0x0 output_pic32_ssd1963\Window.o
 .mdebug.abi32  0x00000000        0x0 output_pic32_ssd1963\Button.o
 .mdebug.abi32  0x00000000        0x0 output_pic32_ssd1963\Chart.o
 .mdebug.abi32  0x00000000        0x0 output_pic32_ssd1963\CheckBox.o
 .mdebug.abi32  0x00000000        0x0 output_pic32_ssd1963\DisplayDriver.o
 .mdebug.abi32  0x00000000        0x0 output_pic32_ssd1963\EditBox.o
 .mdebug.abi32  0x00000000        0x0 output_pic32_ssd1963\Grid.o
 .mdebug.abi32  0x00000000        0x0 output_pic32_ssd1963\GroupBox.o
 .mdebug.abi32  0x00000000        0x0 output_pic32_ssd1963\ListBox.o
 .mdebug.abi32  0x00000000        0x0 output_pic32_ssd1963\Meter.o
 .mdebug.abi32  0x00000000        0x0 output_pic32_ssd1963\Picture.o
 .mdebug.abi32  0x00000000        0x0 output_pic32_ssd1963\Primitive.o
 .mdebug.abi32  0x00000000        0x0 output_pic32_ssd1963\RadioButton.o
 .mdebug.abi32  0x00000000        0x0 output_pic32_ssd1963\Slider.o
 .mdebug.abi32  0x00000000        0x0 output_pic32_ssd1963\StaticText.o
 .mdebug.abi32  0x00000000        0x0 output_pic32_ssd1963\GOLFontDefault.o
 .mdebug.abi32  0x00000000        0x0 output_pic32_ssd1963\GOL.o
 .mdebug.abi32  0x00000000        0x0 output_pic32_ssd1963\uart2.o
 .mdebug.abi32  0x00000000        0x0 output_pic32_ssd1963\JPEGDemo.o
 .mdebug.abi32  0x00000000        0x0 output_pic32_ssd1963\IconsC32.o
 .mdebug.abi32  0x00000000        0x0 output_pic32_ssd1963\SlideShowC32.o
 .mdebug.abi32  0x00000000        0x0 output_pic32_ssd1963\vs1003b.o
 .mdebug.abi32  0x00000000        0x0 C:/Program Files/Microchip/mplabc32/v1.12/bin/../lib/gcc/pic32mx/3.4.4/../../../../pic32mx/lib/size\libc.a(ctypef.o)
 .mdebug.abi32  0x00000000        0x0 C:/Program Files/Microchip/mplabc32/v1.12/bin/../lib/gcc/pic32mx/3.4.4/../../../../pic32mx/lib/size\libc.a(malloc.o)
 .mdebug.abi32  0x00000000        0x0 C:/Program Files/Microchip/mplabc32/v1.12/bin/../lib/gcc/pic32mx/3.4.4/../../../../pic32mx/lib/size\libc.a(rand.o)
 .mdebug.abi32  0x00000000        0x0 C:/Program Files/Microchip/mplabc32/v1.12/bin/../lib/gcc/pic32mx/3.4.4/../../../../pic32mx/lib/size\libc.a(strchr.o)
 .mdebug.abi32  0x00000000        0x0 C:/Program Files/Microchip/mplabc32/v1.12/bin/../lib/gcc/pic32mx/3.4.4/../../../../pic32mx/lib/size\libc.a(strncpy.o)
 .mdebug.abi32  0x00000000        0x0 C:/Program Files/Microchip/mplabc32/v1.12/bin/../lib/gcc/pic32mx/3.4.4/../../../../pic32mx/lib/size\libc.a(sbrk.o)
 .mdebug.abi32  0x00000000        0x0 C:/Program Files/Microchip/mplabc32/v1.12/bin/../lib/gcc/pic32mx/3.4.4/../../../../pic32mx/lib/size\libc.a(default-general-exception-handler.o)
 .mdebug.abi32  0x00000000        0x0 C:/Program Files/Microchip/mplabc32/v1.12/bin/../lib/gcc/pic32mx/3.4.4/../../../../pic32mx/lib/size\libc.a(default-bootstrap-exception-handler.o)
 .mdebug.abi32  0x00000000        0x0 C:/Program Files/Microchip/mplabc32/v1.12/bin/../lib/gcc/pic32mx/3.4.4/../../../../pic32mx/lib/size\libc.a(default-on-reset.o)
 .mdebug.abi32  0x00000000        0x0 C:/Program Files/Microchip/mplabc32/v1.12/bin/../lib/gcc/pic32mx/3.4.4/../../../../pic32mx/lib/size\libc.a(default-on-bootstrap.o)
 .mdebug.abi32  0x00000000        0x0 C:/Program Files/Microchip/mplabc32/v1.12/bin/../lib/gcc/pic32mx/3.4.4/../../../../pic32mx/lib/size\libc.a(ctype.o)
 .mdebug.abi32  0x00000000        0x0 C:/Program Files/Microchip/mplabc32/v1.12/bin/../lib/gcc/pic32mx/3.4.4/../../../../pic32mx/lib/size\libc.a(errno.o)
 .mdebug.abi32  0x00000000        0x0 C:/Program Files/Microchip/mplabc32/v1.12/bin/../lib/gcc/pic32mx/3.4.4/../../../../pic32mx/lib/size\libmchp_peripheral.a(open_core_timer_lib.o)
 .mdebug.abi32  0x00000000        0x0 C:/Program Files/Microchip/mplabc32/v1.12/bin/../lib/gcc/pic32mx/3.4.4/../../../../pic32mx/lib/size\libmchp_peripheral_32MX360F512L.a(pcache.o)
 .mdebug.abi32  0x00000000        0x0 C:/Program Files/Microchip/mplabc32/v1.12/bin/../lib/gcc/pic32mx/3.4.4/../../../../pic32mx/lib/size\libmchp_peripheral_32MX360F512L.a(int_disable_interrupts_lib.o)
 .mdebug.abi32  0x00000000        0x0 C:/Program Files/Microchip/mplabc32/v1.12/bin/../lib/gcc/pic32mx/3.4.4/../../../../pic32mx/lib/size\libmchp_peripheral_32MX360F512L.a(int_restore_interrupts_lib.o)
 .mdebug.abi32  0x00000000        0x0 C:/Program Files/Microchip/mplabc32/v1.12/bin/../lib/gcc/pic32mx/3.4.4/../../../../pic32mx/lib/size\libmchp_peripheral_32MX360F512L.a(int_enable_mv_int_lib.o)
 .mdebug.abi32  0x00000000        0x0 C:/Program Files/Microchip/mplabc32/v1.12/bin/../lib/gcc/pic32mx/3.4.4/../../../../pic32mx/lib/size\libmchp_peripheral_32MX360F512L.a(rtcc_init_lib.o)
 .mdebug.abi32  0x00000000        0x0 C:/Program Files/Microchip/mplabc32/v1.12/bin/../lib/gcc/pic32mx/3.4.4/../../../../pic32mx/lib/size\libmchp_peripheral_32MX360F512L.a(rtcc_set_date_lib.o)
 .mdebug.abi32  0x00000000        0x0 C:/Program Files/Microchip/mplabc32/v1.12/bin/../lib/gcc/pic32mx/3.4.4/../../../../pic32mx/lib/size\libmchp_peripheral_32MX360F512L.a(rtcc_set_time_lib.o)
 .mdebug.abi32  0x00000000        0x0 C:/Program Files/Microchip/mplabc32/v1.12/bin/../lib/gcc/pic32mx/3.4.4/../../../../pic32mx/lib/size\libmchp_peripheral_32MX360F512L.a(spi_getc_spi2_lib_legacy.o)
 .mdebug.abi32  0x00000000        0x0 C:/Program Files/Microchip/mplabc32/v1.12/bin/../lib/gcc/pic32mx/3.4.4/../../../../pic32mx/lib/size\libmchp_peripheral_32MX360F512L.a(spi_open_spi2_lib_legacy.o)
 .mdebug.abi32  0x00000000        0x0 C:/Program Files/Microchip/mplabc32/v1.12/bin/../lib/gcc/pic32mx/3.4.4/../../../../pic32mx/lib/size\libmchp_peripheral_32MX360F512L.a(spi_brg_tbl_lib_legacy.o)
 .mdebug.abi32  0x00000000        0x0 C:/Program Files/Microchip/mplabc32/v1.12/bin/../lib/gcc/pic32mx/3.4.4/../../../../pic32mx/lib/size\libmchp_peripheral_32MX360F512L.a(int_enable_interrupts_lib.o)
 .mdebug.abi32  0x00000000        0x0 C:/Program Files/Microchip/mplabc32/v1.12/bin/../lib/gcc/pic32mx/3.4.4/../../../../pic32mx/lib/size\libmchp_peripheral_32MX360F512L.a(int_tbl_lib.o)
 .mdebug.abi32  0x00000000        0x0 C:/Program Files/Microchip/mplabc32/v1.12/bin/../lib/gcc/pic32mx/3.4.4/../../../../pic32mx/lib/size\libmchp_peripheral_32MX360F512L.a(_rtcc_set_time_and_date_lib.o)
 .mdebug.abi32  0x00000000        0x0 C:/Program Files/Microchip/mplabc32/v1.12/bin/../lib/gcc/pic32mx/3.4.4/../../../../pic32mx/lib/size\libmchp_peripheral_32MX360F512L.a(_rtcc_wait_clock_off_lib.o)
 .mdebug.abi32  0x00000000        0x0 C:/Program Files/Microchip/mplabc32/v1.12/bin/../lib/gcc/pic32mx/3.4.4/../../../../pic32mx/lib/size\libmchp_peripheral_32MX360F512L.a(read_core_timer_lib.o)

.comment        0x00000000     0x1a47
 *(.comment)
 .comment       0x00000000       0x4d output_pic32_ssd1963\MainDemo.o
 .comment       0x0000004d       0x4d output_pic32_ssd1963\rtcc.o
 .comment       0x0000009a       0x4d output_pic32_ssd1963\Fonts.o
 .comment       0x000000e7       0x4d output_pic32_ssd1963\DemoSelection.o
 .comment       0x00000134       0x4d output_pic32_ssd1963\Animation.o
 .comment       0x00000181       0x4d output_pic32_ssd1963\AnimationBitmaps.o
 .comment       0x000001ce       0x4d output_pic32_ssd1963\ECG.o
 .comment       0x0000021b       0x4d output_pic32_ssd1963\Games.o
 .comment       0x00000268       0x4d output_pic32_ssd1963\SnakeBitmaps.o
 .comment       0x000002b5       0x4d output_pic32_ssd1963\ECGBitmaps.o
 .comment       0x00000302       0x4d output_pic32_ssd1963\RGBDemo.o
 .comment       0x0000034f       0x4d output_pic32_ssd1963\MultiFontsDemo.o
 .comment       0x0000039c       0x4d output_pic32_ssd1963\HelloWorldFonts.o
 .comment       0x000003e9       0x4d output_pic32_ssd1963\TimeDateDemo.o
 .comment       0x00000436       0x4d output_pic32_ssd1963\DrawTool.o
 .comment       0x00000483       0x4d output_pic32_ssd1963\SlideShowDemo.o
 .comment       0x000004d0       0x4d output_pic32_ssd1963\Icons.o
 .comment       0x0000051d       0x4d output_pic32_ssd1963\DemoSteps.o
 .comment       0x0000056a       0x4d output_pic32_ssd1963\SideButtons.o
 .comment       0x000005b7       0x4d output_pic32_ssd1963\BitmapFile.o
 .comment       0x00000604       0x4d output_pic32_ssd1963\GraphShow.o
 .comment       0x00000651       0x4d output_pic32_ssd1963\FSIO.o
 .comment       0x0000069e       0x4d output_pic32_ssd1963\SD-SPI.o
 .comment       0x000006eb       0x4d output_pic32_ssd1963\JpegDecoder.o
 .comment       0x00000738       0x4d output_pic32_ssd1963\BmpDecoder.o
 .comment       0x00000785       0x4d output_pic32_ssd1963\GifDecoder.o
 .comment       0x000007d2       0x4d output_pic32_ssd1963\ImageDecoder.o
 .comment       0x0000081f       0x4d output_pic32_ssd1963\jidctint.o
 .comment       0x0000086c       0x4d output_pic32_ssd1963\TouchScreen.o
 .comment       0x000008b9       0x4d output_pic32_ssd1963\Beep.o
 .comment       0x00000906       0x4d output_pic32_ssd1963\EEPROM.o
 .comment       0x00000953       0x4d output_pic32_ssd1963\Window.o
 .comment       0x000009a0       0x4d output_pic32_ssd1963\Button.o
 .comment       0x000009ed       0x4d output_pic32_ssd1963\Chart.o
 .comment       0x00000a3a       0x4d output_pic32_ssd1963\CheckBox.o
 .comment       0x00000a87       0x4d output_pic32_ssd1963\DisplayDriver.o
 .comment       0x00000ad4       0x4d output_pic32_ssd1963\EditBox.o
 .comment       0x00000b21       0x4d output_pic32_ssd1963\Grid.o
 .comment       0x00000b6e       0x4d output_pic32_ssd1963\GroupBox.o
 .comment       0x00000bbb       0x4d output_pic32_ssd1963\ListBox.o
 .comment       0x00000c08       0x4d output_pic32_ssd1963\Meter.o
 .comment       0x00000c55       0x4d output_pic32_ssd1963\Picture.o
 .comment       0x00000ca2       0x4d output_pic32_ssd1963\Primitive.o
 .comment       0x00000cef       0x4d output_pic32_ssd1963\RadioButton.o
 .comment       0x00000d3c       0x4d output_pic32_ssd1963\Slider.o
 .comment       0x00000d89       0x4d output_pic32_ssd1963\StaticText.o
 .comment       0x00000dd6       0x4d output_pic32_ssd1963\GOLFontDefault.o
 .comment       0x00000e23       0x4d output_pic32_ssd1963\GOL.o
 .comment       0x00000e70       0x4d output_pic32_ssd1963\uart2.o
 .comment       0x00000ebd       0x4d output_pic32_ssd1963\JPEGDemo.o
 .comment       0x00000f0a       0x4d output_pic32_ssd1963\IconsC32.o
 .comment       0x00000f57       0x4d output_pic32_ssd1963\SlideShowC32.o
 .comment       0x00000fa4       0x4d output_pic32_ssd1963\vs1003b.o
 .comment       0x00000ff1       0x56 C:/Program Files/Microchip/mplabc32/v1.12/bin/../lib/gcc/pic32mx/3.4.4/../../../../pic32mx/lib/size\libc.a(memset.o)
 .comment       0x00001047       0x56 C:/Program Files/Microchip/mplabc32/v1.12/bin/../lib/gcc/pic32mx/3.4.4/../../../../pic32mx/lib/size\libc.a(strcpy.o)
 .comment       0x0000109d       0x56 C:/Program Files/Microchip/mplabc32/v1.12/bin/../lib/gcc/pic32mx/3.4.4/../../../../pic32mx/lib/size\libc.a(strlen.o)
 .comment       0x000010f3       0x9c C:/Program Files/Microchip/mplabc32/v1.12/bin/../lib/gcc/pic32mx/3.4.4/../../../../pic32mx/lib/size\libc.a(ctypef.o)
 .comment       0x0000118f       0x4d C:/Program Files/Microchip/mplabc32/v1.12/bin/../lib/gcc/pic32mx/3.4.4/../../../../pic32mx/lib/size\libc.a(malloc.o)
 .comment       0x000011dc       0x4d C:/Program Files/Microchip/mplabc32/v1.12/bin/../lib/gcc/pic32mx/3.4.4/../../../../pic32mx/lib/size\libc.a(rand.o)
 .comment       0x00001229       0x4d C:/Program Files/Microchip/mplabc32/v1.12/bin/../lib/gcc/pic32mx/3.4.4/../../../../pic32mx/lib/size\libc.a(strchr.o)
 .comment       0x00001276       0x4d C:/Program Files/Microchip/mplabc32/v1.12/bin/../lib/gcc/pic32mx/3.4.4/../../../../pic32mx/lib/size\libc.a(strncpy.o)
 .comment       0x000012c3       0x98 C:/Program Files/Microchip/mplabc32/v1.12/bin/../lib/gcc/pic32mx/3.4.4/../../../../pic32mx/lib/size\libc.a(sbrk.o)
 .comment       0x0000135b       0x4d C:/Program Files/Microchip/mplabc32/v1.12/bin/../lib/gcc/pic32mx/3.4.4/../../../../pic32mx/lib/size\libc.a(default-general-exception-handler.o)
 .comment       0x000013a8       0x4d C:/Program Files/Microchip/mplabc32/v1.12/bin/../lib/gcc/pic32mx/3.4.4/../../../../pic32mx/lib/size\libc.a(default-bootstrap-exception-handler.o)
 .comment       0x000013f5       0x4d C:/Program Files/Microchip/mplabc32/v1.12/bin/../lib/gcc/pic32mx/3.4.4/../../../../pic32mx/lib/size\libc.a(default-on-reset.o)
 .comment       0x00001442       0x4d C:/Program Files/Microchip/mplabc32/v1.12/bin/../lib/gcc/pic32mx/3.4.4/../../../../pic32mx/lib/size\libc.a(default-on-bootstrap.o)
 .comment       0x0000148f       0x9b C:/Program Files/Microchip/mplabc32/v1.12/bin/../lib/gcc/pic32mx/3.4.4/../../../../pic32mx/lib/size\libc.a(ctype.o)
 .comment       0x0000152a       0x4d C:/Program Files/Microchip/mplabc32/v1.12/bin/../lib/gcc/pic32mx/3.4.4/../../../../pic32mx/lib/size\libc.a(errno.o)
 .comment       0x00001577       0x4d C:/Program Files/Microchip/mplabc32/v1.12/bin/../lib/gcc/pic32mx/3.4.4/../../../../pic32mx/lib/size\libmchp_peripheral.a(open_core_timer_lib.o)
 .comment       0x000015c4       0x4d C:/Program Files/Microchip/mplabc32/v1.12/bin/../lib/gcc/pic32mx/3.4.4/../../../../pic32mx/lib/size\libmchp_peripheral_32MX360F512L.a(pcache.o)
 .comment       0x00001611       0x4d C:/Program Files/Microchip/mplabc32/v1.12/bin/../lib/gcc/pic32mx/3.4.4/../../../../pic32mx/lib/size\libmchp_peripheral_32MX360F512L.a(int_disable_interrupts_lib.o)
 .comment       0x0000165e       0x4d C:/Program Files/Microchip/mplabc32/v1.12/bin/../lib/gcc/pic32mx/3.4.4/../../../../pic32mx/lib/size\libmchp_peripheral_32MX360F512L.a(int_restore_interrupts_lib.o)
 .comment       0x000016ab       0x4d C:/Program Files/Microchip/mplabc32/v1.12/bin/../lib/gcc/pic32mx/3.4.4/../../../../pic32mx/lib/size\libmchp_peripheral_32MX360F512L.a(int_enable_mv_int_lib.o)
 .comment       0x000016f8       0x4d C:/Program Files/Microchip/mplabc32/v1.12/bin/../lib/gcc/pic32mx/3.4.4/../../../../pic32mx/lib/size\libmchp_peripheral_32MX360F512L.a(rtcc_init_lib.o)
 .comment       0x00001745       0x4d C:/Program Files/Microchip/mplabc32/v1.12/bin/../lib/gcc/pic32mx/3.4.4/../../../../pic32mx/lib/size\libmchp_peripheral_32MX360F512L.a(rtcc_set_date_lib.o)
 .comment       0x00001792       0x4d C:/Program Files/Microchip/mplabc32/v1.12/bin/../lib/gcc/pic32mx/3.4.4/../../../../pic32mx/lib/size\libmchp_peripheral_32MX360F512L.a(rtcc_set_time_lib.o)
 .comment       0x000017df       0x4d C:/Program Files/Microchip/mplabc32/v1.12/bin/../lib/gcc/pic32mx/3.4.4/../../../../pic32mx/lib/size\libmchp_peripheral_32MX360F512L.a(spi_getc_spi2_lib_legacy.o)
 .comment       0x0000182c       0x4d C:/Program Files/Microchip/mplabc32/v1.12/bin/../lib/gcc/pic32mx/3.4.4/../../../../pic32mx/lib/size\libmchp_peripheral_32MX360F512L.a(spi_open_spi2_lib_legacy.o)
 .comment       0x00001879       0x4d C:/Program Files/Microchip/mplabc32/v1.12/bin/../lib/gcc/pic32mx/3.4.4/../../../../pic32mx/lib/size\libmchp_peripheral_32MX360F512L.a(spi_brg_tbl_lib_legacy.o)
 .comment       0x000018c6       0x4d C:/Program Files/Microchip/mplabc32/v1.12/bin/../lib/gcc/pic32mx/3.4.4/../../../../pic32mx/lib/size\libmchp_peripheral_32MX360F512L.a(int_enable_interrupts_lib.o)
 .comment       0x00001913       0x4d C:/Program Files/Microchip/mplabc32/v1.12/bin/../lib/gcc/pic32mx/3.4.4/../../../../pic32mx/lib/size\libmchp_peripheral_32MX360F512L.a(int_tbl_lib.o)
 .comment       0x00001960       0x4d C:/Program Files/Microchip/mplabc32/v1.12/bin/../lib/gcc/pic32mx/3.4.4/../../../../pic32mx/lib/size\libmchp_peripheral_32MX360F512L.a(_rtcc_set_time_and_date_lib.o)
 .comment       0x000019ad       0x4d C:/Program Files/Microchip/mplabc32/v1.12/bin/../lib/gcc/pic32mx/3.4.4/../../../../pic32mx/lib/size\libmchp_peripheral_32MX360F512L.a(_rtcc_wait_clock_off_lib.o)
 .comment       0x000019fa       0x4d C:/Program Files/Microchip/mplabc32/v1.12/bin/../lib/gcc/pic32mx/3.4.4/../../../../pic32mx/lib/size\libmchp_peripheral_32MX360F512L.a(read_core_timer_lib.o)

.debug
 *(.debug)

.line
 *(.line)

.debug_srcinfo
 *(.debug_srcinfo)

.debug_sfnames
 *(.debug_sfnames)

.debug_aranges  0x00000000      0xa30
 *(.debug_aranges)
 .debug_aranges
                0x00000000       0x20 output_pic32_ssd1963\MainDemo.o
 .debug_aranges
                0x00000020       0x20 output_pic32_ssd1963\rtcc.o
 .debug_aranges
                0x00000040       0x20 output_pic32_ssd1963\DemoSelection.o
 .debug_aranges
                0x00000060       0x20 output_pic32_ssd1963\Animation.o
 .debug_aranges
                0x00000080       0x20 output_pic32_ssd1963\ECG.o
 .debug_aranges
                0x000000a0       0x20 output_pic32_ssd1963\Games.o
 .debug_aranges
                0x000000c0       0x20 output_pic32_ssd1963\RGBDemo.o
 .debug_aranges
                0x000000e0       0x20 output_pic32_ssd1963\MultiFontsDemo.o
 .debug_aranges
                0x00000100       0x20 output_pic32_ssd1963\TimeDateDemo.o
 .debug_aranges
                0x00000120       0x20 output_pic32_ssd1963\DrawTool.o
 .debug_aranges
                0x00000140       0x20 output_pic32_ssd1963\SlideShowDemo.o
 .debug_aranges
                0x00000160       0x20 output_pic32_ssd1963\DemoSteps.o
 .debug_aranges
                0x00000180       0x20 output_pic32_ssd1963\SideButtons.o
 .debug_aranges
                0x000001a0       0x20 output_pic32_ssd1963\GraphShow.o
 .debug_aranges
                0x000001c0       0x20 output_pic32_ssd1963\FSIO.o
 .debug_aranges
                0x000001e0       0x20 output_pic32_ssd1963\SD-SPI.o
 .debug_aranges
                0x00000200       0x20 output_pic32_ssd1963\JpegDecoder.o
 .debug_aranges
                0x00000220       0x20 output_pic32_ssd1963\BmpDecoder.o
 .debug_aranges
                0x00000240       0x20 output_pic32_ssd1963\GifDecoder.o
 .debug_aranges
                0x00000260       0x20 output_pic32_ssd1963\ImageDecoder.o
 .debug_aranges
                0x00000280       0x20 output_pic32_ssd1963\jidctint.o
 .debug_aranges
                0x000002a0       0x20 output_pic32_ssd1963\TouchScreen.o
 .debug_aranges
                0x000002c0       0x20 output_pic32_ssd1963\Beep.o
 .debug_aranges
                0x000002e0       0x20 output_pic32_ssd1963\EEPROM.o
 .debug_aranges
                0x00000300       0x20 output_pic32_ssd1963\Window.o
 .debug_aranges
                0x00000320       0x20 output_pic32_ssd1963\Button.o
 .debug_aranges
                0x00000340       0x20 output_pic32_ssd1963\Chart.o
 .debug_aranges
                0x00000360       0x20 output_pic32_ssd1963\CheckBox.o
 .debug_aranges
                0x00000380       0x20 output_pic32_ssd1963\DisplayDriver.o
 .debug_aranges
                0x000003a0       0x20 output_pic32_ssd1963\EditBox.o
 .debug_aranges
                0x000003c0       0x20 output_pic32_ssd1963\Grid.o
 .debug_aranges
                0x000003e0       0x20 output_pic32_ssd1963\GroupBox.o
 .debug_aranges
                0x00000400       0x20 output_pic32_ssd1963\ListBox.o
 .debug_aranges
                0x00000420       0x20 output_pic32_ssd1963\Meter.o
 .debug_aranges
                0x00000440       0x20 output_pic32_ssd1963\Picture.o
 .debug_aranges
                0x00000460       0x20 output_pic32_ssd1963\Primitive.o
 .debug_aranges
                0x00000480       0x20 output_pic32_ssd1963\RadioButton.o
 .debug_aranges
                0x000004a0       0x20 output_pic32_ssd1963\Slider.o
 .debug_aranges
                0x000004c0       0x20 output_pic32_ssd1963\StaticText.o
 .debug_aranges
                0x000004e0       0x20 output_pic32_ssd1963\GOL.o
 .debug_aranges
                0x00000500       0x20 output_pic32_ssd1963\uart2.o
 .debug_aranges
                0x00000520       0x20 output_pic32_ssd1963\vs1003b.o
 .debug_aranges
                0x00000540       0xa8 C:/Program Files/Microchip/mplabc32/v1.12/bin/../lib/gcc/pic32mx/3.4.4/../../../../pic32mx/lib/size\libc.a(ctypef.o)
 .debug_aranges
                0x000005e8       0x38 C:/Program Files/Microchip/mplabc32/v1.12/bin/../lib/gcc/pic32mx/3.4.4/../../../../pic32mx/lib/size\libc.a(malloc.o)
 .debug_aranges
                0x00000620       0x30 C:/Program Files/Microchip/mplabc32/v1.12/bin/../lib/gcc/pic32mx/3.4.4/../../../../pic32mx/lib/size\libc.a(rand.o)
 .debug_aranges
                0x00000650       0x28 C:/Program Files/Microchip/mplabc32/v1.12/bin/../lib/gcc/pic32mx/3.4.4/../../../../pic32mx/lib/size\libc.a(strchr.o)
 .debug_aranges
                0x00000678       0x28 C:/Program Files/Microchip/mplabc32/v1.12/bin/../lib/gcc/pic32mx/3.4.4/../../../../pic32mx/lib/size\libc.a(strncpy.o)
 .debug_aranges
                0x000006a0       0x48 C:/Program Files/Microchip/mplabc32/v1.12/bin/../lib/gcc/pic32mx/3.4.4/../../../../pic32mx/lib/size\libc.a(sbrk.o)
 .debug_aranges
                0x000006e8       0x28 C:/Program Files/Microchip/mplabc32/v1.12/bin/../lib/gcc/pic32mx/3.4.4/../../../../pic32mx/lib/size\libc.a(default-general-exception-handler.o)
 .debug_aranges
                0x00000710       0x28 C:/Program Files/Microchip/mplabc32/v1.12/bin/../lib/gcc/pic32mx/3.4.4/../../../../pic32mx/lib/size\libc.a(default-bootstrap-exception-handler.o)
 .debug_aranges
                0x00000738       0x28 C:/Program Files/Microchip/mplabc32/v1.12/bin/../lib/gcc/pic32mx/3.4.4/../../../../pic32mx/lib/size\libc.a(default-on-reset.o)
 .debug_aranges
                0x00000760       0x28 C:/Program Files/Microchip/mplabc32/v1.12/bin/../lib/gcc/pic32mx/3.4.4/../../../../pic32mx/lib/size\libc.a(default-on-bootstrap.o)
 .debug_aranges
                0x00000788       0x28 C:/Program Files/Microchip/mplabc32/v1.12/bin/../lib/gcc/pic32mx/3.4.4/../../../../pic32mx/lib/size\libmchp_peripheral.a(open_core_timer_lib.o)
 .debug_aranges
                0x000007b0       0x30 C:/Program Files/Microchip/mplabc32/v1.12/bin/../lib/gcc/pic32mx/3.4.4/../../../../pic32mx/lib/size\libmchp_peripheral_32MX360F512L.a(pcache.o)
 .debug_aranges
                0x000007e0       0x28 C:/Program Files/Microchip/mplabc32/v1.12/bin/../lib/gcc/pic32mx/3.4.4/../../../../pic32mx/lib/size\libmchp_peripheral_32MX360F512L.a(int_disable_interrupts_lib.o)
 .debug_aranges
                0x00000808       0x28 C:/Program Files/Microchip/mplabc32/v1.12/bin/../lib/gcc/pic32mx/3.4.4/../../../../pic32mx/lib/size\libmchp_peripheral_32MX360F512L.a(int_restore_interrupts_lib.o)
 .debug_aranges
                0x00000830       0x28 C:/Program Files/Microchip/mplabc32/v1.12/bin/../lib/gcc/pic32mx/3.4.4/../../../../pic32mx/lib/size\libmchp_peripheral_32MX360F512L.a(int_enable_mv_int_lib.o)
 .debug_aranges
                0x00000858       0x28 C:/Program Files/Microchip/mplabc32/v1.12/bin/../lib/gcc/pic32mx/3.4.4/../../../../pic32mx/lib/size\libmchp_peripheral_32MX360F512L.a(rtcc_init_lib.o)
 .debug_aranges
                0x00000880       0x28 C:/Program Files/Microchip/mplabc32/v1.12/bin/../lib/gcc/pic32mx/3.4.4/../../../../pic32mx/lib/size\libmchp_peripheral_32MX360F512L.a(rtcc_set_date_lib.o)
 .debug_aranges
                0x000008a8       0x28 C:/Program Files/Microchip/mplabc32/v1.12/bin/../lib/gcc/pic32mx/3.4.4/../../../../pic32mx/lib/size\libmchp_peripheral_32MX360F512L.a(rtcc_set_time_lib.o)
 .debug_aranges
                0x000008d0       0x28 C:/Program Files/Microchip/mplabc32/v1.12/bin/../lib/gcc/pic32mx/3.4.4/../../../../pic32mx/lib/size\libmchp_peripheral_32MX360F512L.a(spi_getc_spi2_lib_legacy.o)
 .debug_aranges
                0x000008f8       0x28 C:/Program Files/Microchip/mplabc32/v1.12/bin/../lib/gcc/pic32mx/3.4.4/../../../../pic32mx/lib/size\libmchp_peripheral_32MX360F512L.a(spi_open_spi2_lib_legacy.o)
 .debug_aranges
                0x00000920       0x28 C:/Program Files/Microchip/mplabc32/v1.12/bin/../lib/gcc/pic32mx/3.4.4/../../../../pic32mx/lib/size\libmchp_peripheral_32MX360F512L.a(int_enable_interrupts_lib.o)
 .debug_aranges
                0x00000948       0x68 C:/Program Files/Microchip/mplabc32/v1.12/bin/../lib/gcc/pic32mx/3.4.4/../../../../pic32mx/lib/size\libmchp_peripheral_32MX360F512L.a(int_tbl_lib.o)
 .debug_aranges
                0x000009b0       0x28 C:/Program Files/Microchip/mplabc32/v1.12/bin/../lib/gcc/pic32mx/3.4.4/../../../../pic32mx/lib/size\libmchp_peripheral_32MX360F512L.a(_rtcc_set_time_and_date_lib.o)
 .debug_aranges
                0x000009d8       0x30 C:/Program Files/Microchip/mplabc32/v1.12/bin/../lib/gcc/pic32mx/3.4.4/../../../../pic32mx/lib/size\libmchp_peripheral_32MX360F512L.a(_rtcc_wait_clock_off_lib.o)
 .debug_aranges
                0x00000a08       0x28 C:/Program Files/Microchip/mplabc32/v1.12/bin/../lib/gcc/pic32mx/3.4.4/../../../../pic32mx/lib/size\libmchp_peripheral_32MX360F512L.a(read_core_timer_lib.o)

.debug_pubnames
                0x00000000     0x39b8
 *(.debug_pubnames)
 .debug_pubnames
                0x00000000      0x38e output_pic32_ssd1963\MainDemo.o
 .debug_pubnames
                0x0000038e      0x11c output_pic32_ssd1963\rtcc.o
 .debug_pubnames
                0x000004aa       0x63 output_pic32_ssd1963\Fonts.o
 .debug_pubnames
                0x0000050d      0x196 output_pic32_ssd1963\DemoSelection.o
 .debug_pubnames
                0x000006a3       0x8a output_pic32_ssd1963\Animation.o
 .debug_pubnames
                0x0000072d       0x6e output_pic32_ssd1963\AnimationBitmaps.o
 .debug_pubnames
                0x0000079b      0x1b1 output_pic32_ssd1963\ECG.o
 .debug_pubnames
                0x0000094c      0x165 output_pic32_ssd1963\Games.o
 .debug_pubnames
                0x00000ab1       0x4e output_pic32_ssd1963\SnakeBitmaps.o
 .debug_pubnames
                0x00000aff       0x3f output_pic32_ssd1963\ECGBitmaps.o
 .debug_pubnames
                0x00000b3e      0x411 output_pic32_ssd1963\RGBDemo.o
 .debug_pubnames
                0x00000f4f      0x149 output_pic32_ssd1963\MultiFontsDemo.o
 .debug_pubnames
                0x00001098       0x7b output_pic32_ssd1963\HelloWorldFonts.o
 .debug_pubnames
                0x00001113      0x1e5 output_pic32_ssd1963\TimeDateDemo.o
 .debug_pubnames
                0x000012f8       0x7c output_pic32_ssd1963\DrawTool.o
 .debug_pubnames
                0x00001374       0x85 output_pic32_ssd1963\SlideShowDemo.o
 .debug_pubnames
                0x000013f9       0x75 output_pic32_ssd1963\Icons.o
 .debug_pubnames
                0x0000146e       0x78 output_pic32_ssd1963\DemoSteps.o
 .debug_pubnames
                0x000014e6       0x25 output_pic32_ssd1963\SideButtons.o
 .debug_pubnames
                0x0000150b      0x24e output_pic32_ssd1963\GraphShow.o
 .debug_pubnames
                0x00001759      0x5d9 output_pic32_ssd1963\FSIO.o
 .debug_pubnames
                0x00001d32      0x1ad output_pic32_ssd1963\SD-SPI.o
 .debug_pubnames
                0x00001edf       0x23 output_pic32_ssd1963\JpegDecoder.o
 .debug_pubnames
                0x00001f02       0x4b output_pic32_ssd1963\BmpDecoder.o
 .debug_pubnames
                0x00001f4d       0x22 output_pic32_ssd1963\GifDecoder.o
 .debug_pubnames
                0x00001f6f      0x139 output_pic32_ssd1963\ImageDecoder.o
 .debug_pubnames
                0x000020a8       0x26 output_pic32_ssd1963\jidctint.o
 .debug_pubnames
                0x000020ce      0x116 output_pic32_ssd1963\TouchScreen.o
 .debug_pubnames
                0x000021e4       0x41 output_pic32_ssd1963\Beep.o
 .debug_pubnames
                0x00002225       0xce output_pic32_ssd1963\EEPROM.o
 .debug_pubnames
                0x000022f3       0x4f output_pic32_ssd1963\Window.o
 .debug_pubnames
                0x00002342       0x61 output_pic32_ssd1963\Button.o
 .debug_pubnames
                0x000023a3      0x17a output_pic32_ssd1963\Chart.o
 .debug_pubnames
                0x0000251d       0x5c output_pic32_ssd1963\CheckBox.o
 .debug_pubnames
                0x00002579      0x1dd output_pic32_ssd1963\DisplayDriver.o
 .debug_pubnames
                0x00002756       0x7b output_pic32_ssd1963\EditBox.o
 .debug_pubnames
                0x000027d1       0xc5 output_pic32_ssd1963\Grid.o
 .debug_pubnames
                0x00002896       0x3d output_pic32_ssd1963\GroupBox.o
 .debug_pubnames
                0x000028d3       0xc4 output_pic32_ssd1963\ListBox.o
 .debug_pubnames
                0x00002997       0x85 output_pic32_ssd1963\Meter.o
 .debug_pubnames
                0x00002a1c       0x43 output_pic32_ssd1963\Picture.o
 .debug_pubnames
                0x00002a5f      0x15f output_pic32_ssd1963\Primitive.o
 .debug_pubnames
                0x00002bbe       0x8c output_pic32_ssd1963\RadioButton.o
 .debug_pubnames
                0x00002c4a       0xc8 output_pic32_ssd1963\Slider.o
 .debug_pubnames
                0x00002d12       0x4b output_pic32_ssd1963\StaticText.o
 .debug_pubnames
                0x00002d5d       0x30 output_pic32_ssd1963\GOLFontDefault.o
 .debug_pubnames
                0x00002d8d      0x1f2 output_pic32_ssd1963\GOL.o
 .debug_pubnames
                0x00002f7f       0xfc output_pic32_ssd1963\uart2.o
 .debug_pubnames
                0x0000307b      0x298 output_pic32_ssd1963\IconsC32.o
 .debug_pubnames
                0x00003313       0x50 output_pic32_ssd1963\SlideShowC32.o
 .debug_pubnames
                0x00003363       0x81 output_pic32_ssd1963\vs1003b.o
 .debug_pubnames
                0x000033e4       0xe1 C:/Program Files/Microchip/mplabc32/v1.12/bin/../lib/gcc/pic32mx/3.4.4/../../../../pic32mx/lib/size\libc.a(ctypef.o)
 .debug_pubnames
                0x000034c5       0x32 C:/Program Files/Microchip/mplabc32/v1.12/bin/../lib/gcc/pic32mx/3.4.4/../../../../pic32mx/lib/size\libc.a(malloc.o)
 .debug_pubnames
                0x000034f7       0x25 C:/Program Files/Microchip/mplabc32/v1.12/bin/../lib/gcc/pic32mx/3.4.4/../../../../pic32mx/lib/size\libc.a(rand.o)
 .debug_pubnames
                0x0000351c       0x1d C:/Program Files/Microchip/mplabc32/v1.12/bin/../lib/gcc/pic32mx/3.4.4/../../../../pic32mx/lib/size\libc.a(strchr.o)
 .debug_pubnames
                0x00003539       0x1e C:/Program Files/Microchip/mplabc32/v1.12/bin/../lib/gcc/pic32mx/3.4.4/../../../../pic32mx/lib/size\libc.a(strncpy.o)
 .debug_pubnames
                0x00003557       0x74 C:/Program Files/Microchip/mplabc32/v1.12/bin/../lib/gcc/pic32mx/3.4.4/../../../../pic32mx/lib/size\libc.a(sbrk.o)
 .debug_pubnames
                0x000035cb       0x31 C:/Program Files/Microchip/mplabc32/v1.12/bin/../lib/gcc/pic32mx/3.4.4/../../../../pic32mx/lib/size\libc.a(default-general-exception-handler.o)
 .debug_pubnames
                0x000035fc       0x33 C:/Program Files/Microchip/mplabc32/v1.12/bin/../lib/gcc/pic32mx/3.4.4/../../../../pic32mx/lib/size\libc.a(default-bootstrap-exception-handler.o)
 .debug_pubnames
                0x0000362f       0x20 C:/Program Files/Microchip/mplabc32/v1.12/bin/../lib/gcc/pic32mx/3.4.4/../../../../pic32mx/lib/size\libc.a(default-on-reset.o)
 .debug_pubnames
                0x0000364f       0x24 C:/Program Files/Microchip/mplabc32/v1.12/bin/../lib/gcc/pic32mx/3.4.4/../../../../pic32mx/lib/size\libc.a(default-on-bootstrap.o)
 .debug_pubnames
                0x00003673       0x1d C:/Program Files/Microchip/mplabc32/v1.12/bin/../lib/gcc/pic32mx/3.4.4/../../../../pic32mx/lib/size\libc.a(ctype.o)
 .debug_pubnames
                0x00003690       0x1c C:/Program Files/Microchip/mplabc32/v1.12/bin/../lib/gcc/pic32mx/3.4.4/../../../../pic32mx/lib/size\libc.a(errno.o)
 .debug_pubnames
                0x000036ac       0x24 C:/Program Files/Microchip/mplabc32/v1.12/bin/../lib/gcc/pic32mx/3.4.4/../../../../pic32mx/lib/size\libmchp_peripheral.a(open_core_timer_lib.o)
 .debug_pubnames
                0x000036d0       0x3b C:/Program Files/Microchip/mplabc32/v1.12/bin/../lib/gcc/pic32mx/3.4.4/../../../../pic32mx/lib/size\libmchp_peripheral_32MX360F512L.a(pcache.o)
 .debug_pubnames
                0x0000370b       0x2b C:/Program Files/Microchip/mplabc32/v1.12/bin/../lib/gcc/pic32mx/3.4.4/../../../../pic32mx/lib/size\libmchp_peripheral_32MX360F512L.a(int_disable_interrupts_lib.o)
 .debug_pubnames
                0x00003736       0x2b C:/Program Files/Microchip/mplabc32/v1.12/bin/../lib/gcc/pic32mx/3.4.4/../../../../pic32mx/lib/size\libmchp_peripheral_32MX360F512L.a(int_restore_interrupts_lib.o)
 .debug_pubnames
                0x00003761       0x36 C:/Program Files/Microchip/mplabc32/v1.12/bin/../lib/gcc/pic32mx/3.4.4/../../../../pic32mx/lib/size\libmchp_peripheral_32MX360F512L.a(int_enable_mv_int_lib.o)
 .debug_pubnames
                0x00003797       0x1f C:/Program Files/Microchip/mplabc32/v1.12/bin/../lib/gcc/pic32mx/3.4.4/../../../../pic32mx/lib/size\libmchp_peripheral_32MX360F512L.a(rtcc_init_lib.o)
 .debug_pubnames
                0x000037b6       0x22 C:/Program Files/Microchip/mplabc32/v1.12/bin/../lib/gcc/pic32mx/3.4.4/../../../../pic32mx/lib/size\libmchp_peripheral_32MX360F512L.a(rtcc_set_date_lib.o)
 .debug_pubnames
                0x000037d8       0x22 C:/Program Files/Microchip/mplabc32/v1.12/bin/../lib/gcc/pic32mx/3.4.4/../../../../pic32mx/lib/size\libmchp_peripheral_32MX360F512L.a(rtcc_set_time_lib.o)
 .debug_pubnames
                0x000037fa       0x1f C:/Program Files/Microchip/mplabc32/v1.12/bin/../lib/gcc/pic32mx/3.4.4/../../../../pic32mx/lib/size\libmchp_peripheral_32MX360F512L.a(spi_getc_spi2_lib_legacy.o)
 .debug_pubnames
                0x00003819       0x1f C:/Program Files/Microchip/mplabc32/v1.12/bin/../lib/gcc/pic32mx/3.4.4/../../../../pic32mx/lib/size\libmchp_peripheral_32MX360F512L.a(spi_open_spi2_lib_legacy.o)
 .debug_pubnames
                0x00003838       0x2a C:/Program Files/Microchip/mplabc32/v1.12/bin/../lib/gcc/pic32mx/3.4.4/../../../../pic32mx/lib/size\libmchp_peripheral_32MX360F512L.a(int_enable_interrupts_lib.o)
 .debug_pubnames
                0x00003862       0xca C:/Program Files/Microchip/mplabc32/v1.12/bin/../lib/gcc/pic32mx/3.4.4/../../../../pic32mx/lib/size\libmchp_peripheral_32MX360F512L.a(int_tbl_lib.o)
 .debug_pubnames
                0x0000392c       0x2a C:/Program Files/Microchip/mplabc32/v1.12/bin/../lib/gcc/pic32mx/3.4.4/../../../../pic32mx/lib/size\libmchp_peripheral_32MX360F512L.a(_rtcc_set_time_and_date_lib.o)
 .debug_pubnames
                0x00003956       0x3e C:/Program Files/Microchip/mplabc32/v1.12/bin/../lib/gcc/pic32mx/3.4.4/../../../../pic32mx/lib/size\libmchp_peripheral_32MX360F512L.a(_rtcc_wait_clock_off_lib.o)
 .debug_pubnames
                0x00003994       0x24 C:/Program Files/Microchip/mplabc32/v1.12/bin/../lib/gcc/pic32mx/3.4.4/../../../../pic32mx/lib/size\libmchp_peripheral_32MX360F512L.a(read_core_timer_lib.o)

.debug_info     0x00000000    0x25f3e
 *(.debug_info .gnu.linkonce.wi.*)
 .debug_info    0x00000000     0x1373 output_pic32_ssd1963\MainDemo.o
 .debug_info    0x00001373      0x811 output_pic32_ssd1963\rtcc.o
 .debug_info    0x00001b84      0x52e output_pic32_ssd1963\Fonts.o
 .debug_info    0x000020b2      0xc03 output_pic32_ssd1963\DemoSelection.o
 .debug_info    0x00002cb5      0xbf8 output_pic32_ssd1963\Animation.o
 .debug_info    0x000038ad      0x579 output_pic32_ssd1963\AnimationBitmaps.o
 .debug_info    0x00003e26      0xf17 output_pic32_ssd1963\ECG.o
 .debug_info    0x00004d3d      0xe0d output_pic32_ssd1963\Games.o
 .debug_info    0x00005b4a      0x53f output_pic32_ssd1963\SnakeBitmaps.o
 .debug_info    0x00006089      0x505 output_pic32_ssd1963\ECGBitmaps.o
 .debug_info    0x0000658e     0x1192 output_pic32_ssd1963\RGBDemo.o
 .debug_info    0x00007720      0xc7c output_pic32_ssd1963\MultiFontsDemo.o
 .debug_info    0x0000839c      0x592 output_pic32_ssd1963\HelloWorldFonts.o
 .debug_info    0x0000892e      0xfbc output_pic32_ssd1963\TimeDateDemo.o
 .debug_info    0x000098ea      0x835 output_pic32_ssd1963\DrawTool.o
 .debug_info    0x0000a11f      0x96c output_pic32_ssd1963\SlideShowDemo.o
 .debug_info    0x0000aa8b      0x575 output_pic32_ssd1963\Icons.o
 .debug_info    0x0000b000      0x5be output_pic32_ssd1963\DemoSteps.o
 .debug_info    0x0000b5be      0x704 output_pic32_ssd1963\SideButtons.o
 .debug_info    0x0000bcc2      0x414 output_pic32_ssd1963\BitmapFile.o
 .debug_info    0x0000c0d6     0x107f output_pic32_ssd1963\GraphShow.o
 .debug_info    0x0000d155     0x2e2b output_pic32_ssd1963\FSIO.o
 .debug_info    0x0000ff80      0xcb6 output_pic32_ssd1963\SD-SPI.o
 .debug_info    0x00010c36     0x125e output_pic32_ssd1963\JpegDecoder.o
 .debug_info    0x00011e94      0xb4c output_pic32_ssd1963\BmpDecoder.o
 .debug_info    0x000129e0      0xd90 output_pic32_ssd1963\GifDecoder.o
 .debug_info    0x00013770      0xa0b output_pic32_ssd1963\ImageDecoder.o
 .debug_info    0x0001417b      0x1f7 output_pic32_ssd1963\jidctint.o
 .debug_info    0x00014372      0xb29 output_pic32_ssd1963\TouchScreen.o
 .debug_info    0x00014e9b      0x532 output_pic32_ssd1963\Beep.o
 .debug_info    0x000153cd      0xcba output_pic32_ssd1963\EEPROM.o
 .debug_info    0x00016087      0x902 output_pic32_ssd1963\Window.o
 .debug_info    0x00016989      0x9e5 output_pic32_ssd1963\Button.o
 .debug_info    0x0001736e     0x15d1 output_pic32_ssd1963\Chart.o
 .debug_info    0x0001893f      0x91d output_pic32_ssd1963\CheckBox.o
 .debug_info    0x0001925c      0xe51 output_pic32_ssd1963\DisplayDriver.o
 .debug_info    0x0001a0ad      0xa16 output_pic32_ssd1963\EditBox.o
 .debug_info    0x0001aac3      0xa98 output_pic32_ssd1963\Grid.o
 .debug_info    0x0001b55b      0x87d output_pic32_ssd1963\GroupBox.o
 .debug_info    0x0001bdd8      0xc3b output_pic32_ssd1963\ListBox.o
 .debug_info    0x0001ca13     0x11af output_pic32_ssd1963\Meter.o
 .debug_info    0x0001dbc2      0x844 output_pic32_ssd1963\Picture.o
 .debug_info    0x0001e406     0x11a7 output_pic32_ssd1963\Primitive.o
 .debug_info    0x0001f5ad      0xf46 output_pic32_ssd1963\RadioButton.o
 .debug_info    0x000204f3     0x1159 output_pic32_ssd1963\Slider.o
 .debug_info    0x0002164c      0x8e4 output_pic32_ssd1963\StaticText.o
 .debug_info    0x00021f30      0x4ba output_pic32_ssd1963\GOLFontDefault.o
 .debug_info    0x000223ea      0xb1b output_pic32_ssd1963\GOL.o
 .debug_info    0x00022f05      0x6ed output_pic32_ssd1963\uart2.o
 .debug_info    0x000235f2      0x414 output_pic32_ssd1963\JPEGDemo.o
 .debug_info    0x00023a06      0x903 output_pic32_ssd1963\IconsC32.o
 .debug_info    0x00024309      0x54a output_pic32_ssd1963\SlideShowC32.o
 .debug_info    0x00024853      0x8d9 output_pic32_ssd1963\vs1003b.o
 .debug_info    0x0002512c      0x2e5 C:/Program Files/Microchip/mplabc32/v1.12/bin/../lib/gcc/pic32mx/3.4.4/../../../../pic32mx/lib/size\libc.a(ctypef.o)
 .debug_info    0x00025411      0x1f3 C:/Program Files/Microchip/mplabc32/v1.12/bin/../lib/gcc/pic32mx/3.4.4/../../../../pic32mx/lib/size\libc.a(malloc.o)
 .debug_info    0x00025604       0x9d C:/Program Files/Microchip/mplabc32/v1.12/bin/../lib/gcc/pic32mx/3.4.4/../../../../pic32mx/lib/size\libc.a(rand.o)
 .debug_info    0x000256a1       0x88 C:/Program Files/Microchip/mplabc32/v1.12/bin/../lib/gcc/pic32mx/3.4.4/../../../../pic32mx/lib/size\libc.a(strchr.o)
 .debug_info    0x00025729       0xab C:/Program Files/Microchip/mplabc32/v1.12/bin/../lib/gcc/pic32mx/3.4.4/../../../../pic32mx/lib/size\libc.a(strncpy.o)
 .debug_info    0x000257d4      0x282 C:/Program Files/Microchip/mplabc32/v1.12/bin/../lib/gcc/pic32mx/3.4.4/../../../../pic32mx/lib/size\libc.a(sbrk.o)
 .debug_info    0x00025a56       0x31 C:/Program Files/Microchip/mplabc32/v1.12/bin/../lib/gcc/pic32mx/3.4.4/../../../../pic32mx/lib/size\libc.a(default-general-exception-handler.o)
 .debug_info    0x00025a87       0x31 C:/Program Files/Microchip/mplabc32/v1.12/bin/../lib/gcc/pic32mx/3.4.4/../../../../pic32mx/lib/size\libc.a(default-bootstrap-exception-handler.o)
 .debug_info    0x00025ab8       0x31 C:/Program Files/Microchip/mplabc32/v1.12/bin/../lib/gcc/pic32mx/3.4.4/../../../../pic32mx/lib/size\libc.a(default-on-reset.o)
 .debug_info    0x00025ae9       0x31 C:/Program Files/Microchip/mplabc32/v1.12/bin/../lib/gcc/pic32mx/3.4.4/../../../../pic32mx/lib/size\libc.a(default-on-bootstrap.o)
 .debug_info    0x00025b1a       0x61 C:/Program Files/Microchip/mplabc32/v1.12/bin/../lib/gcc/pic32mx/3.4.4/../../../../pic32mx/lib/size\libc.a(ctype.o)
 .debug_info    0x00025b7b       0x3f C:/Program Files/Microchip/mplabc32/v1.12/bin/../lib/gcc/pic32mx/3.4.4/../../../../pic32mx/lib/size\libc.a(errno.o)
 .debug_info    0x00025bba       0x30 C:/Program Files/Microchip/mplabc32/v1.12/bin/../lib/gcc/pic32mx/3.4.4/../../../../pic32mx/lib/size\libmchp_peripheral.a(open_core_timer_lib.o)
 .debug_info    0x00025bea       0x42 C:/Program Files/Microchip/mplabc32/v1.12/bin/../lib/gcc/pic32mx/3.4.4/../../../../pic32mx/lib/size\libmchp_peripheral_32MX360F512L.a(pcache.o)
 .debug_info    0x00025c2c       0x30 C:/Program Files/Microchip/mplabc32/v1.12/bin/../lib/gcc/pic32mx/3.4.4/../../../../pic32mx/lib/size\libmchp_peripheral_32MX360F512L.a(int_disable_interrupts_lib.o)
 .debug_info    0x00025c5c       0x30 C:/Program Files/Microchip/mplabc32/v1.12/bin/../lib/gcc/pic32mx/3.4.4/../../../../pic32mx/lib/size\libmchp_peripheral_32MX360F512L.a(int_restore_interrupts_lib.o)
 .debug_info    0x00025c8c       0x30 C:/Program Files/Microchip/mplabc32/v1.12/bin/../lib/gcc/pic32mx/3.4.4/../../../../pic32mx/lib/size\libmchp_peripheral_32MX360F512L.a(int_enable_mv_int_lib.o)
 .debug_info    0x00025cbc       0x30 C:/Program Files/Microchip/mplabc32/v1.12/bin/../lib/gcc/pic32mx/3.4.4/../../../../pic32mx/lib/size\libmchp_peripheral_32MX360F512L.a(rtcc_init_lib.o)
 .debug_info    0x00025cec       0x30 C:/Program Files/Microchip/mplabc32/v1.12/bin/../lib/gcc/pic32mx/3.4.4/../../../../pic32mx/lib/size\libmchp_peripheral_32MX360F512L.a(rtcc_set_date_lib.o)
 .debug_info    0x00025d1c       0x30 C:/Program Files/Microchip/mplabc32/v1.12/bin/../lib/gcc/pic32mx/3.4.4/../../../../pic32mx/lib/size\libmchp_peripheral_32MX360F512L.a(rtcc_set_time_lib.o)
 .debug_info    0x00025d4c       0x30 C:/Program Files/Microchip/mplabc32/v1.12/bin/../lib/gcc/pic32mx/3.4.4/../../../../pic32mx/lib/size\libmchp_peripheral_32MX360F512L.a(spi_getc_spi2_lib_legacy.o)
 .debug_info    0x00025d7c       0x30 C:/Program Files/Microchip/mplabc32/v1.12/bin/../lib/gcc/pic32mx/3.4.4/../../../../pic32mx/lib/size\libmchp_peripheral_32MX360F512L.a(spi_open_spi2_lib_legacy.o)
 .debug_info    0x00025dac        0x0 C:/Program Files/Microchip/mplabc32/v1.12/bin/../lib/gcc/pic32mx/3.4.4/../../../../pic32mx/lib/size\libmchp_peripheral_32MX360F512L.a(spi_brg_tbl_lib_legacy.o)
 .debug_info    0x00025dac       0x30 C:/Program Files/Microchip/mplabc32/v1.12/bin/../lib/gcc/pic32mx/3.4.4/../../../../pic32mx/lib/size\libmchp_peripheral_32MX360F512L.a(int_enable_interrupts_lib.o)
 .debug_info    0x00025ddc       0xc0 C:/Program Files/Microchip/mplabc32/v1.12/bin/../lib/gcc/pic32mx/3.4.4/../../../../pic32mx/lib/size\libmchp_peripheral_32MX360F512L.a(int_tbl_lib.o)
 .debug_info    0x00025e9c       0x30 C:/Program Files/Microchip/mplabc32/v1.12/bin/../lib/gcc/pic32mx/3.4.4/../../../../pic32mx/lib/size\libmchp_peripheral_32MX360F512L.a(_rtcc_set_time_and_date_lib.o)
 .debug_info    0x00025ecc       0x42 C:/Program Files/Microchip/mplabc32/v1.12/bin/../lib/gcc/pic32mx/3.4.4/../../../../pic32mx/lib/size\libmchp_peripheral_32MX360F512L.a(_rtcc_wait_clock_off_lib.o)
 .debug_info    0x00025f0e       0x30 C:/Program Files/Microchip/mplabc32/v1.12/bin/../lib/gcc/pic32mx/3.4.4/../../../../pic32mx/lib/size\libmchp_peripheral_32MX360F512L.a(read_core_timer_lib.o)

.debug_abbrev   0x00000000     0x6f3d
 *(.debug_abbrev)
 .debug_abbrev  0x00000000      0x2f9 output_pic32_ssd1963\MainDemo.o
 .debug_abbrev  0x000002f9      0x26f output_pic32_ssd1963\rtcc.o
 .debug_abbrev  0x00000568      0x164 output_pic32_ssd1963\Fonts.o
 .debug_abbrev  0x000006cc      0x218 output_pic32_ssd1963\DemoSelection.o
 .debug_abbrev  0x000008e4      0x1f2 output_pic32_ssd1963\Animation.o
 .debug_abbrev  0x00000ad6      0x164 output_pic32_ssd1963\AnimationBitmaps.o
 .debug_abbrev  0x00000c3a      0x238 output_pic32_ssd1963\ECG.o
 .debug_abbrev  0x00000e72      0x263 output_pic32_ssd1963\Games.o
 .debug_abbrev  0x000010d5      0x164 output_pic32_ssd1963\SnakeBitmaps.o
 .debug_abbrev  0x00001239      0x164 output_pic32_ssd1963\ECGBitmaps.o
 .debug_abbrev  0x0000139d      0x1f2 output_pic32_ssd1963\RGBDemo.o
 .debug_abbrev  0x0000158f      0x219 output_pic32_ssd1963\MultiFontsDemo.o
 .debug_abbrev  0x000017a8      0x164 output_pic32_ssd1963\HelloWorldFonts.o
 .debug_abbrev  0x0000190c      0x2a7 output_pic32_ssd1963\TimeDateDemo.o
 .debug_abbrev  0x00001bb3      0x1cb output_pic32_ssd1963\DrawTool.o
 .debug_abbrev  0x00001d7e      0x1d5 output_pic32_ssd1963\SlideShowDemo.o
 .debug_abbrev  0x00001f53      0x164 output_pic32_ssd1963\Icons.o
 .debug_abbrev  0x000020b7      0x198 output_pic32_ssd1963\DemoSteps.o
 .debug_abbrev  0x0000224f      0x18c output_pic32_ssd1963\SideButtons.o
 .debug_abbrev  0x000023db      0x12b output_pic32_ssd1963\BitmapFile.o
 .debug_abbrev  0x00002506      0x216 output_pic32_ssd1963\GraphShow.o
 .debug_abbrev  0x0000271c      0x2a1 output_pic32_ssd1963\FSIO.o
 .debug_abbrev  0x000029bd      0x2c7 output_pic32_ssd1963\SD-SPI.o
 .debug_abbrev  0x00002c84      0x25a output_pic32_ssd1963\JpegDecoder.o
 .debug_abbrev  0x00002ede      0x229 output_pic32_ssd1963\BmpDecoder.o
 .debug_abbrev  0x00003107      0x26a output_pic32_ssd1963\GifDecoder.o
 .debug_abbrev  0x00003371      0x23f output_pic32_ssd1963\ImageDecoder.o
 .debug_abbrev  0x000035b0       0x9d output_pic32_ssd1963\jidctint.o
 .debug_abbrev  0x0000364d      0x20d output_pic32_ssd1963\TouchScreen.o
 .debug_abbrev  0x0000385a      0x162 output_pic32_ssd1963\Beep.o
 .debug_abbrev  0x000039bc      0x2bd output_pic32_ssd1963\EEPROM.o
 .debug_abbrev  0x00003c79      0x1b4 output_pic32_ssd1963\Window.o
 .debug_abbrev  0x00003e2d      0x1f6 output_pic32_ssd1963\Button.o
 .debug_abbrev  0x00004023      0x268 output_pic32_ssd1963\Chart.o
 .debug_abbrev  0x0000428b      0x1b4 output_pic32_ssd1963\CheckBox.o
 .debug_abbrev  0x0000443f      0x25e output_pic32_ssd1963\DisplayDriver.o
 .debug_abbrev  0x0000469d      0x1b4 output_pic32_ssd1963\EditBox.o
 .debug_abbrev  0x00004851      0x1eb output_pic32_ssd1963\Grid.o
 .debug_abbrev  0x00004a3c      0x1aa output_pic32_ssd1963\GroupBox.o
 .debug_abbrev  0x00004be6      0x23a output_pic32_ssd1963\ListBox.o
 .debug_abbrev  0x00004e20      0x293 output_pic32_ssd1963\Meter.o
 .debug_abbrev  0x000050b3      0x18e output_pic32_ssd1963\Picture.o
 .debug_abbrev  0x00005241      0x296 output_pic32_ssd1963\Primitive.o
 .debug_abbrev  0x000054d7      0x273 output_pic32_ssd1963\RadioButton.o
 .debug_abbrev  0x0000574a      0x277 output_pic32_ssd1963\Slider.o
 .debug_abbrev  0x000059c1      0x1c1 output_pic32_ssd1963\StaticText.o
 .debug_abbrev  0x00005b82      0x164 output_pic32_ssd1963\GOLFontDefault.o
 .debug_abbrev  0x00005ce6      0x24b output_pic32_ssd1963\GOL.o
 .debug_abbrev  0x00005f31      0x247 output_pic32_ssd1963\uart2.o
 .debug_abbrev  0x00006178      0x12b output_pic32_ssd1963\JPEGDemo.o
 .debug_abbrev  0x000062a3      0x17e output_pic32_ssd1963\IconsC32.o
 .debug_abbrev  0x00006421      0x17e output_pic32_ssd1963\SlideShowC32.o
 .debug_abbrev  0x0000659f      0x22d output_pic32_ssd1963\vs1003b.o
 .debug_abbrev  0x000067cc       0x74 C:/Program Files/Microchip/mplabc32/v1.12/bin/../lib/gcc/pic32mx/3.4.4/../../../../pic32mx/lib/size\libc.a(ctypef.o)
 .debug_abbrev  0x00006840      0x136 C:/Program Files/Microchip/mplabc32/v1.12/bin/../lib/gcc/pic32mx/3.4.4/../../../../pic32mx/lib/size\libc.a(malloc.o)
 .debug_abbrev  0x00006976       0x72 C:/Program Files/Microchip/mplabc32/v1.12/bin/../lib/gcc/pic32mx/3.4.4/../../../../pic32mx/lib/size\libc.a(rand.o)
 .debug_abbrev  0x000069e8       0x5e C:/Program Files/Microchip/mplabc32/v1.12/bin/../lib/gcc/pic32mx/3.4.4/../../../../pic32mx/lib/size\libc.a(strchr.o)
 .debug_abbrev  0x00006a46       0x89 C:/Program Files/Microchip/mplabc32/v1.12/bin/../lib/gcc/pic32mx/3.4.4/../../../../pic32mx/lib/size\libc.a(strncpy.o)
 .debug_abbrev  0x00006acf      0x153 C:/Program Files/Microchip/mplabc32/v1.12/bin/../lib/gcc/pic32mx/3.4.4/../../../../pic32mx/lib/size\libc.a(sbrk.o)
 .debug_abbrev  0x00006c22       0x25 C:/Program Files/Microchip/mplabc32/v1.12/bin/../lib/gcc/pic32mx/3.4.4/../../../../pic32mx/lib/size\libc.a(default-general-exception-handler.o)
 .debug_abbrev  0x00006c47       0x25 C:/Program Files/Microchip/mplabc32/v1.12/bin/../lib/gcc/pic32mx/3.4.4/../../../../pic32mx/lib/size\libc.a(default-bootstrap-exception-handler.o)
 .debug_abbrev  0x00006c6c       0x25 C:/Program Files/Microchip/mplabc32/v1.12/bin/../lib/gcc/pic32mx/3.4.4/../../../../pic32mx/lib/size\libc.a(default-on-reset.o)
 .debug_abbrev  0x00006c91       0x25 C:/Program Files/Microchip/mplabc32/v1.12/bin/../lib/gcc/pic32mx/3.4.4/../../../../pic32mx/lib/size\libc.a(default-on-bootstrap.o)
 .debug_abbrev  0x00006cb6       0x49 C:/Program Files/Microchip/mplabc32/v1.12/bin/../lib/gcc/pic32mx/3.4.4/../../../../pic32mx/lib/size\libc.a(ctype.o)
 .debug_abbrev  0x00006cff       0x30 C:/Program Files/Microchip/mplabc32/v1.12/bin/../lib/gcc/pic32mx/3.4.4/../../../../pic32mx/lib/size\libc.a(errno.o)
 .debug_abbrev  0x00006d2f       0x23 C:/Program Files/Microchip/mplabc32/v1.12/bin/../lib/gcc/pic32mx/3.4.4/../../../../pic32mx/lib/size\libmchp_peripheral.a(open_core_timer_lib.o)
 .debug_abbrev  0x00006d52       0x23 C:/Program Files/Microchip/mplabc32/v1.12/bin/../lib/gcc/pic32mx/3.4.4/../../../../pic32mx/lib/size\libmchp_peripheral_32MX360F512L.a(pcache.o)
 .debug_abbrev  0x00006d75       0x23 C:/Program Files/Microchip/mplabc32/v1.12/bin/../lib/gcc/pic32mx/3.4.4/../../../../pic32mx/lib/size\libmchp_peripheral_32MX360F512L.a(int_disable_interrupts_lib.o)
 .debug_abbrev  0x00006d98       0x23 C:/Program Files/Microchip/mplabc32/v1.12/bin/../lib/gcc/pic32mx/3.4.4/../../../../pic32mx/lib/size\libmchp_peripheral_32MX360F512L.a(int_restore_interrupts_lib.o)
 .debug_abbrev  0x00006dbb       0x23 C:/Program Files/Microchip/mplabc32/v1.12/bin/../lib/gcc/pic32mx/3.4.4/../../../../pic32mx/lib/size\libmchp_peripheral_32MX360F512L.a(int_enable_mv_int_lib.o)
 .debug_abbrev  0x00006dde       0x23 C:/Program Files/Microchip/mplabc32/v1.12/bin/../lib/gcc/pic32mx/3.4.4/../../../../pic32mx/lib/size\libmchp_peripheral_32MX360F512L.a(rtcc_init_lib.o)
 .debug_abbrev  0x00006e01       0x23 C:/Program Files/Microchip/mplabc32/v1.12/bin/../lib/gcc/pic32mx/3.4.4/../../../../pic32mx/lib/size\libmchp_peripheral_32MX360F512L.a(rtcc_set_date_lib.o)
 .debug_abbrev  0x00006e24       0x23 C:/Program Files/Microchip/mplabc32/v1.12/bin/../lib/gcc/pic32mx/3.4.4/../../../../pic32mx/lib/size\libmchp_peripheral_32MX360F512L.a(rtcc_set_time_lib.o)
 .debug_abbrev  0x00006e47       0x23 C:/Program Files/Microchip/mplabc32/v1.12/bin/../lib/gcc/pic32mx/3.4.4/../../../../pic32mx/lib/size\libmchp_peripheral_32MX360F512L.a(spi_getc_spi2_lib_legacy.o)
 .debug_abbrev  0x00006e6a       0x23 C:/Program Files/Microchip/mplabc32/v1.12/bin/../lib/gcc/pic32mx/3.4.4/../../../../pic32mx/lib/size\libmchp_peripheral_32MX360F512L.a(spi_open_spi2_lib_legacy.o)
 .debug_abbrev  0x00006e8d        0x1 C:/Program Files/Microchip/mplabc32/v1.12/bin/../lib/gcc/pic32mx/3.4.4/../../../../pic32mx/lib/size\libmchp_peripheral_32MX360F512L.a(spi_brg_tbl_lib_legacy.o)
 .debug_abbrev  0x00006e8e       0x23 C:/Program Files/Microchip/mplabc32/v1.12/bin/../lib/gcc/pic32mx/3.4.4/../../../../pic32mx/lib/size\libmchp_peripheral_32MX360F512L.a(int_enable_interrupts_lib.o)
 .debug_abbrev  0x00006eb1       0x23 C:/Program Files/Microchip/mplabc32/v1.12/bin/../lib/gcc/pic32mx/3.4.4/../../../../pic32mx/lib/size\libmchp_peripheral_32MX360F512L.a(int_tbl_lib.o)
 .debug_abbrev  0x00006ed4       0x23 C:/Program Files/Microchip/mplabc32/v1.12/bin/../lib/gcc/pic32mx/3.4.4/../../../../pic32mx/lib/size\libmchp_peripheral_32MX360F512L.a(_rtcc_set_time_and_date_lib.o)
 .debug_abbrev  0x00006ef7       0x23 C:/Program Files/Microchip/mplabc32/v1.12/bin/../lib/gcc/pic32mx/3.4.4/../../../../pic32mx/lib/size\libmchp_peripheral_32MX360F512L.a(_rtcc_wait_clock_off_lib.o)
 .debug_abbrev  0x00006f1a       0x23 C:/Program Files/Microchip/mplabc32/v1.12/bin/../lib/gcc/pic32mx/3.4.4/../../../../pic32mx/lib/size\libmchp_peripheral_32MX360F512L.a(read_core_timer_lib.o)

.debug_line     0x00000000     0xd291
 *(.debug_line)
 .debug_line    0x00000000      0x3ff output_pic32_ssd1963\MainDemo.o
 .debug_line    0x000003ff      0x2d0 output_pic32_ssd1963\rtcc.o
 .debug_line    0x000006cf      0x173 output_pic32_ssd1963\Fonts.o
 .debug_line    0x00000842      0x364 output_pic32_ssd1963\DemoSelection.o
 .debug_line    0x00000ba6      0x2d2 output_pic32_ssd1963\Animation.o
 .debug_line    0x00000e78      0x17e output_pic32_ssd1963\AnimationBitmaps.o
 .debug_line    0x00000ff6      0x489 output_pic32_ssd1963\ECG.o
 .debug_line    0x0000147f      0x3ac output_pic32_ssd1963\Games.o
 .debug_line    0x0000182b      0x17a output_pic32_ssd1963\SnakeBitmaps.o
 .debug_line    0x000019a5      0x178 output_pic32_ssd1963\ECGBitmaps.o
 .debug_line    0x00001b1d      0x672 output_pic32_ssd1963\RGBDemo.o
 .debug_line    0x0000218f      0x2f1 output_pic32_ssd1963\MultiFontsDemo.o
 .debug_line    0x00002480      0x17d output_pic32_ssd1963\HelloWorldFonts.o
 .debug_line    0x000025fd      0x43c output_pic32_ssd1963\TimeDateDemo.o
 .debug_line    0x00002a39      0x25d output_pic32_ssd1963\DrawTool.o
 .debug_line    0x00002c96      0x25b output_pic32_ssd1963\SlideShowDemo.o
 .debug_line    0x00002ef1      0x173 output_pic32_ssd1963\Icons.o
 .debug_line    0x00003064      0x1b2 output_pic32_ssd1963\DemoSteps.o
 .debug_line    0x00003216      0x1cb output_pic32_ssd1963\SideButtons.o
 .debug_line    0x000033e1      0x13a output_pic32_ssd1963\BitmapFile.o
 .debug_line    0x0000351b      0x38c output_pic32_ssd1963\GraphShow.o
 .debug_line    0x000038a7     0x13fe output_pic32_ssd1963\FSIO.o
 .debug_line    0x00004ca5      0x359 output_pic32_ssd1963\SD-SPI.o
 .debug_line    0x00004ffe      0x5d8 output_pic32_ssd1963\JpegDecoder.o
 .debug_line    0x000055d6      0x4e6 output_pic32_ssd1963\BmpDecoder.o
 .debug_line    0x00005abc      0x475 output_pic32_ssd1963\GifDecoder.o
 .debug_line    0x00005f31      0x2c8 output_pic32_ssd1963\ImageDecoder.o
 .debug_line    0x000061f9      0x172 output_pic32_ssd1963\jidctint.o
 .debug_line    0x0000636b      0x421 output_pic32_ssd1963\TouchScreen.o
 .debug_line    0x0000678c      0x178 output_pic32_ssd1963\Beep.o
 .debug_line    0x00006904      0x21a output_pic32_ssd1963\EEPROM.o
 .debug_line    0x00006b1e      0x2c3 output_pic32_ssd1963\Window.o
 .debug_line    0x00006de1      0x355 output_pic32_ssd1963\Button.o
 .debug_line    0x00007136      0xc0b output_pic32_ssd1963\Chart.o
 .debug_line    0x00007d41      0x2d5 output_pic32_ssd1963\CheckBox.o
 .debug_line    0x00008016      0x4cf output_pic32_ssd1963\DisplayDriver.o
 .debug_line    0x000084e5      0x2e0 output_pic32_ssd1963\EditBox.o
 .debug_line    0x000087c5      0x34e output_pic32_ssd1963\Grid.o
 .debug_line    0x00008b13      0x2b9 output_pic32_ssd1963\GroupBox.o
 .debug_line    0x00008dcc      0x428 output_pic32_ssd1963\ListBox.o
 .debug_line    0x000091f4      0x42b output_pic32_ssd1963\Meter.o
 .debug_line    0x0000961f      0x271 output_pic32_ssd1963\Picture.o
 .debug_line    0x00009890      0x507 output_pic32_ssd1963\Primitive.o
 .debug_line    0x00009d97      0x30d output_pic32_ssd1963\RadioButton.o
 .debug_line    0x0000a0a4      0x44e output_pic32_ssd1963\Slider.o
 .debug_line    0x0000a4f2      0x2c3 output_pic32_ssd1963\StaticText.o
 .debug_line    0x0000a7b5      0x192 output_pic32_ssd1963\GOLFontDefault.o
 .debug_line    0x0000a947      0x4ba output_pic32_ssd1963\GOL.o
 .debug_line    0x0000ae01      0x1f8 output_pic32_ssd1963\uart2.o
 .debug_line    0x0000aff9      0x13a output_pic32_ssd1963\JPEGDemo.o
 .debug_line    0x0000b133      0x176 output_pic32_ssd1963\IconsC32.o
 .debug_line    0x0000b2a9      0x17a output_pic32_ssd1963\SlideShowC32.o
 .debug_line    0x0000b423      0x1e8 output_pic32_ssd1963\vs1003b.o
 .debug_line    0x0000b60b      0x254 C:/Program Files/Microchip/mplabc32/v1.12/bin/../lib/gcc/pic32mx/3.4.4/../../../../pic32mx/lib/size\libc.a(ctypef.o)
 .debug_line    0x0000b85f      0x25b C:/Program Files/Microchip/mplabc32/v1.12/bin/../lib/gcc/pic32mx/3.4.4/../../../../pic32mx/lib/size\libc.a(malloc.o)
 .debug_line    0x0000baba      0x1b9 C:/Program Files/Microchip/mplabc32/v1.12/bin/../lib/gcc/pic32mx/3.4.4/../../../../pic32mx/lib/size\libc.a(rand.o)
 .debug_line    0x0000bc73      0x1a1 C:/Program Files/Microchip/mplabc32/v1.12/bin/../lib/gcc/pic32mx/3.4.4/../../../../pic32mx/lib/size\libc.a(strchr.o)
 .debug_line    0x0000be14      0x1a7 C:/Program Files/Microchip/mplabc32/v1.12/bin/../lib/gcc/pic32mx/3.4.4/../../../../pic32mx/lib/size\libc.a(strncpy.o)
 .debug_line    0x0000bfbb      0x3a9 C:/Program Files/Microchip/mplabc32/v1.12/bin/../lib/gcc/pic32mx/3.4.4/../../../../pic32mx/lib/size\libc.a(sbrk.o)
 .debug_line    0x0000c364       0xba C:/Program Files/Microchip/mplabc32/v1.12/bin/../lib/gcc/pic32mx/3.4.4/../../../../pic32mx/lib/size\libc.a(default-general-exception-handler.o)
 .debug_line    0x0000c41e       0xbc C:/Program Files/Microchip/mplabc32/v1.12/bin/../lib/gcc/pic32mx/3.4.4/../../../../pic32mx/lib/size\libc.a(default-bootstrap-exception-handler.o)
 .debug_line    0x0000c4da       0xa9 C:/Program Files/Microchip/mplabc32/v1.12/bin/../lib/gcc/pic32mx/3.4.4/../../../../pic32mx/lib/size\libc.a(default-on-reset.o)
 .debug_line    0x0000c583       0xad C:/Program Files/Microchip/mplabc32/v1.12/bin/../lib/gcc/pic32mx/3.4.4/../../../../pic32mx/lib/size\libc.a(default-on-bootstrap.o)
 .debug_line    0x0000c630      0x102 C:/Program Files/Microchip/mplabc32/v1.12/bin/../lib/gcc/pic32mx/3.4.4/../../../../pic32mx/lib/size\libc.a(ctype.o)
 .debug_line    0x0000c732      0x17c C:/Program Files/Microchip/mplabc32/v1.12/bin/../lib/gcc/pic32mx/3.4.4/../../../../pic32mx/lib/size\libc.a(errno.o)
 .debug_line    0x0000c8ae       0xa9 C:/Program Files/Microchip/mplabc32/v1.12/bin/../lib/gcc/pic32mx/3.4.4/../../../../pic32mx/lib/size\libmchp_peripheral.a(open_core_timer_lib.o)
 .debug_line    0x0000c957       0x9d C:/Program Files/Microchip/mplabc32/v1.12/bin/../lib/gcc/pic32mx/3.4.4/../../../../pic32mx/lib/size\libmchp_peripheral_32MX360F512L.a(pcache.o)
 .debug_line    0x0000c9f4       0xae C:/Program Files/Microchip/mplabc32/v1.12/bin/../lib/gcc/pic32mx/3.4.4/../../../../pic32mx/lib/size\libmchp_peripheral_32MX360F512L.a(int_disable_interrupts_lib.o)
 .debug_line    0x0000caa2       0xae C:/Program Files/Microchip/mplabc32/v1.12/bin/../lib/gcc/pic32mx/3.4.4/../../../../pic32mx/lib/size\libmchp_peripheral_32MX360F512L.a(int_restore_interrupts_lib.o)
 .debug_line    0x0000cb50       0xa9 C:/Program Files/Microchip/mplabc32/v1.12/bin/../lib/gcc/pic32mx/3.4.4/../../../../pic32mx/lib/size\libmchp_peripheral_32MX360F512L.a(int_enable_mv_int_lib.o)
 .debug_line    0x0000cbf9       0xa2 C:/Program Files/Microchip/mplabc32/v1.12/bin/../lib/gcc/pic32mx/3.4.4/../../../../pic32mx/lib/size\libmchp_peripheral_32MX360F512L.a(rtcc_init_lib.o)
 .debug_line    0x0000cc9b       0xa6 C:/Program Files/Microchip/mplabc32/v1.12/bin/../lib/gcc/pic32mx/3.4.4/../../../../pic32mx/lib/size\libmchp_peripheral_32MX360F512L.a(rtcc_set_date_lib.o)
 .debug_line    0x0000cd41       0xa6 C:/Program Files/Microchip/mplabc32/v1.12/bin/../lib/gcc/pic32mx/3.4.4/../../../../pic32mx/lib/size\libmchp_peripheral_32MX360F512L.a(rtcc_set_time_lib.o)
 .debug_line    0x0000cde7       0xac C:/Program Files/Microchip/mplabc32/v1.12/bin/../lib/gcc/pic32mx/3.4.4/../../../../pic32mx/lib/size\libmchp_peripheral_32MX360F512L.a(spi_getc_spi2_lib_legacy.o)
 .debug_line    0x0000ce93       0xac C:/Program Files/Microchip/mplabc32/v1.12/bin/../lib/gcc/pic32mx/3.4.4/../../../../pic32mx/lib/size\libmchp_peripheral_32MX360F512L.a(spi_open_spi2_lib_legacy.o)
 .debug_line    0x0000cf3f        0x0 C:/Program Files/Microchip/mplabc32/v1.12/bin/../lib/gcc/pic32mx/3.4.4/../../../../pic32mx/lib/size\libmchp_peripheral_32MX360F512L.a(spi_brg_tbl_lib_legacy.o)
 .debug_line    0x0000cf3f       0xad C:/Program Files/Microchip/mplabc32/v1.12/bin/../lib/gcc/pic32mx/3.4.4/../../../../pic32mx/lib/size\libmchp_peripheral_32MX360F512L.a(int_enable_interrupts_lib.o)
 .debug_line    0x0000cfec       0x9f C:/Program Files/Microchip/mplabc32/v1.12/bin/../lib/gcc/pic32mx/3.4.4/../../../../pic32mx/lib/size\libmchp_peripheral_32MX360F512L.a(int_tbl_lib.o)
 .debug_line    0x0000d08b       0xb0 C:/Program Files/Microchip/mplabc32/v1.12/bin/../lib/gcc/pic32mx/3.4.4/../../../../pic32mx/lib/size\libmchp_peripheral_32MX360F512L.a(_rtcc_set_time_and_date_lib.o)
 .debug_line    0x0000d13b       0xad C:/Program Files/Microchip/mplabc32/v1.12/bin/../lib/gcc/pic32mx/3.4.4/../../../../pic32mx/lib/size\libmchp_peripheral_32MX360F512L.a(_rtcc_wait_clock_off_lib.o)
 .debug_line    0x0000d1e8       0xa9 C:/Program Files/Microchip/mplabc32/v1.12/bin/../lib/gcc/pic32mx/3.4.4/../../../../pic32mx/lib/size\libmchp_peripheral_32MX360F512L.a(read_core_timer_lib.o)

.debug_frame    0x00000000     0x3370
 *(.debug_frame)
 .debug_frame   0x00000000       0xf4 output_pic32_ssd1963\MainDemo.o
 .debug_frame   0x000000f4       0xe8 output_pic32_ssd1963\rtcc.o
 .debug_frame   0x000001dc       0xa4 output_pic32_ssd1963\DemoSelection.o
 .debug_frame   0x00000280       0x80 output_pic32_ssd1963\Animation.o
 .debug_frame   0x00000300      0x154 output_pic32_ssd1963\ECG.o
 .debug_frame   0x00000454       0xd8 output_pic32_ssd1963\Games.o
 .debug_frame   0x0000052c      0x15c output_pic32_ssd1963\RGBDemo.o
 .debug_frame   0x00000688       0xa4 output_pic32_ssd1963\MultiFontsDemo.o
 .debug_frame   0x0000072c       0x90 output_pic32_ssd1963\TimeDateDemo.o
 .debug_frame   0x000007bc       0x98 output_pic32_ssd1963\DrawTool.o
 .debug_frame   0x00000854       0x50 output_pic32_ssd1963\SlideShowDemo.o
 .debug_frame   0x000008a4       0x30 output_pic32_ssd1963\DemoSteps.o
 .debug_frame   0x000008d4       0x2c output_pic32_ssd1963\SideButtons.o
 .debug_frame   0x00000900       0xd4 output_pic32_ssd1963\GraphShow.o
 .debug_frame   0x000009d4      0x844 output_pic32_ssd1963\FSIO.o
 .debug_frame   0x00001218      0x16c output_pic32_ssd1963\SD-SPI.o
 .debug_frame   0x00001384      0x1d4 output_pic32_ssd1963\JpegDecoder.o
 .debug_frame   0x00001558       0x74 output_pic32_ssd1963\BmpDecoder.o
 .debug_frame   0x000015cc      0x1a8 output_pic32_ssd1963\GifDecoder.o
 .debug_frame   0x00001774       0x58 output_pic32_ssd1963\ImageDecoder.o
 .debug_frame   0x000017cc       0x34 output_pic32_ssd1963\jidctint.o
 .debug_frame   0x00001800       0xfc output_pic32_ssd1963\TouchScreen.o
 .debug_frame   0x000018fc       0x38 output_pic32_ssd1963\Beep.o
 .debug_frame   0x00001934      0x150 output_pic32_ssd1963\EEPROM.o
 .debug_frame   0x00001a84       0x90 output_pic32_ssd1963\Window.o
 .debug_frame   0x00001b14       0xac output_pic32_ssd1963\Button.o
 .debug_frame   0x00001bc0      0x1d0 output_pic32_ssd1963\Chart.o
 .debug_frame   0x00001d90       0xac output_pic32_ssd1963\CheckBox.o
 .debug_frame   0x00001e3c      0x2b0 output_pic32_ssd1963\DisplayDriver.o
 .debug_frame   0x000020ec       0xc0 output_pic32_ssd1963\EditBox.o
 .debug_frame   0x000021ac       0xf0 output_pic32_ssd1963\Grid.o
 .debug_frame   0x0000229c       0x70 output_pic32_ssd1963\GroupBox.o
 .debug_frame   0x0000230c      0x13c output_pic32_ssd1963\ListBox.o
 .debug_frame   0x00002448       0xd8 output_pic32_ssd1963\Meter.o
 .debug_frame   0x00002520       0x74 output_pic32_ssd1963\Picture.o
 .debug_frame   0x00002594      0x1dc output_pic32_ssd1963\Primitive.o
 .debug_frame   0x00002770       0xcc output_pic32_ssd1963\RadioButton.o
 .debug_frame   0x0000283c      0x13c output_pic32_ssd1963\Slider.o
 .debug_frame   0x00002978       0x88 output_pic32_ssd1963\StaticText.o
 .debug_frame   0x00002a00      0x18c output_pic32_ssd1963\GOL.o
 .debug_frame   0x00002b8c      0x118 output_pic32_ssd1963\uart2.o
 .debug_frame   0x00002ca4       0xf4 output_pic32_ssd1963\vs1003b.o
 .debug_frame   0x00002d98      0x120 C:/Program Files/Microchip/mplabc32/v1.12/bin/../lib/gcc/pic32mx/3.4.4/../../../../pic32mx/lib/size\libc.a(ctypef.o)
 .debug_frame   0x00002eb8       0x68 C:/Program Files/Microchip/mplabc32/v1.12/bin/../lib/gcc/pic32mx/3.4.4/../../../../pic32mx/lib/size\libc.a(malloc.o)
 .debug_frame   0x00002f20       0x38 C:/Program Files/Microchip/mplabc32/v1.12/bin/../lib/gcc/pic32mx/3.4.4/../../../../pic32mx/lib/size\libc.a(rand.o)
 .debug_frame   0x00002f58       0x20 C:/Program Files/Microchip/mplabc32/v1.12/bin/../lib/gcc/pic32mx/3.4.4/../../../../pic32mx/lib/size\libc.a(strchr.o)
 .debug_frame   0x00002f78       0x20 C:/Program Files/Microchip/mplabc32/v1.12/bin/../lib/gcc/pic32mx/3.4.4/../../../../pic32mx/lib/size\libc.a(strncpy.o)
 .debug_frame   0x00002f98       0x8c C:/Program Files/Microchip/mplabc32/v1.12/bin/../lib/gcc/pic32mx/3.4.4/../../../../pic32mx/lib/size\libc.a(sbrk.o)
 .debug_frame   0x00003024       0x20 C:/Program Files/Microchip/mplabc32/v1.12/bin/../lib/gcc/pic32mx/3.4.4/../../../../pic32mx/lib/size\libc.a(default-general-exception-handler.o)
 .debug_frame   0x00003044       0x20 C:/Program Files/Microchip/mplabc32/v1.12/bin/../lib/gcc/pic32mx/3.4.4/../../../../pic32mx/lib/size\libc.a(default-bootstrap-exception-handler.o)
 .debug_frame   0x00003064       0x20 C:/Program Files/Microchip/mplabc32/v1.12/bin/../lib/gcc/pic32mx/3.4.4/../../../../pic32mx/lib/size\libc.a(default-on-reset.o)
 .debug_frame   0x00003084       0x20 C:/Program Files/Microchip/mplabc32/v1.12/bin/../lib/gcc/pic32mx/3.4.4/../../../../pic32mx/lib/size\libc.a(default-on-bootstrap.o)
 .debug_frame   0x000030a4       0x20 C:/Program Files/Microchip/mplabc32/v1.12/bin/../lib/gcc/pic32mx/3.4.4/../../../../pic32mx/lib/size\libmchp_peripheral.a(open_core_timer_lib.o)
 .debug_frame   0x000030c4       0x30 C:/Program Files/Microchip/mplabc32/v1.12/bin/../lib/gcc/pic32mx/3.4.4/../../../../pic32mx/lib/size\libmchp_peripheral_32MX360F512L.a(pcache.o)
 .debug_frame   0x000030f4       0x20 C:/Program Files/Microchip/mplabc32/v1.12/bin/../lib/gcc/pic32mx/3.4.4/../../../../pic32mx/lib/size\libmchp_peripheral_32MX360F512L.a(int_disable_interrupts_lib.o)
 .debug_frame   0x00003114       0x20 C:/Program Files/Microchip/mplabc32/v1.12/bin/../lib/gcc/pic32mx/3.4.4/../../../../pic32mx/lib/size\libmchp_peripheral_32MX360F512L.a(int_restore_interrupts_lib.o)
 .debug_frame   0x00003134       0x28 C:/Program Files/Microchip/mplabc32/v1.12/bin/../lib/gcc/pic32mx/3.4.4/../../../../pic32mx/lib/size\libmchp_peripheral_32MX360F512L.a(int_enable_mv_int_lib.o)
 .debug_frame   0x0000315c       0x30 C:/Program Files/Microchip/mplabc32/v1.12/bin/../lib/gcc/pic32mx/3.4.4/../../../../pic32mx/lib/size\libmchp_peripheral_32MX360F512L.a(rtcc_init_lib.o)
 .debug_frame   0x0000318c       0x28 C:/Program Files/Microchip/mplabc32/v1.12/bin/../lib/gcc/pic32mx/3.4.4/../../../../pic32mx/lib/size\libmchp_peripheral_32MX360F512L.a(rtcc_set_date_lib.o)
 .debug_frame   0x000031b4       0x28 C:/Program Files/Microchip/mplabc32/v1.12/bin/../lib/gcc/pic32mx/3.4.4/../../../../pic32mx/lib/size\libmchp_peripheral_32MX360F512L.a(rtcc_set_time_lib.o)
 .debug_frame   0x000031dc       0x20 C:/Program Files/Microchip/mplabc32/v1.12/bin/../lib/gcc/pic32mx/3.4.4/../../../../pic32mx/lib/size\libmchp_peripheral_32MX360F512L.a(spi_getc_spi2_lib_legacy.o)
 .debug_frame   0x000031fc       0x20 C:/Program Files/Microchip/mplabc32/v1.12/bin/../lib/gcc/pic32mx/3.4.4/../../../../pic32mx/lib/size\libmchp_peripheral_32MX360F512L.a(spi_open_spi2_lib_legacy.o)
 .debug_frame   0x0000321c       0x20 C:/Program Files/Microchip/mplabc32/v1.12/bin/../lib/gcc/pic32mx/3.4.4/../../../../pic32mx/lib/size\libmchp_peripheral_32MX360F512L.a(int_enable_interrupts_lib.o)
 .debug_frame   0x0000323c       0xa0 C:/Program Files/Microchip/mplabc32/v1.12/bin/../lib/gcc/pic32mx/3.4.4/../../../../pic32mx/lib/size\libmchp_peripheral_32MX360F512L.a(int_tbl_lib.o)
 .debug_frame   0x000032dc       0x34 C:/Program Files/Microchip/mplabc32/v1.12/bin/../lib/gcc/pic32mx/3.4.4/../../../../pic32mx/lib/size\libmchp_peripheral_32MX360F512L.a(_rtcc_set_time_and_date_lib.o)
 .debug_frame   0x00003310       0x40 C:/Program Files/Microchip/mplabc32/v1.12/bin/../lib/gcc/pic32mx/3.4.4/../../../../pic32mx/lib/size\libmchp_peripheral_32MX360F512L.a(_rtcc_wait_clock_off_lib.o)
 .debug_frame   0x00003350       0x20 C:/Program Files/Microchip/mplabc32/v1.12/bin/../lib/gcc/pic32mx/3.4.4/../../../../pic32mx/lib/size\libmchp_peripheral_32MX360F512L.a(read_core_timer_lib.o)

.debug_str      0x00000000     0x78c3
 *(.debug_str)
 .debug_str     0x00000000      0xac3 output_pic32_ssd1963\MainDemo.o
                                0xb92 (size before relaxing)
 .debug_str     0x00000ac3      0x11b output_pic32_ssd1963\rtcc.o
                                0x448 (size before relaxing)
 .debug_str     0x00000bde       0x39 output_pic32_ssd1963\Fonts.o
                                0x381 (size before relaxing)
 .debug_str     0x00000c17      0x2c9 output_pic32_ssd1963\DemoSelection.o
                                0xa26 (size before relaxing)
 .debug_str     0x00000ee0      0x15a output_pic32_ssd1963\Animation.o
                                0x8fc (size before relaxing)
 .debug_str     0x0000103a       0x2f output_pic32_ssd1963\AnimationBitmaps.o
                                0x396 (size before relaxing)
 .debug_str     0x00001069      0x263 output_pic32_ssd1963\ECG.o
                                0x9fd (size before relaxing)
 .debug_str     0x000012cc      0x21e output_pic32_ssd1963\Games.o
                                0x9e4 (size before relaxing)
 .debug_str     0x000014ea       0x24 output_pic32_ssd1963\SnakeBitmaps.o
                                0x37a (size before relaxing)
 .debug_str     0x0000150e       0x1b output_pic32_ssd1963\ECGBitmaps.o
                                0x371 (size before relaxing)
 .debug_str     0x00001529      0x40b output_pic32_ssd1963\RGBDemo.o
                                0xb8d (size before relaxing)
 .debug_str     0x00001934      0x147 output_pic32_ssd1963\MultiFontsDemo.o
                                0x8fb (size before relaxing)
 .debug_str     0x00001a7b       0x5b output_pic32_ssd1963\HelloWorldFonts.o
                                0x39b (size before relaxing)
 .debug_str     0x00001ad6      0x1ff output_pic32_ssd1963\TimeDateDemo.o
                                0x9c9 (size before relaxing)
 .debug_str     0x00001cd5       0x69 output_pic32_ssd1963\DrawTool.o
                                0x72f (size before relaxing)
 .debug_str     0x00001d3e       0xb2 output_pic32_ssd1963\SlideShowDemo.o
                                0x7da (size before relaxing)
 .debug_str     0x00001df0       0x4b output_pic32_ssd1963\Icons.o
                                0x392 (size before relaxing)
 .debug_str     0x00001e3b       0x49 output_pic32_ssd1963\DemoSteps.o
                                0x3c5 (size before relaxing)
 .debug_str     0x00001e84       0x3c output_pic32_ssd1963\SideButtons.o
                                0x534 (size before relaxing)
 .debug_str     0x00001ec0        0xd output_pic32_ssd1963\BitmapFile.o
                                0x311 (size before relaxing)
 .debug_str     0x00001ecd      0x4c0 output_pic32_ssd1963\GraphShow.o
                                0xc27 (size before relaxing)
 .debug_str     0x0000238d      0xfc6 output_pic32_ssd1963\FSIO.o
                               0x1409 (size before relaxing)
 .debug_str     0x00003353      0x431 output_pic32_ssd1963\SD-SPI.o
                                0x7e0 (size before relaxing)
 .debug_str     0x00003784      0x5b3 output_pic32_ssd1963\JpegDecoder.o
                                0x9da (size before relaxing)
 .debug_str     0x00003d37      0x167 output_pic32_ssd1963\BmpDecoder.o
                                0x622 (size before relaxing)
 .debug_str     0x00003e9e      0x3ac output_pic32_ssd1963\GifDecoder.o
                                0x888 (size before relaxing)
 .debug_str     0x0000424a      0x1ac output_pic32_ssd1963\ImageDecoder.o
                                0x69f (size before relaxing)
 .debug_str     0x000043f6       0x95 output_pic32_ssd1963\jidctint.o
                                0x1b8 (size before relaxing)
 .debug_str     0x0000448b      0x220 output_pic32_ssd1963\TouchScreen.o
                                0x656 (size before relaxing)
 .debug_str     0x000046ab       0x99 output_pic32_ssd1963\Beep.o
                                0x3ba (size before relaxing)
 .debug_str     0x00004744      0x157 output_pic32_ssd1963\EEPROM.o
                                0x505 (size before relaxing)
 .debug_str     0x0000489b       0xf7 output_pic32_ssd1963\Window.o
                                0x6ad (size before relaxing)
 .debug_str     0x00004992       0xdf output_pic32_ssd1963\Button.o
                                0x6ef (size before relaxing)
 .debug_str     0x00004a71      0x98f output_pic32_ssd1963\Chart.o
                               0x107e (size before relaxing)
 .debug_str     0x00005400       0x8f output_pic32_ssd1963\CheckBox.o
                                0x685 (size before relaxing)
 .debug_str     0x0000548f      0x24e output_pic32_ssd1963\DisplayDriver.o
                                0x68e (size before relaxing)
 .debug_str     0x000056dd       0xb7 output_pic32_ssd1963\EditBox.o
                                0x6e3 (size before relaxing)
 .debug_str     0x00005794       0xb7 output_pic32_ssd1963\Grid.o
                                0x662 (size before relaxing)
 .debug_str     0x0000584b      0x19b output_pic32_ssd1963\GroupBox.o
                                0x6e0 (size before relaxing)
 .debug_str     0x000059e6      0x19c output_pic32_ssd1963\ListBox.o
                                0x7c9 (size before relaxing)
 .debug_str     0x00005b82      0x16e output_pic32_ssd1963\Meter.o
                                0x886 (size before relaxing)
 .debug_str     0x00005cf0       0xd2 output_pic32_ssd1963\Picture.o
                                0x60e (size before relaxing)
 .debug_str     0x00005dc2      0x214 output_pic32_ssd1963\Primitive.o
                                0x633 (size before relaxing)
 .debug_str     0x00005fd6       0xeb output_pic32_ssd1963\RadioButton.o
                                0x731 (size before relaxing)
 .debug_str     0x000060c1      0x1e3 output_pic32_ssd1963\Slider.o
                                0x816 (size before relaxing)
 .debug_str     0x000062a4       0xda output_pic32_ssd1963\StaticText.o
                                0x66d (size before relaxing)
 .debug_str     0x0000637e       0x2e output_pic32_ssd1963\GOLFontDefault.o
                                0x37d (size before relaxing)
 .debug_str     0x000063ac      0x138 output_pic32_ssd1963\GOL.o
                                0x740 (size before relaxing)
 .debug_str     0x000064e4      0x156 output_pic32_ssd1963\uart2.o
                                0x46c (size before relaxing)
 .debug_str     0x0000663a        0xb output_pic32_ssd1963\JPEGDemo.o
                                0x30f (size before relaxing)
 .debug_str     0x00006645       0x8a output_pic32_ssd1963\IconsC32.o
                                0x540 (size before relaxing)
 .debug_str     0x000066cf       0x22 output_pic32_ssd1963\SlideShowC32.o
                                0x37c (size before relaxing)
 .debug_str     0x000066f1       0xf3 output_pic32_ssd1963\vs1003b.o
                                0x52d (size before relaxing)
 .debug_str     0x000067e4       0xef C:/Program Files/Microchip/mplabc32/v1.12/bin/../lib/gcc/pic32mx/3.4.4/../../../../pic32mx/lib/size\libc.a(ctypef.o)
                                0x14b (size before relaxing)
 .debug_str     0x000068d3       0xc7 C:/Program Files/Microchip/mplabc32/v1.12/bin/../lib/gcc/pic32mx/3.4.4/../../../../pic32mx/lib/size\libc.a(malloc.o)
                                0x157 (size before relaxing)
 .debug_str     0x0000699a       0x7d C:/Program Files/Microchip/mplabc32/v1.12/bin/../lib/gcc/pic32mx/3.4.4/../../../../pic32mx/lib/size\libc.a(rand.o)
                                 0xf6 (size before relaxing)
 .debug_str     0x00006a17       0x74 C:/Program Files/Microchip/mplabc32/v1.12/bin/../lib/gcc/pic32mx/3.4.4/../../../../pic32mx/lib/size\libc.a(strchr.o)
                                 0xe8 (size before relaxing)
 .debug_str     0x00006a8b       0x7b C:/Program Files/Microchip/mplabc32/v1.12/bin/../lib/gcc/pic32mx/3.4.4/../../../../pic32mx/lib/size\libc.a(strncpy.o)
                                 0xfb (size before relaxing)
 .debug_str     0x00006b06       0xec C:/Program Files/Microchip/mplabc32/v1.12/bin/../lib/gcc/pic32mx/3.4.4/../../../../pic32mx/lib/size\libc.a(sbrk.o)
                                0x19d (size before relaxing)
 .debug_str     0x00006bf2       0xa5 C:/Program Files/Microchip/mplabc32/v1.12/bin/../lib/gcc/pic32mx/3.4.4/../../../../pic32mx/lib/size\libc.a(default-general-exception-handler.o)
                                 0xec (size before relaxing)
 .debug_str     0x00006c97       0xa9 C:/Program Files/Microchip/mplabc32/v1.12/bin/../lib/gcc/pic32mx/3.4.4/../../../../pic32mx/lib/size\libc.a(default-bootstrap-exception-handler.o)
                                 0xf0 (size before relaxing)
 .debug_str     0x00006d40       0x83 C:/Program Files/Microchip/mplabc32/v1.12/bin/../lib/gcc/pic32mx/3.4.4/../../../../pic32mx/lib/size\libc.a(default-on-reset.o)
                                 0xca (size before relaxing)
 .debug_str     0x00006dc3       0x8b C:/Program Files/Microchip/mplabc32/v1.12/bin/../lib/gcc/pic32mx/3.4.4/../../../../pic32mx/lib/size\libc.a(default-on-bootstrap.o)
                                 0xd2 (size before relaxing)
 .debug_str     0x00006e4e       0x6c C:/Program Files/Microchip/mplabc32/v1.12/bin/../lib/gcc/pic32mx/3.4.4/../../../../pic32mx/lib/size\libc.a(ctype.o)
                                 0xd1 (size before relaxing)
 .debug_str     0x00006eba       0x6c C:/Program Files/Microchip/mplabc32/v1.12/bin/../lib/gcc/pic32mx/3.4.4/../../../../pic32mx/lib/size\libc.a(errno.o)
                                 0xb9 (size before relaxing)
 .debug_str     0x00006f26       0x97 C:/Program Files/Microchip/mplabc32/v1.12/bin/../lib/gcc/pic32mx/3.4.4/../../../../pic32mx/lib/size\libmchp_peripheral.a(open_core_timer_lib.o)
                                 0xde (size before relaxing)
 .debug_str     0x00006fbd       0x9e C:/Program Files/Microchip/mplabc32/v1.12/bin/../lib/gcc/pic32mx/3.4.4/../../../../pic32mx/lib/size\libmchp_peripheral_32MX360F512L.a(pcache.o)
                                 0xe5 (size before relaxing)
 .debug_str     0x0000705b       0xa3 C:/Program Files/Microchip/mplabc32/v1.12/bin/../lib/gcc/pic32mx/3.4.4/../../../../pic32mx/lib/size\libmchp_peripheral_32MX360F512L.a(int_disable_interrupts_lib.o)
                                 0xea (size before relaxing)
 .debug_str     0x000070fe       0xa3 C:/Program Files/Microchip/mplabc32/v1.12/bin/../lib/gcc/pic32mx/3.4.4/../../../../pic32mx/lib/size\libmchp_peripheral_32MX360F512L.a(int_restore_interrupts_lib.o)
                                 0xea (size before relaxing)
 .debug_str     0x000071a1       0xa9 C:/Program Files/Microchip/mplabc32/v1.12/bin/../lib/gcc/pic32mx/3.4.4/../../../../pic32mx/lib/size\libmchp_peripheral_32MX360F512L.a(int_enable_mv_int_lib.o)
                                 0xf0 (size before relaxing)
 .debug_str     0x0000724a       0x8b C:/Program Files/Microchip/mplabc32/v1.12/bin/../lib/gcc/pic32mx/3.4.4/../../../../pic32mx/lib/size\libmchp_peripheral_32MX360F512L.a(rtcc_init_lib.o)
                                 0xd2 (size before relaxing)
 .debug_str     0x000072d5       0x92 C:/Program Files/Microchip/mplabc32/v1.12/bin/../lib/gcc/pic32mx/3.4.4/../../../../pic32mx/lib/size\libmchp_peripheral_32MX360F512L.a(rtcc_set_date_lib.o)
                                 0xd9 (size before relaxing)
 .debug_str     0x00007367       0x92 C:/Program Files/Microchip/mplabc32/v1.12/bin/../lib/gcc/pic32mx/3.4.4/../../../../pic32mx/lib/size\libmchp_peripheral_32MX360F512L.a(rtcc_set_time_lib.o)
                                 0xd9 (size before relaxing)
 .debug_str     0x000073f9       0x95 C:/Program Files/Microchip/mplabc32/v1.12/bin/../lib/gcc/pic32mx/3.4.4/../../../../pic32mx/lib/size\libmchp_peripheral_32MX360F512L.a(spi_getc_spi2_lib_legacy.o)
                                 0xdc (size before relaxing)
 .debug_str     0x0000748e       0x95 C:/Program Files/Microchip/mplabc32/v1.12/bin/../lib/gcc/pic32mx/3.4.4/../../../../pic32mx/lib/size\libmchp_peripheral_32MX360F512L.a(spi_open_spi2_lib_legacy.o)
                                 0xdc (size before relaxing)
 .debug_str     0x00007523       0xa1 C:/Program Files/Microchip/mplabc32/v1.12/bin/../lib/gcc/pic32mx/3.4.4/../../../../pic32mx/lib/size\libmchp_peripheral_32MX360F512L.a(int_enable_interrupts_lib.o)
                                 0xe8 (size before relaxing)
 .debug_str     0x000075c4      0x113 C:/Program Files/Microchip/mplabc32/v1.12/bin/../lib/gcc/pic32mx/3.4.4/../../../../pic32mx/lib/size\libmchp_peripheral_32MX360F512L.a(int_tbl_lib.o)
                                0x15a (size before relaxing)
 .debug_str     0x000076d7       0xa4 C:/Program Files/Microchip/mplabc32/v1.12/bin/../lib/gcc/pic32mx/3.4.4/../../../../pic32mx/lib/size\libmchp_peripheral_32MX360F512L.a(_rtcc_set_time_and_date_lib.o)
                                 0xeb (size before relaxing)
 .debug_str     0x0000777b       0xb1 C:/Program Files/Microchip/mplabc32/v1.12/bin/../lib/gcc/pic32mx/3.4.4/../../../../pic32mx/lib/size\libmchp_peripheral_32MX360F512L.a(_rtcc_wait_clock_off_lib.o)
                                 0xf8 (size before relaxing)
 .debug_str     0x0000782c       0x97 C:/Program Files/Microchip/mplabc32/v1.12/bin/../lib/gcc/pic32mx/3.4.4/../../../../pic32mx/lib/size\libmchp_peripheral_32MX360F512L.a(read_core_timer_lib.o)
                                 0xde (size before relaxing)

.debug_loc
 *(.debug_loc)

.debug_macinfo  0x00000000     0x8cb5
 *(.debug_macinfo)
 .debug_macinfo
                0x00000000      0xca4 C:/Program Files/Microchip/mplabc32/v1.12/bin/../lib/gcc/pic32mx/3.4.4/../../../../pic32mx/lib/size\libc.a(ctypef.o)
 .debug_macinfo
                0x00000ca4      0xcca C:/Program Files/Microchip/mplabc32/v1.12/bin/../lib/gcc/pic32mx/3.4.4/../../../../pic32mx/lib/size\libc.a(malloc.o)
 .debug_macinfo
                0x0000196e      0xbcc C:/Program Files/Microchip/mplabc32/v1.12/bin/../lib/gcc/pic32mx/3.4.4/../../../../pic32mx/lib/size\libc.a(rand.o)
 .debug_macinfo
                0x0000253a      0xafc C:/Program Files/Microchip/mplabc32/v1.12/bin/../lib/gcc/pic32mx/3.4.4/../../../../pic32mx/lib/size\libc.a(strchr.o)
 .debug_macinfo
                0x00003036      0xafc C:/Program Files/Microchip/mplabc32/v1.12/bin/../lib/gcc/pic32mx/3.4.4/../../../../pic32mx/lib/size\libc.a(strncpy.o)
 .debug_macinfo
                0x00003b32     0x11af C:/Program Files/Microchip/mplabc32/v1.12/bin/../lib/gcc/pic32mx/3.4.4/../../../../pic32mx/lib/size\libc.a(sbrk.o)
 .debug_macinfo
                0x00004ce1      0x945 C:/Program Files/Microchip/mplabc32/v1.12/bin/../lib/gcc/pic32mx/3.4.4/../../../../pic32mx/lib/size\libc.a(default-general-exception-handler.o)
 .debug_macinfo
                0x00005626      0x945 C:/Program Files/Microchip/mplabc32/v1.12/bin/../lib/gcc/pic32mx/3.4.4/../../../../pic32mx/lib/size\libc.a(default-bootstrap-exception-handler.o)
 .debug_macinfo
                0x00005f6b      0x945 C:/Program Files/Microchip/mplabc32/v1.12/bin/../lib/gcc/pic32mx/3.4.4/../../../../pic32mx/lib/size\libc.a(default-on-reset.o)
 .debug_macinfo
                0x000068b0      0x945 C:/Program Files/Microchip/mplabc32/v1.12/bin/../lib/gcc/pic32mx/3.4.4/../../../../pic32mx/lib/size\libc.a(default-on-bootstrap.o)
 .debug_macinfo
                0x000071f5      0xcef C:/Program Files/Microchip/mplabc32/v1.12/bin/../lib/gcc/pic32mx/3.4.4/../../../../pic32mx/lib/size\libc.a(ctype.o)
 .debug_macinfo
                0x00007ee4      0xdd1 C:/Program Files/Microchip/mplabc32/v1.12/bin/../lib/gcc/pic32mx/3.4.4/../../../../pic32mx/lib/size\libc.a(errno.o)

.debug_weaknames
 *(.debug_weaknames)

.debug_funcnames
 *(.debug_funcnames)

.debug_typenames
 *(.debug_typenames)

.debug_varnames
 *(.debug_varnames)
OUTPUT(output_pic32_ssd1963\GMAP SDCard SSD1963 PIC32.elf elf32-tradlittlemips)

.debug_ranges   0x00000000       0x78
 .debug_ranges  0x00000000       0x18 output_pic32_ssd1963\FSIO.o
 .debug_ranges  0x00000018       0x48 output_pic32_ssd1963\BmpDecoder.o
 .debug_ranges  0x00000060       0x18 output_pic32_ssd1963\GifDecoder.o
